:020000040000FA
:0408000090EF07F07E
:020808003BD0E3
:0808180087D0E26BE36BE46B97
:10082000E56BF86A080EF76E000EF66A0900F550DF
:10083000E527E86AE423E323E223FF0EF762F6D715
:10084000FA0EF662F3D7E51FE41FE31FE21FE52B64
:0A085000E86AE423E323E223FFD764
:10088000026ED8CF03F0D9CF05F0DACF04F0E1CF74
:1008900007F0E2CF06F0E9CF09F0EACF08F09EBA00
:1008A0000BD0F2B201D030D0F292A081A0A32CD014
:1008B00091C092F0916B28D0AECFC9F03D8E0A0E58
:1008C000C95D22E00D0EC9630BD06B511DE022EE15
:1008D00000F0D926C9C0DFFF6B6BC9EC5DF014D006
:1008E00022EE00F06B51D926C9C0DFFF6B2B3E0E04
:1008F000C96302D03F8008D03FA006D0200EC96354
:1009000003D03F823F906B6B05C0D9FF04C0DAFF74
:1009100007C0E1FF06C0E2FF09C0E9FF08C0EAFF27
:10092000025003C0D8FF1000006ED8CF01F0E9CF0D
:100930000AF0EACF0BF0A4AA18D0A49A1AEE00F09D
:100940006ECFF7F00A0EF75DD8B4AED2F851E126BB
:10095000F7C0E7FF0D0EF76306D0E12AE76AF86BF0
:1009600081EC67F0A1D2F82B9FD2F0A203D0F092D5
:1009700035809AD2F2A498D2F294AA2F1ED00A0EF1
:10098000AA6FA0B3912B39B002D0809816D083AE55
:10099000808883BE809883AE678983BE67996739F4
:1009A0006719010BE8A009D067A904D067816785A2
:1009B000679303D0679167956783AB67AB07B167B0
:1009C000B107AD5305E0AE0703E1640EAE6FAD07AE
:1009D000AF5305E0B00703E1640EB06FAF07B25349
:1009E00005E0B40703E10A0EB46FB207B35305E0A4
:1009F000B50703E1640EB56FB307B65305E0B7075B
:100A000003E10A0EB76FB607B85305E0B90703E173
:100A1000640EB96FB80760EC07F036B462D036B236
:100A200024D036B00DD035A06FD03590C26BC36BDB
:100A3000366A376A36800A0EB46F050EB26F64D01C
:100A4000B26702D0366A60D035A05ED0359036905D
:100A50003682C26BC46BC36B0A0EB46F140EB26FD6
:100A6000640EB56F2D0EB36F4FD0C22B35B017D0BB
:100A7000B2674AD036923684369636A80CD0358284
:100A8000358635843698640EB56F2D0EB36FC46B02
:100A9000C26BC36B39D035923594359635D03590CD
:100AA0000A0EB46F140EB26F36B605D0C2C0C3F0D2
:100AB000C26B367629D03676C251C327430EC36146
:100AC0000BD00F0EC36508D0C36BC26BC42B050ED1
:100AD000C4651AD0368818D03696C46BC26BC36B07
:100AE00013D0B36704D0366AC00E35160DD035A0CA
:100AF0000BD03590C46BC26BC36B3682369436967E
:100B00000A0EB46F1E0EB26F3AA6E3EF05F03AB0CC
:100B1000BDEF05F03AB2A1EF05F06C2FE3EF05F061
:100B2000140E6C6F80746D2FE3EF05F01D50D8B478
:100B30003A841BC06DF03A828086809480828090D7
:100B400042D06C2FE3EF05F0140E6C6F6D2FE3EFC6
:100B500005F01C5008E06D6F3A923A8080868094D0
:100B60008092808030D01AC06DF03A923A90C52BB6
:100B7000808680948092808026D03AB2D2EF05F0B1
:100B80006C2FE3EF05F0140E6C6F80746D2FE3EFA4
:100B900005F01DC06DF03A823A8480868094808290
:100BA000809011D06C2FE3EF05F0140E6C6F6D2F59
:100BB000E3EF05F01AC06DF03A923A90C52B8086AB
:100BC000809480928080BFAF6FD1010EC06308D047
:100BD000000EC16304D0D8EC61F0C12B65D164D1A3
:100BE000020EC06345D0000EC1630BD0C12BE0C91B
:100BF000E8FFFF0BD8B458D15CEC07F0E3EC61F0F0
:100C000053D1010EC1630DD0B6674ED1C12BE1C9DE
:100C1000E8FFFF0BD8B448D15CEC07F018EC62F0A9
:100C200043D1020EC1630DD0B6673ED1C12BE2C9DC
:100C3000E8FFFF0BD8B438D15CEC07F0E3EC61F0CF
:100C400033D1030EC1630DD0B6672ED1C12BE3C9DA
:100C5000E8FFFF0BD8B428D15CEC07F018EC62F089
:100C600023D1040EC16320D1B6671ED1C16B1CD144
:100C7000030EC06345D0000EC1630BD0C12BE4C985
:100C8000E8FFFF0BD8B410D15CEC07F0EEEC61F09C
:100C90000BD1010EC1630DD0B66706D1C12BE5C9DA
:100CA000E8FFFF0BD8B400D15CEC07F018EC62F061
:100CB000FBD0020EC1630DD0B667F6D0C12BE6C9DA
:100CC000E8FFFF0BD8B4F0D05CEC07F0EEEC61F07D
:100CD000EBD0030EC1630DD0B667E6D0C12BE7C9D8
:100CE000E8FFFF0BD8B4E0D05CEC07F018EC62F042
:100CF000DBD0040EC163D8D0B667D6D0C16BD4D0D8
:100D0000040EC06345D0000EC1630BD0C12BE8C9EF
:100D1000E8FFFF0BD8B4C8D05CEC07F0F9EC61F049
:100D2000C3D0010EC1630DD0B667BED0C12BE9C9D7
:100D3000E8FFFF0BD8B4B8D05CEC07F018EC62F019
:100D4000B3D0020EC1630DD0B667AED0C12BEAC9D5
:100D5000E8FFFF0BD8B4A8D05CEC07F0F9EC61F029
:100D6000A3D0030EC1630DD0B6679ED0C12BEBC9D3
:100D7000E8FFFF0BD8B498D05CEC07F018EC62F0F9
:100D800093D0040EC16390D0B6678ED0C16B8CD067
:100D9000050EC06363D0000EC16307D0C12B0A0EDD
:100DA0005CEC07F0D8EC61F07FD0010EC16309D094
:100DB000B6677AD018EC62F0C12B0A0E5CEC07F033
:100DC00073D0020EC16309D0B6676ED0D8EC61F063
:100DD000C12B0A0E5CEC07F067D0030EC16309D08B
:100DE000B66762D018EC62F0C12B0A0E5CEC07F01B
:100DF0005BD0040EC16309D0B66756D0C12BD8ECC6
:100E000061F00A0E5CEC07F04FD0050EC16309D00B
:100E1000B6674AD018EC62F0C12B0A0E5CEC07F002
:100E200043D0060EC16309D0B6673ED0D8EC61F05E
:100E3000C12BFA0E5CEC07F037D0070EC16307D068
:100E4000B66732D0C12BF00E5CEC07F02DD0080E47
:100E5000C1632AD0B66728D0C16B26D0060EC06306
:100E600023D0000EC16307D004EC62F0C12B0A0E40
:100E70005CEC07F019D0010EC16309D0B66714D03D
:100E800018EC62F0C12B0A0E5CEC07F00DD0020EDC
:100E9000C1630AD0B66708D004EC62F0010EC16FDE
:100EA0000A0E5CEC07F000D00AC0E9FF0BC0EAFFB5
:100EB000005001C0D8FF1000B66F0A0EB76F1200C5
:100EC0000001D42BFA0ED46324D0D46BD32B040EA0
:100ED000D3631FD0D36BD52BBA67BA07010EBB5FA4
:100EE000E86ABC5BBB6707D0BC6705D026C0BBF017
:100EF00027C0BCF06481010EBD5FE86ABE5BBD67C0
:100F000007D0BE6705D065C0BDF066C0BEF0648581
:100F100034801200D880EF50E75ED8A0E76C120052
:100F2000C26A0F0EC16E070EB46E806A816A826A51
:100F3000836A846A856A866A000E926E070E936ED3
:100F4000B80E946EA10E956E090E966E000E976EF9
:100F5000140E986E82928290838684888492848410
:100F6000808A8186D66AD76A530ED56ED58E336A4B
:100F7000326A0001D36BD46BD56BF86BA16B996BA4
:100F8000A66BA76B346A646BBF6B356A366A376AC7
:100F9000386A396A3A6A3B6A576A586A596A5A6AB9
:100FA000676B3D6A3F6AA06B6B6B426A8A6B140E7B
:100FB000976F00EE43F0EE6A972FFDD7400E976FC4
:100FC00004EEC0F0EE6A972FFDD7976B0DEE00F0A0
:100FD0001EEE00F0EE68E668972FFCD7120E976FB2
:100FE00001EE8CF011EE9EF0200EEE6EE66E972F65
:100FF000FBD79EEC64F0B1EC63F08E6FC0EC63F055
:101000008F6FCEEC63F08388690EAF6E260EAC6EE8
:10101000920EAB6E080E6F6E260E6C6E920E6B6E9D
:10102000D08EF28AF194F294F288F292F16AF06A28
:10103000F0889F8A9D8A9F989D98A59AA38AA598D3
:10104000A398F28CF28EF28C57EC66F0B8EC66F056
:10105000A66BA76B76EC63F080868094808280908C
:101060008690E30EF76E940EF66E20EED6F018EC36
:1010700066F0FF0EF76EB20EF66E20EEE6F018EC9C
:1010800066F036EC66F0640EAE6F0A0EAD6FAD67BB
:1010900047EF08F04CEC62F094EC34F030A2A3EC93
:1010A00034F030B213D039AE09D0F90EF76E140E09
:1010B000F66E20EEE6F018EC66F008D0F90EF76E4A
:1010C000240EF66E20EEE6F018EC66F039AC09D08E
:1010D000F80EF76EF40EF66E20EED6F018EC66F011
:1010E00008D0F90EF76E040EF66E20EED6F018EC6E
:1010F00066F036EC66F0640EAE6F140EAD6FAD6741
:10110000FED744EC62F0C8EC62F0A66BA76B76ECFD
:1011100063F0A68776EC63F0A78976EC63F0300E77
:101120002414E86664873994F90EF76E340EF66E6F
:1011300020EED6F018EC66F0E40EF76E040EF66EB4
:1011400020EEE6F018EC66F036EC66F08280576A26
:10115000640EAE6F050EAD6FAD67FED78290640E64
:10116000AE6F140EAD6FAD67FED7050E976F3D9055
:101170003D92DF0EF76EFA0EF66E23EE00F011ECE4
:1011800066F0DE6A02EC66F0640EAE6F140EAD6FB0
:101190003DB0E2EF08F0AD67FBD7972FE8D7E40E3C
:1011A000F76E540EF66E20EED6F018EC66F0E40EF4
:1011B000F76E640EF66E20EEE6F018EC66F036EC94
:1011C00066F0FFD73D903D92E00EF76E580EF66E3A
:1011D00023EE00F011EC66F0DE6A02EC66F0640EBD
:1011E000AE6F320EAD6F3DB0FCEF08F03DB2CFEF09
:1011F00008F0AD67F8D7D3D7640EAE6F0A0EAD6FA7
:10120000AD67FED73D903D92E00EF76E740EF66E20
:1012100023EE00F011EC66F0DE6A02EC66F0640E7C
:10122000AE6F320EAD6F3DB01CEF09F03DB2CFEFA7
:1012300008F0AD67F8D7B3D7640EAE6F140EAD6F7C
:10124000AD67FED73D903D92E00EF76E8C0EF66EC8
:1012500023EE00F011EC66F0DE6A02EC66F0640E3C
:10126000AE6F320EAD6F3DB03CEF09F03DB2CFEF47
:1012700008F0AD67F8D793D73D903D92E10EF76E39
:10128000400EF66E23EE00F011EC66F0DE6A02EC22
:1012900066F0640EAE6F640EAD6F3DB056EF09F0B0
:1012A0003DB2CFEF08F0AD67F8D779D7640EAE6FD7
:1012B0000A0EAD6FAD67FED73D903D92E00EF76E22
:1012C000E00EF66E23EE00F011EC66F0DE6A02EC42
:1012D00066F0640EAE6F640EAD6F57B678EF09F02E
:1012E00057B078EF09F03DB03D90AD67F6D757D7CE
:1012F0005796E50EF76E040EF66E20EEE6F018EC4B
:1013000066F036EC66F03D903D92E10EF76E040E0D
:10131000F66E23EE00F011EC66F0DE6A02EC66F089
:10132000640EAE6F320EAD6F3DB09FEF09F03DB26F
:101330009CEF09F0AD67F8D73D92CFEF08F03D90F4
:101340003D92E00EF76E100EF66E23EE00F011ECFB
:1013500066F0DE6A02EC66F0640EAE6F320EAD6FC0
:101360003DB0BBEF09F03DB2B8EF09F0AD67F8D77B
:101370003D92CFEF08F0388C3D903D92E00EF76E35
:10138000A60EF66E23EE00F011EC66F0DE6A02ECBB
:1013900066F0640EAE6F320EAD6F3DB0D7EF09F060
:1013A0003DB2D5EF09F0AD67F8D73D92F8D63D9044
:1013B000389C100E976F08EE52F018EE22F0EECF28
:1013C000E6FF972FFCD703EE00F0410EEE6E540EB1
:1013D000EE6E2B0EEE6E570EEE6E4D0EEE6E420E54
:1013E000EE6E530EEE6E3D0EEE6E1FC084F07CEC82
:1013F00061F07FC0EEFF80C0EEFF81C0EEFFEE6ABD
:101400003D6A02EC66F0640EAE6F320EAD6F3DB019
:1014100011EF0AF03DB20FEF0AF0AD67F8D73D9239
:10142000BED63D90E60EF76E440EF66E20EED6F078
:1014300018EC66F020C084F07CEC61F0200EE16FC7
:10144000E46F300E806380C0E1F081C0E2F021C023
:1014500084F07CEC61F0300E806380C0E4F081C0E9
:10146000E5F01FC0F4F16AEC5DF036EC66F0640E56
:10147000AE6F320EAD6FAD67FED7E40EF76E240E81
:10148000F66E20EED6F018EC66F0E40EF76E340E31
:10149000F66E20EEE6F018EC66F0310EE96F36ECF1
:1014A00066F0060EC06FC16BBF8F399639823886E1
:1014B0003498ABEC30F0E86640EF0FF038823D9A9C
:1014C0003D903D92E10EF76E6C0EF66E23EE00F04D
:1014D00011EC66F0DE6A02EC66F0640EAE6F320E5E
:1014E000AD6F3DB090EF0AF03DB27BEF0AF0AD6713
:1014F000F8D7CFEF08F03D92E40EF76E740EF66E5B
:1015000020EED6F018EC66F0E40EF76E840EF66E60
:1015100020EEE6F018EC66F036EC66F077EF14F0AB
:101520003D90640EAE6F040EAD6FAD67FED73D907B
:101530003D92E10EF76E7A0EF66E23EE00F011EC9E
:1015400066F0DE6A02EC66F0640EAE6F320EAD6FCE
:101550003DBAB4EF0AF03DB0B8EF0AF03DB2B6EFD5
:101560000AF0AD67F5D71BD63D9AF2D73D9217D654
:101570003D90E50EF76E940EF66E20EED6F018EC68
:1015800066F0E50EF76EA40EF66E20EEE6F018ECAF
:1015900066F001EE7CF010EEDEF0080E976FEECFF5
:1015A000E6FF972FFCD7310E39B4320EE96F36ECD7
:1015B00066F0976B640EAE6F640EAD6F57B0EDEFD3
:1015C0000AF057B810EF0BF034B008EF0BF03DB055
:1015D00006EF0BF0AD67F2D724D05990E40EF76E0A
:1015E000F40EF66E20EED6F018EC66F0E40EF76E10
:1015F000E40EF66E20EEE6F018EC66F0310E39B42B
:10160000320EF06F36EC66F03DEF0AF03D90D6D723
:101610003490070E9715F56F972B36EC66F0CED702
:1016200057983D903D92E00EF76E1C0EF66E23EE3D
:1016300000F011EC66F0DE6A02EC66F0640EAE6F4C
:10164000320EAD6F3DB02DEF0BF03DB22AEF0BF037
:10165000AD67F8D73D92CFEF08F03D9003EE00F074
:10166000410EEE6E540EEE6E2B0EEE6E570EEE6EBB
:10167000560EEE6E520EEE6E3D0EEE6E20C084F0F3
:101680007CEC61F07FC0EEFF80C0EEFF81C0EEFF1A
:101690002C0EEE6E21C084F07CEC61F07FC0EEFF7A
:1016A00080C0EEFF81C0EEFFEE6A3D6A02EC66F09C
:1016B000640EAE6F320EAD6F3DB066EF0BF03DB213
:1016C00064EF0BF0AD67F8D73D92C2D33D903D90EB
:1016D0003D92E00EF76E800EF66E23EE00F011ECF8
:1016E00066F0DE6A02EC66F0640EAE6F320EAD6F2D
:1016F0003DB082EF0BF03DB280EF0BF0AD67F8D755
:101700003D92A6D3F8EC3AF0640EAE6F320EAD6F98
:101710003DB092EF0BF03DB290EF0BF0AD67F8D714
:101720003D9296D3D9EC3AF0640EAE6F320EAD6FA7
:101730003DB0A2EF0BF03DB2A0EF0BF0AD67F8D7D4
:101740003D9286D33D9018EE22F0E6CF7FF0E6CFB3
:1017500080F0E6CF81F0330E7F6307D0340E8063D4
:1017600004D0330E816301D028D0330E7F6307D0BD
:10177000340E806304D0340E816301D01ED0340E49
:101780007F6307D0340E806304D0330E816301D0B1
:1017900014D0360E7F6307D0350E806304D0370E29
:1017A000816301D00AD0350E7F6307D0340E806389
:1017B00004D0310E816301D00BD13D903D92E20EF9
:1017C000F76EB20EF66E23EE00F011EC66F0DE6AF4
:1017D00002EC66F0640EAE6F320EAD6F3DB0F8EF06
:1017E0000BF03DB2F6EF0BF0AD67F8D73D9230D37A
:1017F0003D903D92E20EF76EA40EF66E23EE00F0E1
:1018000011EC66F0DE6A02EC66F0640EAE6F320E2A
:10181000AD6F3DB013EF0CF03DB211EF0CF0AD67C2
:10182000F8D73D9215D33D903D92E20EF76E980E9B
:10183000F66E23EE00F011EC66F0DE6A02EC66F064
:10184000640EAE6F320EAD6F3DB02EEF0CF03DB2B8
:101850002CEF0CF0AD67F8D73D92FAD23D903D9059
:101860003D92E20EF76E580EF66E23EE00F011EC8C
:1018700066F0DE6A02EC66F0640EAE6F320EAD6F9B
:101880003DB06EEF0DF03DB248EF0CF0AD67F8D70C
:101890003D92FF0EF76E020EF66E20EED6F018ECBB
:1018A00066F0FF0EF76E120EF66E20EEE6F018EC04
:1018B00066F036EC66F0640EAE6F280EAD6FAD6765
:1018C000FED731D43D903D92E20EF76E280EF66EB3
:1018D00023EE00F011EC66F0DE6A02EC66F0640EB6
:1018E000AE6F320EAD6F3DB07DEF0CF03DB27BEFD1
:1018F0000CF0AD67F8D73D92ABD23D903D92E20E31
:10190000F76E1A0EF66E23EE00F011EC66F0DE6A4A
:1019100002EC66F0640EAE6F320EAD6F3DB098EF24
:101920000CF03DB296EF0CF0AD67F8D73D9290D237
:101930003D903D92E20EF76E0C0EF66E23EE00F037
:1019400011EC66F0DE6A02EC66F0640EAE6F320EE9
:10195000AD6F3DB0B3EF0CF03DB2B1EF0CF0AD6741
:10196000F8D73D9275D23D903D903D92E10EF76ED5
:10197000F20EF66E23EE00F011EC66F0DE6A02EC79
:1019800066F0640EAE6F320EAD6F3DB06EEF0DF0CF
:101990003DB2CDEF0CF0AD67F8D73D92FF0EF76E7C
:1019A000020EF66E20EED6F018EC66F0FF0EF76E23
:1019B000120EF66E20EEE6F018EC66F036EC66F0ED
:1019C000640EAE6F280EAD6FAD67FED793EF08F0D3
:1019D0003D903D92E20EF76EF60EF66E23EE00F0AD
:1019E00011EC66F0DE6A02EC66F0640EAE6F320E49
:1019F000AD6F3DB003EF0DF03DB201EF0DF0AD67FF
:101A0000F8D73D9225D23D903D92E20EF76EE80E5A
:101A1000F66E23EE00F011EC66F0DE6A02EC66F082
:101A2000640EAE6F320EAD6F3DB01EEF0DF03DB2E5
:101A30001CEF0DF0AD67F8D73D920AD23D903D9274
:101A4000E20EF76EDA0EF66E23EE00F011EC66F0A1
:101A5000DE6A02EC66F0640EAE6F320EAD6F3DB022
:101A600039EF0DF03DB237EF0DF0AD67F8D73D928D
:101A7000EFD13D903D903D92E20EF76EC00EF66EB6
:101A800023EE00F011EC66F0DE6A02EC66F0640E04
:101A9000AE6F320EAD6F3DB06EEF0DF03DB253EF55
:101AA0000DF0AD67F8D73D92FF0EF76E020EF66EA1
:101AB00020EED6F018EC66F0FF0EF76E120EF66E02
:101AC00020EEE6F018EC66F036EC66F0640EAE6FD1
:101AD000280EAD6FAD67FED793EF08F03D903D92B5
:101AE000E10EF76EE60EF66E23EE00F011EC66F0F6
:101AF000DE6A02EC66F0640EAE6F320EAD6F3DB082
:101B000089EF0DF03DB287EF0DF0AD67F8D73D924C
:101B10009FD13D903D92E00EF76EEC0EF66E23EEF7
:101B200000F011EC66F0DE6A02EC66F0640EAE6F57
:101B3000320EAD6F3DB0A4EF0DF03DB2A2EF0DF04F
:101B4000AD67F8D73D9284D13D903D92E10EF76E9E
:101B50002A0EF66E23EE00F011EC66F0DE6A02EC5F
:101B600066F0640EAE6F320EAD6F3DB0BFEF0DF09C
:101B70003DB2BDEF0DF0AD67F8D73D9269D13D9014
:101B80003D92E10EF76E340EF66E23EE00F011EC8E
:101B900066F0DE6A02EC66F0640EAE6F320EAD6F78
:101BA0003DB0DAEF0DF03DB2D8EF0DF0AD67F8D7EC
:101BB0003D924ED13D903D92E10EF76EB80EF66E1D
:101BC00023EE00F011EC66F0DE6A02EC66F0640EC3
:101BD000AE6F320EAD6F3DB00CEF0EF03DB2F3EFD5
:101BE0000DF0AD67F8D73D92FF0EF76E420EF66E20
:101BF00020EED6F018EC66F0FF0EF76E520EF66E81
:101C000020EEE6F018EC66F036EC66F0640EAE6F8F
:101C1000280EAD6FAD67FED73D90FA0EF76E040E3D
:101C2000F66E20EED6F018EC66F0FA0EF76E140E93
:101C3000F66E20EEE6F018EC66F036EC66F03D90BD
:101C40003D92E30EF76E040EF66E23EE00F011ECFB
:101C500066F0DE6A02EC66F0640EAE6F640EAD6F85
:101C60003DB03AEF0EF03DB238EF0EF0AD67F8D769
:101C70003D925FD03D903D92E30EF76E100EF66EF2
:101C800023EE00F011EC66F0DE6A02EC66F0640E02
:101C9000AE6F640EAD6F3DB055EF0EF03DB253EF39
:101CA0000EF0AD67F8D73D9244D03D903D92E30EE3
:101CB000F76E1C0EF66E23EE00F011EC66F0DE6A95
:101CC00002EC66F0640EAE6F640EAD6F3DB070EF67
:101CD0000EF03DB26EEF0EF0AD67F8D73D9229D011
:101CE0003D903D92E30EF76E3A0EF66E23EE00F055
:101CF00011EC66F0DE6A02EC66F0640EAE6FFA0E6E
:101D0000AD6F3DB097EF0EF03DB295EF0EF0AD67C1
:101D1000F8D7640EAE6FFA0EAD6F3DB097EF0EF0D0
:101D20003DB295EF0EF0AD67F8D73D9202D03D90F1
:101D300018D0FF0EF76E620EF66E20EED6F018EC9D
:101D400066F0FF0EF76E720EF66E20EEE6F018ECFF
:101D500066F036EC66F0640EAE6F280EAD6FAD67C0
:101D6000FED761EC5DF03D903D92E00EF76EC60E41
:101D7000F66E23EE00F011EC66F0DE6A02EC66F01F
:101D8000640EAE6F640EAD6F3DB0CEEF0EF03DB29F
:101D9000CCEF0EF0AD67F8D73D925AD009EE00F0C7
:101DA000EECF5BF0EECF5CF0EECF5DF0EECF5EF00D
:101DB000EECF00F0EECF00F0EECF00F0EECF00F06F
:101DC000EECF5FF0EECF60F0EECF61F0EECF62F0DD
:101DD000636B640EAE6F050EAD6FAD67FED73D90C1
:101DE0003D92DF0EF76EFE0EF66E23EE00F011EC64
:101DF00066F0DE6A02EC66F0640EAE6F320EAD6F16
:101E00003DB00BEF0FF03DB208EF0FF0AD67F8D724
:101E10003D92CFEF08F03D903D92E10EF76E400EFF
:101E2000F66E23EE00F011EC66F0DE6A02EC66F06E
:101E3000640EAE6F640EAD6F3DB026EF0FF03DB295
:101E400024EF0FF0AD67F8D73D9202D03D9018D047
:101E5000E60EF76E840EF66E20EED6F018EC66F005
:101E6000E60EF76E940EF66E20EEE6F018EC66F0D5
:101E700036EC66F0640EAE6F320EAD6FAD67FED716
:101E8000040E9A6F9AC0E5F0576A586A596AD2EC04
:101E900061F0809A358C320EAB6FAB67FED782AAA9
:101EA00064EF0FF0F70EF76E240EF66E20EED6F00C
:101EB00018EC66F0F70EF76E340EF66E20EEE6F0D4
:101EC00018EC66F0358E11D0F70EF76E040EF66E34
:101ED00020EED6F018EC66F0F70EF76E140EF66EE4
:101EE00020EEE6F018EC66F0359E808A359C36ECE4
:101EF00066F0640EAE6F140EAD6FAD67FED722ECC8
:101F000066F02CEC66F0808680948082809000D011
:101F100067936795349A30B0348A34B893EF08F0F9
:101F200026C0BBF027C0BCF0A66BA76B76EC63F0B5
:101F3000A68776EC63F0809A358C320EAB6FAB6778
:101F4000FED7359E82BA358E808A359CF8EC3AF001
:101F5000640EAE6F320EAD6F3DB0B5EF0FF03DB217
:101F6000B4EF0FF0AD67F8D73D923D90389E389EA4
:101F7000576A586A3D6A3E6AF66B120E976F01EE19
:101F80008CF011EE9EF0200EEE6EE66E972FFBD7D2
:101F900039A41DD039963982060EC06FC16BBF8F30
:101FA000E70EF76EA40EF66E20EED6F018EC66F093
:101FB000E70EF76EB40EF66E20EEE6F018EC66F063
:101FC00036EC66F03886ABEC30F0E8665BD0A66B9A
:101FD000A76B76EC63F0D2EC61F038B6BBD264A7A5
:101FE00015D0649724C09AF09A3B030E9A17000EFE
:101FF0009A5DD8B4F6D2010E9A5DD8B400D3020E21
:102000009A5DD8B4A5D3CF0E2416EBD2FF0EF76E8F
:10201000A20EF66E20EED6F018EC66F0F60EF76E15
:10202000940EF66E20EEE6F018EC66F035BE13D096
:1020300000EEEEF0200E4E0EEE6E6F0EEE6E200EE7
:10204000EE6E4C0EEE6E690EEE6E6E0EEE6E650E60
:10205000EE6E200EEE6E38B2348238B2388038B26E
:102060000FD0389000EEE6F04E0EEE6E6F0EEE6E74
:10207000200EEE6E470EEE6E530EEE6E4D0EEE6EB1
:1020800036EC66F034BA8FEF10F067B5A8EF12F0B7
:1020900067B3A6EF12F081A284EF14F05AB052EFAA
:1020A00012F05AB255EF12F05AB455EF12F05AB678
:1020B00055EF12F05AB852EF12F05ABA55EF12F02B
:1020C00035B264EF18F038B485EF1EF03BB676EF0A
:1020D00026F038BA45EF29F057B069EF12F057B241
:1020E0007FEF12F059B09EEF12F059B2A3EF12F049
:1020F00034B059EF14F06BA203D06B9800006B88DA
:1021000024C081F0300E8117100E815D54E024C090
:1021100081F0030E8117010E8163B4D7FBD0349A8E
:102120003D903D92E00EF76E660EF66E23EE00F0E7
:1021300011EC66F0DE6A02EC66F0640EAE6F320EF1
:10214000AD6F3DB0C4EF10F03DB2A9EF10F0AD6738
:10215000F8D73D92FE0EF76EC20EF66E20EED6F068
:1021600018EC66F0FE0EF76ED20EF66E20EEE6F07C
:1021700018EC66F036EC66F0640EAE6F280EAD6FAC
:10218000AD67FED73090C4D63D90FE0EF76EE20EDE
:10219000F66E20EED6F018EC66F0FE0EF76EF20E3C
:1021A000F66E20EEE6F018EC66F036EC66F081A2F2
:1021B00084EF14F0FCD764A565D76495040E976F7F
:1021C0008A2B040E8A618A6B19EEA2F0080E8A032C
:1021D000F350E126F450E222E6CF7CF0E6CF7DF02A
:1021E000E6CF7EF0E6CF7FF0E6CF80F0E6CF81F05D
:1021F000E6CF7AF0E6CF7BF0200E7D5D04E07A67D3
:102200001FD07B671DD08A2B972FDED7E60EF76E87
:10221000240EF66E20EED6F018EC66F0E60EF76EA1
:10222000340EF66E20EEE6F018EC66F036EC66F052
:10223000640EAE6F320EAD6FAD67FED73DEF0AF0A4
:1022400003EE00F0410EEE6E540EEE6E2B0EEE6EAF
:10225000430EEE6E4F0EEE6E500EEE6E530EEE6EA1
:102260003D0EEE6E310EEE6E2C0EEE6E320EEE6EFA
:102270002C0EEE6E7CC0EEFF7DC0EEFF7EC0EEFF4A
:102280007FC0EEFF80C0EEFF81C0EEFF000EEE6E5D
:102290003D6A576A586A02EC66F0640EAE6FC80E6B
:1022A000AD6F3DB080EF11F03DB259EF11F0AD6769
:1022B000F8D73D92E50EF76ED40EF66E20EED6F00E
:1022C00018EC66F0E50EF76EF40EF66E20EEE6F012
:1022D00018EC66F07CC0E0F07DC0E1F07EC0E2F07A
:1022E0007FC0E3F080C0E4F081C0E5F036EC66F03A
:1022F000640EAE6F320EAD6FAD67FED73DEF0AF0E4
:1023000064957AC065F07BC066F065C0BDF066C0BC
:10231000BEF07CD664A1B6D6649161EC5DF03D90D0
:102320003D92E00EF76EC60EF66E23EE00F011EC55
:1023300066F0DE6A02EC66F0640EAE6F640EAD6F9E
:102340003DB0AAEF11F03DB2A8EF11F0AD67F8D79C
:102350003D9298D6060E976F632B060E6361636BF2
:1023600009EE16F0160E6303F350E926F450EA2640
:10237000EECF7AF0EECF7BF0EECF7CF0EECF7DF0BB
:10238000EECF7EF0EECF7FF0300E286412D07A517F
:10239000286285D07B51296282D07C512A627FD00D
:1023A0007D512B627CD07E512C6279D07F512D6281
:1023B00076D0EECF7AF0EECF7BF0EECF7CF0EECFA2
:1023C0007DF0200E7A5D6BE07A515B620AD07B5122
:1023D0005C6207D07C515D6204D07D515E6201D0A9
:1023E0005ED07AC0C2F97BC0C3F97CC0C4F97DC09D
:1023F000C5F909EE24F0160E6303F350E926F450F4
:10240000EA26EECFC6F9EECFC7F9EECFC8F9EECF88
:10241000C9F9EECF7EF0EECF7FF0EECF80F0EECFB9
:1024200081F0200E7F5D300ED8B47F6F200E805D6E
:10243000300ED8B4806F32EC61F0845125602FD01B
:10244000C2C95BF0C3C95CF0C4C95DF0C5C95EF028
:1024500003EE00F0410EEE6E540EEE6E2B0EEE6E9D
:10246000430EEE6EEE6E450EEE6E4C0EEE6EEE6EA2
:102470003D0EEE6EC6C9EEFFC7C9EEFFC8C9EEFF3E
:10248000C9C9EEFFEE6A5A6A02EC66F0C6C95FF08F
:10249000C7C960F0C8C961F0C9C962F0F3D5972F08
:1024A0005BD7F0D55A905A98EDD55A6AEE0EF76E72
:1024B000F40EF66E20EED6F018EC66F0EF0EF76E26
:1024C000040EF66E20EEE6F018EC66F036EC66F0E0
:1024D000D9D5579038903492E40EF76E940EF66E7C
:1024E00020EED6F018EC66F0E40EF76EB40EF66E41
:1024F00020EEE6F018EC66F036EC66F0C3D55792A5
:1025000038903492E40EF76E940EF66E20EED6F00C
:1025100018EC66F0E40EF76EC40EF66E20EEE6F0F0
:1025200018EC66F036EC66F039963982640EAE6FC0
:10253000140EAD6FAD67FED73DEF0AF0599038909D
:1025400034923DEF0AF059923DEF0AF06793C2D7FB
:102550006795D6D738961EC09AF09A3B030E9A1705
:10256000000E9A630ED03D903D92E00EF76E340E51
:10257000F66E23EE00F011EC66F0DE6A02EC66F017
:102580001ED0010E9A630ED03D903D92E00EF76E84
:10259000400EF66E23EE00F011EC66F0DE6A02ECFF
:1025A00066F00DD03D903D92E00EF76E4C0EF66E4B
:1025B00023EE00F011EC66F0DE6A02EC66F0640EC9
:1025C000AE6F320EAD6F3DB0EFEF12F03DB2ECEFFB
:1025D00012F0AD67F8D703D53D92EFEF0FF03D90C5
:1025E000FED43D903D92E10EF76E460EF66E23EE60
:1025F00000F011EC66F0DE6A02EC66F007D5040E1E
:10260000976F8A6B19EEA2F0080E8A03F350E12649
:10261000F450E222E6CF7CF0E6CF7DF0E6CF7EF00C
:10262000E6CF7FF0E6CF80F0E6CF81F0E6CF7AF01C
:10263000E6CF7BF0200E7D5D04E07A671FD07B67DC
:102640001DD08A2B972FDED7E60EF76E240EF66E7E
:1026500020EED6F018EC66F0E60EF76E340EF66E4D
:1026600020EEE6F018EC66F036EC66F0640EAE6F25
:10267000280EAD6FAD67FED73DEF0AF003EE00F018
:10268000410EEE6E540EEE6E2B0EEE6E430EEE6E9F
:102690004F0EEE6E500EEE6E530EEE6E3D0EEE6E63
:1026A000310EEE6E2C0EEE6E320EEE6E2C0EEE6EC7
:1026B0007CC0EEFF7DC0EEFF7EC0EEFF7FC0EEFF70
:1026C00080C0EEFF81C0EEFF000EEE6E3D6A576ADD
:1026D000586A02EC66F0640EAE6FC80EAD6F3DB086
:1026E0009EEF13F03DB277EF13F0AD67F8D73D9250
:1026F000E50EF76ED40EF66E20EED6F018EC66F00E
:10270000E50EF76EF40EF66E20EEE6F018EC66F0CD
:102710007CC0E0F07DC0E1F07EC0E2F07FC0E3F07D
:1027200080C0E4F081C0E5F036EC66F0640EAE6F78
:10273000320EAD6FAD67FED73DEF0AF064957AC0FB
:1027400065F07BC066F065C0BDF066C0BEF05ED4CB
:10275000E50EF76EB40EF66E20EED6F018EC66F0CD
:10276000E50EF76EC40EF66E20EEE6F018EC66F09D
:10277000200E9BC99AF09A631AD0E60EF76E040EEB
:10278000F66E20EED6F018EC66F0E60EF76E140E3C
:10279000F66E20EEE6F018EC66F036EC66F0640EAD
:1027A000AE6F280EAD6FAD67FED73DEF0AF003EEBA
:1027B00000F0410EEE6E540EEE6E2B0EEE6E430EDA
:1027C000EE6E4F0EEE6E500EEE6E530EEE6E3D0E32
:1027D000EE6E310EEE6E2C0EEE6E320EEE6E2C0E96
:1027E000EE6E19EE9AF0060E976F200EE75C05E08C
:1027F000E6CFEEFF972FF5EF13F0000EEE6E3D6A79
:10280000576A586A02EC66F0640EAE6FC80EAD6F80
:102810003DB035EF14F03DB210EF14F0AD67F8D7CE
:102820003D92E50EF76ED40EF66E20EED6F018EC63
:1028300066F0E50EF76EF40EF66E20EEE6F018EC9C
:1028400066F0060E976F19EE9AF000EEE0F0E6CF14
:10285000EEFF972FFCD736EC66F0640EAE6F320EAB
:10286000AD6FAD67FED73DEF0AF0E50EF76ED40E03
:10287000F66E20EED6F018EC66F0E50EF76EE40E7C
:10288000F66E20EEE6F018EC66F0060E976F19EE85
:102890009AF000EEE0F0E6CFEEFF972FFCD736EC93
:1028A00066F0640EAE6F320EAD6FAD67FED706EF09
:1028B00010F0EDEC5CF042EF10F0A66BA76B76EC3D
:1028C00063F0A68776EC63F0BFC081F0030E81173A
:1028D000816705D0020EC06FC16BBF8F0CD0010E97
:1028E000816305D0030EC06FC16BBF8F04D0060E8D
:1028F000C06FC16BBF8F81A27BEF14F0FC0EBF0BCA
:10290000D2EC61F088EF0FF044EC62F0C8EC62F0BA
:10291000A66BA76B76EC63F0A68776EC63F0A789CD
:1029200076EC63F0320EAB6FAB67FED722EC66F04D
:102930002CEC66F0E60EF76EA40EF66E20EED6F0E6
:1029400018EC66F02CEC66F036EC66F0010EC06F09
:10295000C16BBF8F51EC5DF03494640EAB6FAB670D
:10296000FED7640EAE6FFA0EAD6F81B2BFEF14F0FA
:10297000A0B10AD0AD67F9D7010EBF139ED7D2EC34
:1029800061F0348288EF0FF0D2EC61F001EED2F00A
:1029900010EEE6F09E6B349434961FEC62F09DC00E
:1029A000EEFF9DC0E6FF36EC66F09E2B230E9D5D8C
:1029B000D8B434842A0E9D5DD8B43486640EAE6FCC
:1029C00017C0ADF081B23DEF15F0A0B104D0AD67F6
:1029D000F9D789EF15F01FEC62F09E2B230E9D6353
:1029E00006D034B4E8EF34F034B649D008D02A0E1B
:1029F0009D63FFEF14F034B67DD034B4B4D0020E32
:102A00009E6307D034A405D02B0EE8CFD2F1E8CFD7
:102A1000E6F034943496110E9E6117EF15F09DC0C8
:102A2000EEFF9DC0E6FF36EC66F0DEEF14F0E7C087
:102A3000E6F0E8C0E7F0E9C0E8F0EAC0E9F0EBC092
:102A4000EAF0ECC0EBF0EDC0ECF0EEC0EDF0EFC062
:102A5000EEF0F0C0EFF0F1C0F0F0F2C0F1F0F3C032
:102A6000F2F0F4C0F3F0F5C0F4F09DC0EEFF9DC0AD
:102A7000F5F036EC66F0DEEF14F088EF0FF0FF0EA5
:102A8000F76E820EF66E20EED6F018EC66F02CECA7
:102A900066F0100E976F08EE22F010EEE6F0EECF23
:102AA000E6FF972FFCD736EC66F081B288EF0FF087
:102AB000A0B15CEF15F0F9D71FEC62F0FF0EF76ED6
:102AC000920EF66E20EED6F018EC66F0FF0EF76E62
:102AD000B20EF66E20EEE6F018EC66F036EC66F01C
:102AE00081B288EF0FF0A0B177EF15F0F9D71FECA6
:102AF00062F0C5D7E70EF76E940EF66E20EEE6F0A4
:102B000018EC66F036EC66F081A284EF15F088EFE1
:102B10000FF038EC30F0E866DDEF15F0040EC06F12
:102B2000C16BBF8F39B60AD0E70EF76EB40EF66EE2
:102B300020EED6F018EC66F039940AD0E70EF76E66
:102B4000C40EF66E20EED6F018EC66F039843982A9
:102B500036EC66F03886ABEC30F0E86602D0DBEF9E
:102B60001CF088EF0FF0E70EF76E140EF66E20EEF5
:102B7000D6F018EC66F0E70EF76E240EF66E20EE37
:102B8000E6F018EC66F036EC66F0809A358CA66BB1
:102B9000A76B76EC63F0A68976EC63F0A68376ECFF
:102BA00063F081B2D5EF15F0FCD7A66BA76B76EC7E
:102BB00063F0808A359C88EF0FF0E70EF76E540EB5
:102BC000F66E20EED6F018EC66F02CEC66F036ECE3
:102BD00066F0809A358CA66BA76B76EC63F0A68FB7
:102BE00076EC63F0A68976EC63F0A68376EC63F06E
:102BF000320EAB6FAB67FED782AA4DEF16F0358E63
:102C0000640EAE6F080EAD6FAD67FED79E6B01EE22
:102C1000D2F011EE78F0200EE76430D0040E976FFA
:102C2000EF50E7622BD0EE50E650200EE76201D065
:102C300002D0972FF5D797C09AF010EEE6F0040E69
:102C4000976F01EE78F00CAECDEC2DF00CBE0EECD3
:102C50002EF0E86639D00F5009E0976F640EAE6F22
:102C60000A0EAD6FAD67FED7972FF8D701EED2F001
:102C70009A510508E926E86AEA2204D001EED2F06A
:102C800010EEE6F0200E976F0CAECDEC2DF00CBEE2
:102C90000EEC2EF0E86618D02DD0808A359C359E3B
:102CA000F90EF76E540EF66E20EED6F018EC66F0C4
:102CB000F90EF76E640EF66E20EEE6F018EC66F094
:102CC00036EC66F077EF14F0808A359CF90EF76EDB
:102CD000E40EF66E20EED6F018EC66F0F90EF76E04
:102CE000F40EF66E20EEE6F018EC66F036EC66F0C8
:102CF0006FEF14F0A66BA76B76EC63F0A68976EC09
:102D000063F0A68376EC63F0A78976EC63F0A68780
:102D100076EC63F0E70EF76E640EF66E20EED6F0FA
:102D200018EC66F036EC66F0C8EC62F01FEC62F06E
:102D3000A06B579C349481B2AFEF16F038B4C8EF53
:102D400016F03DB6D4EF16F057BCB7EF16F0A0A1C1
:102D5000F2D71FEC62F0230E9D63EDD74FD0FA0E31
:102D6000AB6FAB67FED781B22CEF18F0E4D7579C5E
:102D7000010E7063E0D738943D96E70EF76E640E4F
:102D8000F66E20EED6F018EC66F036EC66F0D3D78F
:102D90003894F60EF76EF40EF66E20EED6F018ECC0
:102DA00066F036EC66F0C7D73D960BEC18F0030ED4
:102DB0001E140208D8A4BFD7F8EC33F03BA0BBD751
:102DC0003D903D92640EAE6F140EAD6F3D903D92FE
:102DD000E00EF76E040EF66E23EE00F011EC66F0D6
:102DE000DE6A02EC66F03DB0FAEF16F03DB2FCEFA1
:102DF00016F0F9D73D909FD73D929DD73484E70ECA
:102E0000F76E740EF66E20EED6F018EC66F02CEC31
:102E100066F036EC66F051EC5DF001EED2F010EEAB
:102E2000E6F09E6B640EAE6F17C0ADF081B22CEF72
:102E300018F038B4D5EF17F03DB6E1EF17F057BCF6
:102E4000C4EF17F0A0B128EF17F0AD67EFD742D06D
:102E50001FEC62F0230E9D6309D034A43BD001EE39
:102E600050F0200EEF6253D0349442D034942A0EA6
:102E70009D5D35E09E2B110E9E6107D09DC0EEFF3B
:102E80009DC0E6FF36EC66F0CDD7E7C0E6F0E8C0BF
:102E9000E7F0E9C0E8F0EAC0E9F0EBC0EAF0ECC026
:102EA000EBF0EDC0ECF0EEC0EDF0EFC0EEF0F0C0F6
:102EB000EFF0F1C0F0F0F2C0F1F0F3C0F2F0F4C0C6
:102EC000F3F0F5C0F4F09DC0EEFF9DC0F5F036ECD8
:102ED00066F0A8D701EED2F0200EEF6233D051ECAD
:102EE0005DF02CEC66F0B2EC34F01FEC62F012D71F
:102EF000E70EF76ED40EF66E20EED6F018EC66F004
:102F000036EC66F0CDEC34F01FEC62F003D751ECF8
:102F10005DF0100E8B6F9E6B11EED2F001EE50F053
:102F2000200EEF5C05E0EECFE6FF9E2B8B2FF8D74F
:102F3000100E8B6F01EED2F010EEE6F0EECFE6FF52
:102F40008B2FFCD7A66BA76B76EC63F0A68F76EC85
:102F500063F0A78B76EC63F0040EC06FC16BBF8F7C
:102F600024AC06D0A68D76EC63F0A78376EC63F0F4
:102F7000E70EF76E840EF66E20EED6F018EC66F0D3
:102F800036EC66F04CEF1BF0579C010E70634AD78D
:102F900038943D96E70EF76E640EF66E20EED6F08E
:102FA00018EC66F036EC66F03DD73894F60EF76E06
:102FB000F40EF66E20EED6F018EC66F036EC66F005
:102FC00031D73D960BEC18F0030E1E140208D8A45E
:102FD00029D7F8EC33F03BA025D73D903D92640E05
:102FE000AE6F140EAD6F3D903D92E00EF76E040E85
:102FF000F66E23EE00F011EC66F0DE6A02EC66F08D
:103000003DB007EF18F03DB209EF18F0ECD63D9057
:1030100009D73D9207D700EEDBF00B0E976F200E1D
:10302000EE6E972F0FEF18F001EE8CF010EEDBF044
:103030000A0E976FEECFE6FF972F1AEF18F036ECD7
:1030400066F0100E976F01EE8CF011EE9EF0EECF51
:10305000E6FF972FFCD7120044EC62F0A06BC8EC9F
:1030600062F0808A359CA66BA76B76EC63F0F70E56
:10307000F76E640EF66E20EED6F018EC66F0F70EE2
:10308000F76E740EF66E20EEE6F018EC66F07DEC4E
:1030900033F036EC66F0640EAE6F140EAD6FAD67B4
:1030A000FED7C00E351688EF0FF0808A359C3C0E97
:1030B000AB6FAB67FED7809A358C280EAB6FAB67D2
:1030C000FED79F2FF2D71200640EAE6F140EAD6FB5
:1030D00035B403D0AD67FCD70FD0A66BA76B76ECE9
:1030E00063F0A78B76EC63F0819651EC2FF081862C
:1030F000A66BA76B76EC63F0F60EF76ED40EF66E49
:1031000020EED6F018EC66F0F60EF76ED40EF66EE2
:1031100020EEE6F018EC66F036EC66F015EC30F0D8
:10312000640EAE6F1E0EAD6F36B202D0AD67FCD727
:103130000CC081F0030E81178167A3D037B006D091
:1031400001EE8CF0200EEE6EEE6E0AD010EEE6F080
:1031500001EE8CF0100E976FE6CFEEFF972FFCD7A5
:1031600019EC2FF0A66BA76B76EC63F0A78976ECD1
:1031700063F0A68776EC63F0140E6C6F1AC06DF0E6
:103180003A903A923A863A94C56B808680948092BF
:10319000808016A44ED016C081F0030E811781677F
:1031A00018D0140E6C6F1AC06DF03A903A923A86AD
:1031B0003A94C56B80868094809280803AA4FED732
:1031C000640EAE6F060EAD6FAD67FED79FEC2EF0AE
:1031D00030D0010E816312D078EC33F04EEC2EF03B
:1031E000140E6C6F1AC06DF03A903A923A863A9487
:1031F000C56B80868094809280801BD0020E816394
:10320000D0D7140E6C6F1AC06DF03A903A923A868D
:103210003A94C56B80868094809280803AA4FED7D1
:10322000640EAE6F060EAD6FAD67FED79FEC2EF04D
:1032300000D081A22BEF19F035A620EF19F0F9D7B5
:103240003A6A8086809480828090FA0EAB6FAB677A
:10325000FED788EF0FF0D2EC61F03A6A8086809456
:103260008082809071EC33F0809A358C3596FA0E1E
:10327000AB6FAB67FED72CEC66F036EC66F07AEFFE
:1032800016F0010E8163E8D0A66BA76B76EC63F0B5
:10329000A68F76EC63F0A78B76EC63F0A68D76ECC8
:1032A00063F0A78376EC63F044EC62F0C8EC62F064
:1032B000809A358C3596E70EF76E540EF66E20EE3A
:1032C000D6F018EC66F051EC5DF02CEC66F036ECC4
:1032D00066F0640EAE6F050EAD6FAD67FED7050EDE
:1032E000C06FC16BBF8F01EED2F010EEE6F09E6BA7
:1032F000640EAE6F640EAD6FA0B103D0AD67FCD7A6
:10330000A3D0D2EC61F01FEC62F0230E9D6301D0DC
:10331000DAD79DC0EEFF9DC0E6FF36EC66F09E2B2F
:1033200011509E6149D0640EAE6F12C0ADF0640EB4
:10333000B06F1350AF6FA0B109D010509E6103D091
:10334000AF67F9D781D0AD67F6D736D01FEC62F002
:10335000230E9D6301D0B7D79E2B110E9E6107D01F
:103360009DC0EEFF9DC0E6FF36EC66F0D9D7E7C002
:10337000E6F0E8C0E7F0E9C0E8F0EAC0E9F0EBC049
:10338000EAF0ECC0EBF0EDC0ECF0EEC0EDF0EFC019
:10339000EEF0F0C0EFF0F1C0F0F0F2C0F1F0F3C0E9
:1033A000F2F0F4C0F3F0F5C0F4F09DC0EEFF9DC064
:1033B000F5F036EC66F0B4D7A66BA76B76EC63F04D
:1033C000A68F76EC63F0A78B76EC63F0040EC06FEB
:1033D000C16BBF8F24ACF3EF19F0A68D76EC63F0D0
:1033E000A78376EC63F00CA657D110509E6554D19C
:1033F000100E976F01EED2F011EE8CF0EECFE6FFDB
:10340000972FFCD7ACEC33F03CB846D1808A359C82
:10341000FE0EF76E820EF66E20EED6F018EC66F019
:10342000FE0EF76E920EF66E20EEE6F018EC66F0E9
:1034300036EC66F0640EAE6F140EAD6FAD67FED75E
:10344000C00E351688EF0FF0A66BA76B76EC63F015
:10345000808A359C88EF0FF0020E81636FD601EEF3
:1034600050F0200EEF6213D0F70EF76E440EF66E9A
:1034700020EED6F018EC66F0F70EF76E540EF66EEE
:1034800020EEE6F018EC66F036EC66F057D60E50FB
:103490003BE1A66BA76B76EC63F0A68F76EC63F04E
:1034A000A78B76EC63F024AC0CD0809A358CA68D7B
:1034B00076EC63F0A78376EC63F0040EC06FC16B0B
:1034C000BF8FE70EF76E840EF66E20EED6F018EC86
:1034D00066F02CEC66F051EC5DF0100E8B6F11EE87
:1034E000D2F001EE50F0EECFE6FF8B2FFCD7100E9E
:1034F0008B6F01EED2F010EEE6F0EECFE6FF8B2FF1
:10350000FCD736EC66F0C8D001EE50F037B006D0EC
:1035100001EE8CF0200EEE6EEE6E0AD010EEE6F0AC
:1035200001EE8CF0100E976FE6CFEEFF972FFCD7D1
:1035300019EC2FF0A66BA76B76EC63F0A78976ECFD
:1035400063F0A68776EC63F0140E6C6F1AC06DF012
:103550003A903A923A863A94C56B808680948092EB
:10356000808016A44DD016C081F0030E81178167AC
:1035700018D0140E6C6F1AC06DF03A903A923A86D9
:103580003A94C56B80868094809280803AA4FED75E
:10359000640EAE6F060EAD6FAD67FED79FEC2EF0DA
:1035A0002FD0010E816312D078EC33F04EEC2EF068
:1035B000140E6C6F1AC06DF03A903A923A863A94B3
:1035C000C56B80868094809280801AD0020E8163C1
:1035D000E8D5140E6C6F1AC06DF03A903A923A86A4
:1035E0003A94C56B80868094809280803AA4FED7FE
:1035F000640EAE6F060EAD6FAD67FED7DCEC2EF03D
:10360000A66BA76B76EC63F0A68F76EC63F0A78BC6
:1036100076EC63F024AC0CD0809A358CA68D76ECD9
:1036200063F0A78376EC63F0040EC06FC16BBF8FAD
:1036300081A22BEF19F024BC03D035A641EF1BF07B
:103640000E50C563F5D73A6A808680948082809058
:1036500051EC5DF0100E8B6F11EED2F001EE50F0D8
:10366000EECFE6FF8B2FFCD7100E8B6F01EED2F062
:1036700010EEE6F0EECFE6FF8B2FFCD736EC66F0CF
:103680000BD03A6A8086809480828090FA0EAB6F6D
:10369000AB67FED788EF0FF00CA406D038EC30F003
:1036A000E8661FD039B60BD0E70EF76EB40EF66E93
:1036B00020EED6F018EC66F0399639940AD0E70E71
:1036C000F76EC40EF66E20EED6F018EC66F0398474
:1036D000398236EC66F03886ABEC30F0E86601D023
:1036E0002AD0FE0EF76EA20EF66E20EED6F018EC83
:1036F00066F0FE0EF76EB20EF66E20EEE6F018ECF7
:1037000066F036EC66F0809A358CA68F76EC63F026
:10371000A78B76EC63F0030EC06FC16BBF8F640E96
:10372000AE6F140EAD6FAD67FED7808A359CC00EAC
:10373000351688EF0FF011EC29F0E60EF76EE40E67
:10374000F66E20EED6F018EC66F0310E39B4320E7B
:10375000E56F36EC66F0D5EC62F044EC62F02FECED
:103760005CF01E0EBA6FA0B13BEC5CF0A0B5E5D0EA
:10377000A0AB03D0AF51D8B4E0D057B0E3EF1BF00B
:1037800057B4E5EF1BF057BAE7EF1BF057BCE9EF72
:103790001BF058B0EEEF1BF058B2F0EF1BF03DB24B
:1037A000F5EF1BF03DB013EF1CF03EB0F7EF1BF050
:1037B0003EB205EF1CF035BC03D035A69DEF1CF0E2
:1037C000BA67D1D7A7D05790A5D05794CCD7579ADE
:1037D000CAD7579C010E7063C6D79CD058909AD018
:1037E000589224BCD2EC61F0BED73D9293D03E906B
:1037F000FD0EF76E340EF66E20EED6F018EC66F085
:10380000CEEC1CF036EC66F0AAD03E92FD0EF76EC0
:10381000540EF66E20EED6F018EC66F0CEEC1CF0EE
:1038200036EC66F09CD03D90D2EC61F0809A358CFD
:10383000A66BA76B76EC63F0A78B76EC63F0A68D96
:1038400076EC63F0A78376EC63F0E60EF76EF40E89
:10385000F66E20EED6F018EC66F0310E39B4320E6A
:10386000E56F36EC66F044EC62F0A0B13BEC5CF046
:10387000A0B563D0A0AB03D0AF51D8B45ED057B0E1
:1038800058EF1CF057BC5AEF1CF058B05FEF1CF01B
:103890003DB061EF1CF03DB263EF1CF03EB065EF50
:1038A0001CF03EB273EF1CF03DB481EF1CF0DDD78D
:1038B000579030D0579C010E7063D7D72BD05890BB
:1038C00029D03D90D2D73D9225D03E90FD0EF76E87
:1038D000340EF66E20EED6F018EC66F0CEEC1CF04E
:1038E00036EC66F03CD03E92FD0EF76E540EF66E4E
:1038F00020EED6F018EC66F0CEEC1CF036EC66F05C
:103900002ED03D94030E1E140208D8A4AED7F8ECB6
:1039100033F0ABD7F70EF76EA40EF66E20EED6F0AE
:1039200018EC66F0F70EF76EB40EF66E20EEE6F0C9
:1039300018EC66F036EC66F012D0F70EF76E840ED7
:10394000F66E20EED6F018EC66F0F70EF76E940ED9
:10395000F66E20EEE6F018EC66F036EC66F0D2EC8F
:1039600061F0A66BA76B76EC63F0808A359C3D9086
:103970003D92E00EF76E040EF66E23EE00F011ECB1
:1039800066F0DE6A02EC66F0640EAE6F140EAD6F88
:10399000AD67FED7C00E351688EF0FF02CEC66F041
:1039A000100E976F11EED2F000EEE6F0E6CFEEFFCC
:1039B000972FFCD71200A66BA76B76EC63F0A7815C
:1039C00076EC63F0A68776EC63F024AC03D0A68592
:1039D00076EC63F003EE00F0410EEE6E540EEE6EE8
:1039E000440EEE6E9EC097F011EED2F0E6CFEEFFE1
:1039F000972FF6EF1CF03B0EEE6E000EEE6E3D6A5A
:103A00003E6A576A586A02EC66F0E60EF76EE40EFC
:103A1000F66E20EED6F018EC66F0310E39B4320EA8
:103A2000E8CFE5F036EC66F03C0EBA6F57B036EFF3
:103A30001DF057BC3CEF1DF058B045EF1DF058B2DB
:103A400055EF1DF03DB25AEF1DF03DB080EF1DF077
:103A50003EB060EF1DF03EB270EF1DF081B256EF48
:103A60001EF0BA67E3D7D2EC61F00DD15790D2ECDB
:103A700061F0020EBF1307D1579C010E7063D6D7B9
:103A8000D2EC61F0010EBF13FED05890D2EC61F081
:103A9000020EBF13E40EF76EF40EF66E20EEE6F0A3
:103AA00018EC66F036EC66F013D1589224BCD2ECD8
:103AB00061F0BCD73D92D2EC61F0020EBF13E3D0AF
:103AC0003E90D2EC61F0FD0EF76E740EF66E20EEB5
:103AD000D6F018EC66F036EC66F0000EBF13D3D0CB
:103AE0003E92D2EC61F0FD0EF76E940EF66E20EE73
:103AF000D6F018EC66F036EC66F0000EBF13C3D0BB
:103B00003D90D2EC61F0A66BA76B76EC63F0A781D9
:103B100076EC63F0A68576EC63F0A68F76EC63F026
:103B200071EC33F0640EAB6FAB67FED7E60EF76E49
:103B3000F40EF66E20EED6F018EC66F0310E39B4C5
:103B4000320EE8CFE5F036EC66F081B256EF1EF0AB
:103B500035B658D057B0C0EF1DF057BCC4EF1DF0BC
:103B600058B0CBEF1DF03DB2D9EF1DF03EB0DDEF08
:103B70001DF03EB2EBEF1DF03DB4F9EF1DF0E5D7BF
:103B80005790020EBF137FD0579C010E7063DDD794
:103B9000010EBF1378D05890020EBF13E40EF76EDB
:103BA000F40EF66E20EEE6F018EC66F036EC66F0F9
:103BB0008FD03D92020EBF1366D03E90FD0EF76E81
:103BC000740EF66E20EED6F018EC66F036EC66F069
:103BD000000EBF1358D03E92FD0EF76E940EF66E97
:103BE00020EED6F018EC66F036EC66F0000EBF134F
:103BF0004AD03D94030E1E140208D8A4A6D7F8ECB0
:103C000033F0A3D7809A358CF60EF76EB40EF66EAD
:103C100020EED6F018EC66F0F60EF76EC40EF66ED7
:103C200020EEE6F018EC66F036EC66F0640EAE6F4F
:103C3000280EAD6F020EC06FC16BBF8FAD67FED790
:103C4000D2EC61F0808A359CC00E3516E60EF76E18
:103C5000F40EF66E20EED6F018EC66F0310E39B4A4
:103C6000320EE8CFE5F09EC097F02CEC66F011EE36
:103C7000D2F000EEE6F0E6CFEEFF972F3BEF1EF01E
:103C800036EC66F062D7F70EF76EA40EF66E20EEF5
:103C9000D6F018EC66F0F70EF76EB40EF66E20EE66
:103CA000E6F018EC66F036EC66F012D0F70EF76E20
:103CB000640EF66E20EED6F018EC66F0F70EF76E96
:103CC000740EF66E20EEE6F018EC66F036EC66F058
:103CD0007DEC33F03D903D92E00EF76E040EF66EF3
:103CE00023EE00F011EC66F0DE6A02EC66F0640E82
:103CF000AE6F140EAD6FAD67FED73D903D923E6A3C
:103D0000579A579C8B6B5DEF14F0E60EF76EB40E6E
:103D1000F66E20EED6F018EC66F0E70EF76E340E75
:103D2000F66E20EEE6F018EC66F036EC66F0C56B49
:103D30003B923D963E6A5790579C5890640EAE6FEA
:103D4000FA0EAD6F57B0BAEF1EF057BCBCEF1EF0C5
:103D500058B0C1EF1EF03EB0C3EF1EF03EB2C3EF4D
:103D60001EF03DB6E2EF1EF038B4F9EF1EF0AD677D
:103D7000E9D70AD0579008D0579C010E7063E2D75C
:103D800003D0589001D03E6A3D903D923D903D92C7
:103D9000E00EF76E040EF66E23EE00F011EC66F006
:103DA000DE6A02EC66F0640EAE6F140EAD6F3DB0CD
:103DB000DFEF1EF03DB2DFEF1EF0AD67F8D73894AD
:103DC00088EF0FF03D963BB2BDD73B822CEC66F0FE
:103DD00001EE8CF0200EEF5CB5E010EEE6F0100E78
:103DE000976FEECFE6FF972FF1EF1EF036EC66F0FF
:103DF000A9D73894C52B010EC565A4D71EC081F084
:103E0000030E81178167AAEF20F034D0F80EF76E09
:103E1000240EF66E20EED6F018EC66F0F80EF76E73
:103E2000340EF66E20EEE6F018EC66F036EC66F036
:103E30003B903B923D903D92E00EF76E040EF66E85
:103E400023EE00F011EC66F0DE6A02EC66F0640E20
:103E5000AE6F140EAD6F3DB033EF1FF03DB233EFD8
:103E60001FF0AD67F8D7AD67FED73D903D923D9608
:103E7000E7EF0FF01EA40CD0ACEC33F03CB208D04E
:103E8000500EEA6303D01EBE03D0C0D716A6BED71D
:103E90003D903D923E6A5790579C589019EC2FF0F8
:103EA000A66BA76B76EC63F0A78976EC63F0A68728
:103EB00076EC63F016B40ED0140E6C6F1AC06DF071
:103EC0003A903A923A863A94C56B80868094809272
:103ED000808034D016C081F0030E8117816718D01E
:103EE000140E6C6F1AC06DF03A903A923A863A947A
:103EF000C56B80868094809280803AA4FED7640E41
:103F0000AE6F060EAD6FAD67FED79FEC2EF016D0EC
:103F1000010E816312D078EC33F04EEC2EF0140ECB
:103F20006C6F1AC06DF03A903A923A863A94C56B2B
:103F3000808680948092808001D0D2D781B2A8EF11
:103F40001FF0640EAB6FAB67FED781A2C2EF1FF00C
:103F500057B0B2EF1FF057BCB6EF1FF058B0B4EF38
:103F60001FF0ECD7579006D0589004D0579C010E04
:103F70007063E4D738943A6A808680948082809017
:103F800088EF0FF03A6A808680948082809071EC8E
:103F900033F0FA0EAB6FAB67FED7E60EF76EF40E9A
:103FA000F66E20EED6F018EC66F036EC66F0A66BF6
:103FB000A76B76EC63F0A78176EC63F0A68576ECD0
:103FC00063F0A68F76EC63F038BE0DD03D903D9245
:103FD000E00EF76E0A0EF66E23EE00F011EC66F0BE
:103FE000DE6A02EC66F081B20BEF20F03DB03D904E
:103FF00057BC54EF20F035B613EF20F03DB402EF7C
:1040000020F0F1D73D94030E1E140208D8A4EBD77C
:10401000F8EC33F0E8D7FA0EAB6FAB67FED781B29E
:104020006EEF20F0E0D7809A358CF60EF76EB40E66
:10403000F66E20EED6F018EC66F0F60EF76EC40EB3
:10404000F66E20EEE6F018EC66F036EC66F0640EE4
:10405000AE6F280EAD6F020EC06FC16BBF8FAD6724
:10406000FED7D2EC61F0808A359CC00E3516E60E84
:10407000F76EF40EF66E20EED6F018EC66F0310E08
:1040800039B4320EE8CFE5F02CEC66F001EE8CF09E
:1040900010EEE6F0100E976FEECFE6FF972F4CEF85
:1040A00020F036EC66F09FD7579C010E70639BD7CB
:1040B0003894F70EF76EA40EF66E20EED6F018ECDC
:1040C00066F0F70EF76EB40EF66E20EEE6F018EC22
:1040D00066F036EC66F0010EBF1312D0F70EF76EE5
:1040E000640EF66E20EED6F018EC66F0F70EF76E62
:1040F000740EF66E20EEE6F018EC66F036EC66F024
:104100007DEC33F0320EAB6FAB67FED73D903D9246
:104110003D903D92E00EF76E040EF66E23EE00F039
:1041200011EC66F0DE6A02EC66F0640EAE6F140EFF
:10413000AD6F3DB0A1EF20F03DB2A1EF20F0AD6733
:10414000F8D7640EAE6F140EAD6FAD67FED738941E
:104150005DEF14F0010E8163DAD11EA417D0ACEC30
:1041600033F03BA003D03CB00BD050D6500EEA63E6
:1041700003D01EBE05D04AD616A648D648EF1FF07B
:1041800001EE60F0200EEF6201D0BCD0100E976FF0
:1041900001EE60F011EED2F0EECFE6FF972FFCD7E4
:1041A000A66BA76B76EC63F0A68F76EC63F0A78B1B
:1041B00076EC63F0809A358C320EAB6FAB67FED72E
:1041C00082AACCEF21F0358E640EAE6F0A0EAD6F71
:1041D000AD67FED744EC62F038BE0ED03D903D9204
:1041E000E00EF76E0A0EF66E23EE00F011EC66F0AC
:1041F000DE6A02EC66F0388EF70EF76ED40EF66EBD
:1042000020EED6F018EC66F036EC66F02CEC66F09A
:10421000640EAE6F050EAD6F3DB03D90AD67FCD73F
:10422000389401EED2F010EEE6F0100E976F0CAE5F
:10423000CDEC2DF00CBE0EEC2EF0E8664AD03DB071
:104240003D9057B03EEF21F057BC40EF21F058B001
:1042500045EF21F03DB247EF21F0A66BA76B76EC5E
:1042600063F0A68776EC63F0A78D76EC63F0A68DFD
:1042700076EC63F0A78376EC63F0B8D0579009D062
:10428000579C010E7063B2D004D0589002D03D927A
:1042900000D0F70EF76EA40EF66E20EED6F018ECF6
:1042A00066F0F70EF76EB40EF66E20EEE6F018EC40
:1042B00066F036EC66F0A66BA76B76EC63F0808A4E
:1042C000359C640EAE6F140EAD6FAD67FED788EFF0
:1042D0000FF0F90EF76EE40EF66E20EED6F018EC45
:1042E00066F0F90EF76EF40EF66E20EEE6F018ECBE
:1042F00066F036EC66F0808A359CA66BA76B76EC90
:1043000063F05FD0A66BA76B76EC63F0A68776ECC4
:1043100063F0A78D76EC63F0A68D76EC63F0A7834F
:1043200076EC63F0809A358C640EAB6FAB67FED78A
:1043300082AACCEF21F0358E3D903D92E20EF76ED1
:10434000400EF66E23EE00F011EC66F0DE6A02EC31
:1043500066F0640EAE6F0A0EAD6F3DB03D90AD6776
:10436000FCD73C9E349438BE41D0388E3D903D926F
:10437000E00EF76E0A0EF66E23EE00F011EC66F01A
:10438000DE6A02EC66F0640EAE6F0A0EAD6F3DB0F1
:104390003D90AD67FCD72AD0808A359C359EF70EBC
:1043A000F76E040EF66E20EED6F018EC66F0F70EFF
:1043B000F76E140EF66E20EEE6F018EC66F036ECB2
:1043C00066F03D903D92E00EF76E040EF66E23EE21
:1043D00000F011EC66F0DE6A02EC66F0640EAE6F7F
:1043E000140EAD6FAD67FED788EF0FF044EC62F0AE
:1043F000C8EC62F0A06B020EC06FC16BBF8FE60EFF
:10440000F76EF40EF66E20EED6F018EC66F02CEC9B
:1044100066F001EE8CF0200EEF5C09E010EEE6F0A5
:10442000100E976FEECFE6FF972F12EF22F036ECCB
:1044300066F0A0B10CD03DB03D9057B033EF22F004
:1044400057BC37EF22F058B035EF22F0F2D73CAE30
:10445000F8EC3AF03C8E1FEC62F0230E9D63E9D736
:104460001EACE7D735D0579006D0589004D0579C53
:10447000010E7063DED7F70EF76EA40EF66E20EE17
:10448000D6F018EC66F0F70EF76EB40EF66E20EE6E
:10449000E6F018EC66F036EC66F0A66BA76B76ECEF
:1044A00063F0808A359C3D903D92E00EF76E040EDD
:1044B000F66E23EE00F011EC66F0DE6A02EC66F0B8
:1044C000640EAE6F140EAD6FAD67FED788EF0FF0C0
:1044D000F70EF76EE40EF66E20EED6F018EC66F0EE
:1044E000F70EF76EF40EF66E20EEE6F018EC66F0BE
:1044F00036EC66F0A66BA76B76EC63F0808A359C91
:10450000640EAE6F140EAD6FAD67FED739D6020ED6
:104510008163EFEF22F0100E976F11EE8CF001EE39
:104520009EF0E6CFEEFF972FFCD7F8EC33F03BA0E0
:10453000ADD43CA420D03B903B923D903D92E00E08
:10454000F76E040EF66E23EE00F011EC66F0DE6AF4
:1045500002EC66F03DB0B1EF22F03DB2B1EF22F0D7
:10456000F9D73D903D923D963B86640EB96F320E71
:10457000B86FE7EF0FF0F80EF76E240EF66E20EE30
:10458000D6F018EC66F0F80EF76E340EF66E20EEEC
:10459000E6F018EC66F036EC66F03B903B923D900E
:1045A0003D92E00EF76E040EF66E23EE00F011EC75
:1045B00066F0DE6A02EC66F0640EAE6F140EAD6F4C
:1045C0003DB0E8EF22F03DB2E8EF22F0AD67F8D75A
:1045D000AD67FED73D903D923D96E7EF0FF01EC0D0
:1045E00081F0030E8117030E816388EF0FF0100E28
:1045F000976F11EE8CF001EE9EF0E6CFEEFF972F55
:10460000FCD746EC34F03CA6B6D73B903B923D90AD
:104610003D92E00EF76E040EF66E23EE00F011EC04
:1046200066F0DE6A02EC66F03DB01BEF23F03DB2AF
:104630001BEF23F0F9D73D903D923D963B86640EEB
:10464000B96F320EB86FE7EF0FF038EC30F0E86674
:1046500002D039B60AD0E70EF76EB40EF66E20EE31
:10466000D6F018EC66F039960AD0E70EF76EC40E55
:10467000F66E20EED6F018EC66F039823984E60E3C
:10468000F76EC40EF66E20EED6F018EC66F036EC3F
:1046900066F03886ABEC30F0E86688EF0FF011EC8E
:1046A00029F0E60EF76EE40EF66E20EED6F018EC6A
:1046B00066F0310E39B4320EE56F36EC66F0640EFA
:1046C000AE6FFA0EAD6F3DB099EF23F057B078EFB3
:1046D00023F057BC7AEF23F058B07FEF23F03EB0C1
:1046E00081EF23F03EB28DEF23F0AD67ECD7B2D26D
:1046F0005790B0D2579C010E7063E5D7ABD258905B
:10470000A9D23E90FE0EF76E420EF66E20EED6F067
:1047100018EC66F036EC66F09DD23E92FE0EF76E17
:10472000320EF66E20EED6F018EC66F036EC66F03F
:1047300091D244EC62F0C8EC62F0A06BA66BA76B60
:1047400076EC63F0A78776EC63F0A78D76EC63F0E8
:10475000E70EF76E040EF66E20EED6F018EC66F05B
:104760002CEC66F051EC5DF036EC66F0050EC06F97
:10477000C16BBF8F9E6BA0B11CD03DB03D9057B0B8
:10478000D0EF23F057BCD2EF23F058B0D7EF23F08F
:104790003DB4CCEF23F0EFD73D9446EC34F0EBD7AB
:1047A000579058D2579C010E7063E5D753D288EFCB
:1047B0000FF0D2EC61F01FEC62F0230E9D5DD0E0B3
:1047C00000EEE6F011EED2F09DC0EEFF9DC0E6FFD8
:1047D00036EC66F09E2B640EAE6F17C0ADF0A0B144
:1047E00011D03DB03D9057B03CEF24F057BC3EEFA8
:1047F00024F058B043EF24F03DB438EF24F0AD6717
:10480000EED743D01FEC62F0230E9D6301D0A8D7F2
:104810009E2B110E9E6107D09DC0EEFF9DC0E6FF4E
:1048200036EC66F0D8D7E7C0E6F0E8C0E7F0E9C0BC
:10483000E8F0EAC0E9F0EBC0EAF0ECC0EBF0EDC064
:10484000ECF0EEC0EDF0EFC0EEF0F0C0EFF0F1C034
:10485000F0F0F2C0F1F0F3C0F2F0F4C0F3F0F5C004
:10486000F4F09DC0EEFF9DC0F5F036EC66F0B3D7D6
:104870003D9446EC34F0B3D75790ECD1579C010EE1
:104880007063ADD7E7D188EF0FF038EC30F0E86611
:1048900001D0CBD0809A358C640EAB6FAB67FED75E
:1048A00082AACCEF21F0358EA66BA76B76EC63F075
:1048B000A68F76EC63F0A78D76EC63F0A68D76EC90
:1048C00063F0A78376EC63F0640EAE6F080EAD6FF5
:1048D000AD67FED79E6B01EED2F011EE78F0200EA0
:1048E000E76430D0040E976FEF50E7622BD0EE50A4
:1048F000E650200EE76201D002D0972FF5D797C07F
:104900009AF010EEE6F0040E976F01EE78F00CAE20
:10491000CDEC2DF00CBE0EEC2EF0E8665DD00F5005
:1049200009E0976F640EAE6F0A0EAD6FAD67FED7EC
:10493000972FF8D701EED2F09A510508E926E86AD8
:10494000EA2204D001EED2F010EEE6F0200E976FCE
:104950000CAECDEC2DF00CBE0EEC2EF0E8663CD08B
:10496000A66BA76B76EC63F0A68776EC63F0A78D59
:1049700076EC63F0A68D76EC63F0A78376EC63F0BB
:10498000F6EF21F0808A359C359EF90EF76E540EB5
:10499000F66E20EED6F018EC66F0F90EF76E640EA7
:1049A000F66E20EEE6F018EC66F036EC66F03D9020
:1049B0003D92E00EF76E040EF66E23EE00F011EC61
:1049C00066F0DE6A02EC66F0640EAE6F140EAD6F38
:1049D000AD67FED788EF0FF0808A359CF90EF76E31
:1049E000E40EF66E20EED6F018EC66F0F90EF76ED7
:1049F000F40EF66E20EEE6F018EC66F036EC66F09B
:104A00003D903D92E00EF76E040EF66E23EE00F040
:104A100011EC66F0DE6A02EC66F0640EAE6F140E06
:104A2000AD6FAD67FED788EF0FF0FD0EF76EF20E9B
:104A3000F66E20EED6F018EC66F02CEC66F09EC018
:104A400097F001EED2F010EEE6F0EECFE6FF972FF2
:104A5000FCD736EC66F03D903D92E30EF76E700E9B
:104A6000F66E23EE00F011EC66F0DE6A02EC66F002
:104A7000640EAE6F320EAD6F3DB04CEF25F03DB21F
:104A80004FEF26F057BC48EF25F0AD67F5D7E2D0E1
:104A9000579C010E7063F0D703EE00F0410EEE6EEE
:104AA000540EEE6E440EEE6E9EC097F011EED2F0F4
:104AB000E6CFEEFF972F58EF25F03B0EEE6E000E7F
:104AC000EE6E3D6A3E6A576A586A02EC66F0FE0E68
:104AD000F76E220EF66E20EED6F018EC66F036EC8D
:104AE00066F03C0EBA6F57B091EF25F057BC93EFCC
:104AF00025F058B098EF25F058B29AEF25F03DB266
:104B00009CEF25F03DB0BEEF25F03EB09EEF25F0C6
:104B10003EB2AAEF25F03DB4B6EF25F0BA67E3D771
:104B200099D0579097D0579C010E7063DCD792D0E4
:104B3000589090D05892D7D73D928CD03E90FE0E90
:104B4000F76E420EF66E20EED6F018EC66F036ECFC
:104B500066F080D03E92FE0EF76E320EF66E20EEBC
:104B6000D6F018EC66F036EC66F074D03D94030E87
:104B70001E140208D8B446EC34F0B5D73D903D90F1
:104B80003D92E30EF76E880EF66E23EE00F011EC08
:104B900066F0DE6A02EC66F0FE0EF76E520EF66EFE
:104BA00020EED6F018EC66F0C8EC62F01FEC62F074
:104BB000A06B36EC66F0A0B113D057B0F6EF25F03D
:104BC00057BC02EF26F058B0F8EF25F03DB0FAEFF1
:104BD00025F03DB2FCEF25F03DB4FEEF25F0EBD71C
:104BE0001FEC62F0230E9D63E6D715D0579032D0AC
:104BF000589030D03D90DFD73D9251D03D9446EC57
:104C000034F0D9D7579C010E706301D023D0579C44
:104C1000020E7063D0D71EAC1DD03D903D92E30EC6
:104C2000F76E7C0EF66E23EE00F011EC66F0DE6A95
:104C300002EC66F0640EAE6F320EAD6F3DB027EF42
:104C400026F03DB24FEF26F0AD67F8D703D0388E8F
:104C500099EF23F0FE0EF76E020EF66E20EED6F000
:104C600018EC66F0FE0EF76E120EF66E20EEE6F011
:104C700018EC66F03D903D92E00EF76E040EF66E75
:104C800023EE00F011EC66F0DE6A02EC66F0640ED2
:104C9000AE6F140EAD6FAD67FED788EF0FF0FE0E4E
:104CA000F76E620EF66E20EED6F018EC66F0FE0E91
:104CB000F76E720EF66E20EEE6F018EC66F036EC4B
:104CC00066F03D903D92E00EF76E040EF66E23EE18
:104CD00000F011EC66F0DE6A02EC66F0640EAE6F76
:104CE000140EAD6FAD67FED788EF0FF0B86742EFD7
:104CF00010F0400E976F14EEC0F0E76606D0E65055
:104D0000972FFBD73B9642EF10F03B94E7B23B84E2
:104D1000E76A97514008A26F9E6B15EE08F00A0EE5
:104D2000A203F350E126F450E222E7CF3CF051EC2D
:104D30005DF001EED2F015EE00F00A0EA203F35082
:104D4000E126F450E222080ECB6F200E806FE73888
:104D50000F0B300F816F3F0E816180C081F0080E14
:104D6000CB6305D03B0E816302D02B0E816F81C0D7
:104D7000EEFF200E815D12E09E2BE6500F0B9A6F26
:104D8000300F816F3F0E816180C081F081C0EEFFE6
:104D9000200E815F03E09E2BCB2FD9D71EC081F060
:104DA000030E8117020E816325EF23F03BB402D07E
:104DB0001EB6BAD038EC30F0E86602D039B60AD068
:104DC000E70EF76EB40EF66E20EED6F018EC66F035
:104DD00039960AD0E70EF76EC40EF66E20EED6F0C6
:104DE00018EC66F039823984E60EF76EC40EF66E62
:104DF00020EED6F018EC66F036EC66F03886ABECB8
:104E000030F0E86688EF0FF011EC29F0E60EF76E4F
:104E1000E40EF66E20EED6F018EC66F0310E39B4E2
:104E2000320EE56F36EC66F0640EAE6FFA0EAD6FC3
:104E30003DB051EF27F057B02DEF27F057BC2FEFC3
:104E400027F058B034EF27F03EB036EF27F03EB2EF
:104E500043EF27F0AD67ECD722D0579020D0579C76
:104E6000010E7063E5D71BD0589019D03E90FD0E0F
:104E7000F76EB40EF66E20EED6F018EC66F036EC57
:104E800066F04FEF27F03E92FD0EF76ED40EF66EF1
:104E900020EED6F018EC66F036EC66F000D03BEF72
:104EA00022F0388E3BA4C0EF20F01DEE00F0080E7B
:104EB000A203F350E126F450E22251EC5DF09E6B28
:104EC00001EED2F0080ECB6F200E806FE7380F0B8B
:104ED000300F816F3F0E816180C081F081C0EEFF95
:104EE000200E816512D09E2BE6500F0B9A6F300F6B
:104EF000816F3F0E816180C081F081C0EEFF200E86
:104F0000816503D09E2BCB2FE1D71DEE00F0080E5C
:104F1000A203F350E126F450E222080E976FE668F0
:104F2000972FFDD7D0EF20F0E70EF76E540EF66EF8
:104F300020EED6F018EC66F02CEC66F036EC66F05D
:104F4000809A358CA66BA76B76EC63F0A68F76EC17
:104F500063F0A68976EC63F0A68376EC63F0320EFC
:104F6000AB6FAB67FED782AAF4EF28F0358E640EE4
:104F7000AE6F080EAD6FAD67FED79E6B01EED2F03F
:104F80002B0EEF6202D001EED3F011EE70F0200E86
:104F9000E76435D0080E976FEF50E76230D0EE50DF
:104FA000E650200EE76201D002D0972FF5D797C0C8
:104FB0009AF010EEE6F0040E976F01EE78F00CAE6A
:104FC000CDEC2DF00CBE0EEC2EF0E866F1D00F50BB
:104FD00009E0976F640EAE6F0A0EAD6FAD67FED736
:104FE000972FF8D701EED2F02B0EEF6202D001EE30
:104FF000D3F09A510908E926E86AEA224AD001EE7C
:10500000D2F02B0EEF6202D001EED3F011EE78F069
:10501000200EE76435D0040E976FEF50E76230D072
:10502000EE50E650200EE76201D002D0972FF5D760
:1050300097C09AF010EEE6F0040E976F01EE78F04C
:105040000CAECDEC2DF00CBE0EEC2EF0E866B0D020
:105050000F5009E0976F640EAE6F0A0EAD6FAD672B
:10506000FED7972FF8D701EED2F02B0EEF6202D0C9
:1050700001EED3F09A510508E926E86AEA2209D040
:1050800001EED2F02B0EEF6202D001EED3F010EE63
:10509000E6F0200E976F0CAECDEC2DF00CBE0EECB2
:1050A0002EF0E86685D0A66BA76B76EC63F0A78937
:1050B00076EC63F0A68776EC63F019EC2FF016B46B
:1050C0000ED0140E6C6F1AC06DF03A903A923A8678
:1050D0003A94C56B80868094809280802BD016A0F5
:1050E00012D078EC33F04EEC2EF0140E6C6F1AC028
:1050F0006DF03A903A923A863A94C56B80868094E5
:105100008092808017D0140E6C6F1AC06DF03A90A8
:105110003A923A863A94C56B8086809480928080D9
:105120003AA4FED7640EAE6F060EAD6FAD67FED724
:105130009FEC2EF0640EB06FFA0EAF6F81B2A8EF45
:1051400028F0640EAB6FAB67FED781A2CFEF28F0DB
:10515000AF67F4D7808A359CA66BA76B76EC63F0BB
:10516000F80EF76E040EF66E20EED6F018EC66F030
:10517000F80EF76E140EF66E20EEE6F018EC66F000
:1051800036EC66F03A6A8086809480828090640E65
:10519000AE6F140EAD6FAB67FED788EF0FF03A6AB3
:1051A000808680948082809071EC33F07AEF16F0E4
:1051B000808A359CF90EF76EE40EF66E20EED6F07E
:1051C00018EC66F0F90EF76EF40EF66E20EEE6F0CF
:1051D00018EC66F036EC66F0640EAE6F140EAD6F30
:1051E000AD67FED788EF0FF0808A359C359EF90EAB
:1051F000F76E540EF66E20EED6F018EC66F0F90E4F
:10520000F76E640EF66E20EEE6F018EC66F036EC03
:1052100066F0640EAE6F140EAD6FAD67FED788EF0B
:105220000FF02CEC66F09E6B11EED2F003EE00F066
:10523000410EEE6E540EEE6E440EEE6E200E976F23
:10524000E750200804E0E6CFEEFF972FF9D73B0E9A
:10525000EE6E000EEE6E00EEE6F011EED2F0100EE5
:10526000976FE750200804E0E6CFEEFF972FF9D7BD
:1052700036EC66F03D903D923E6A57905794579AAF
:10528000579C589002EC66F01200140E976F00EED7
:1052900043F0426AEF6607D0422AEE50972FFAD7C2
:1052A000389A88EF0FF0EF6A200E976F08EE32F011
:1052B000200EEE6E972FFCD73F9E42C084F07CEC10
:1052C00061F03D903D9203EE00F0410EEE6E540E03
:1052D000EE6E2B0EEE6E430EEE6E4D0EEE6E470E24
:1052E000EE6E520EEE6E3D0EEE6E300E7F637FC0A0
:1052F000EEFF806380C0EEFF81C0EEFF000EEE6E19
:1053000002EC66F0640EAE6FFA0EAD6F3DB0A1EF29
:1053100029F03DB28EEF29F0AD67F8D73D92FA0E35
:10532000F76E240EF66E20EEE6F018EC66F036EC22
:1053300066F0640EAE6F1E0EAD6FAD67FED788EFE0
:105340000FF03D902EA0EED018EE52F0430EE66224
:105350006CD0620EE662A5D2120E976F01EEB0F02D
:10536000200EEE6E972FFCD7000EE7620BD0120EC8
:10537000976F18EE32F001EEB0F0E6CFEEFF972F08
:10538000FCD70BD0100E976F01EEB0F0000EE75C6B
:1053900004E0E6CFEEFF972FF9D77EEC2DF03BA08F
:1053A0009BD23CA414D01E50030B020828E13B867C
:1053B00014EEC0F0A251E126E86AE222E768640E2A
:1053C000B96F140EB86F43EC2DF088EF0FF0FA0EA2
:1053D000F76E840EF66E20EEE6F018EC66F000EE46
:1053E000D6F011EEB0F0100E976FE6CFEEFF972FCC
:1053F000FCD736EC66F043EC2DF088EF0FF0FF0E93
:10540000F76E220EF66E20EED6F018EC66F0FF0E68
:10541000F76E320EF66E20EEE6F018EC66F036EC23
:1054200066F043EC2DF088EF0FF02EA27BD0120E29
:10543000976F08EE00F011EEB0F0200EEE6EE66E03
:10544000972FFBD718EE52F0530EE6626BD0630E27
:10545000E66227D2000EE75CD8B423D2100E976F15
:1054600008EE00F02E0EE75C07E0000EE75C04E0BB
:10547000E6CFEEFF972FF6D7000EE7620BD0120EA5
:10548000976F18EE32F001EEB0F0E6CFEEFF972FF7
:10549000FCD711D02E0EE66204D2000EE75CEFE0DE
:1054A000100E976F01EEB0F0000EE75C04E0E6CF5F
:1054B000EEFF972FF9D73C6A7EEC2DF03BA00CD283
:1054C0003CA485D71E50030B020899E13B8614EEDD
:1054D000C0F0A251E126E86AE222020EE76E1DEE5C
:1054E00000F0080EA203F350E126F450E222080E69
:1054F000CB6F08EE00F0200EEF64EF68EE38F00B93
:10550000816F200EEF64EF680F0EEE148111E66ECE
:10551000CB2FF1D7640EB96F140EB86F43EC2DF09A
:1055200088EF0FF02EB41CD0FC0EF76ED40EF66E82
:1055300020EED6F018EC66F0FC0EF76EE40EF66E78
:1055400020EEE6F018EC66F036EC66F043EC2DF059
:10555000640EAE6F140EAD6FAD67FED788EF0FF01F
:1055600001EE2EF0200EEF5C19E0100E976F01EEA9
:105570002EF018EE32F02B0EE76202D018EE33F068
:10558000EE50E6620BD0972FFBD7100E976F01EE0F
:10559000B0F0200EEE6E972FFCD712D02EA810D0B0
:1055A000100E976F01EE1CF018EE32F02B0EE76232
:1055B00002D018EE33F0EE50E66285D1972FFBD77C
:1055C000080E976F01EE0CF018EE52F0200EEF620D
:1055D00002D0EE5005D0EE50E6625AD1972FF6D7A2
:1055E000100E976F01EEB0F0200EEE6E972FFCD7E5
:1055F0002E0EE66256D1410EE6629DD0640EE66242
:1056000099D0640EE66295D02E0EE66291D0100E0F
:10561000976F01EEB0F02E0EE75C04E0E6CFEEFFF0
:10562000972FF9D72E0EE6623CD13C6A590EE762FD
:1056300002D03C8004D04E0EE76233D13C90E6505D
:105640002E0EE6622ED1590EE76202D03C8204D0C3
:105650004E0EE76226D13C92E6502E0EE66221D134
:10566000590EE76202D03C8404D04E0EE76219D195
:105670003C94E6502E0EE66214D1590EE76202D039
:105680003C8604D04E0EE7620CD13C96E6502E0EBE
:10569000E66207D1590EE76202D03C8804D04E0E74
:1056A000E762FFD03C987EEC2DF03BA00BD015EECE
:1056B00008F00A0EA203F350E126F450E2223CC0A7
:1056C000E7FF21D0B9EC2DF03BA0F4D015EE00F0AF
:1056D0000A0EA203F350E126F450E222080ECB6F2B
:1056E00001EEB0F0200EEF64EF68EE38F00B816F42
:1056F000200EEF64EF680F0EEE148111E66ECB2FD3
:10570000F1D73CC0E6FF05EE00F00A0EA203F3500D
:10571000E926F450EA22010EAA6E200EA96EF3507B
:10572000A926F450AA220A0ECB6FE9EC65F0E9D065
:10573000E106E106E106E106430EE66243D06C0EA7
:10574000E6623FD0720EE6623BD02E0EE66237D0A4
:10575000100E976F01EEB0F0000EE75C07E02E0E22
:10576000E75C04E0E6CFEEFF972FF6D77EEC2DF056
:105770003BA0B2D015EE00F00A0EA203F350E126D2
:10578000F450E222080ECB6FFF0EE66ECB2FFCD753
:10579000E66AE66805EE00F00A0EA203F350E92679
:1057A000F450EA22010EAA6E200EA96EF350A9262B
:1057B000F450AA220A0ECB6FE9EC65F0A2D0E10604
:1057C000E106E106E106460EE6626BD06C0EE6628B
:1057D00068D06D0EE66265D02E0EE66262D0100EC5
:1057E000976F01EEB0F02E0EE75C0AE02F0EE76433
:1057F00058D03A0EE76055D0E6CFEEFF972FF3D79B
:105800002E0EE6624ED03C6A590EE76202D03C682A
:1058100004D04E0EE76245D03C6AE6502E0EE6629A
:1058200040D02F0EE7643DD03A0EE7603AD0E6CF85
:105830009AF00F0E9A17100E976F11EEB0F001EE5E
:1058400050F0E6CFEEFF972FFCD7FC0E0C16020EA1
:105850003C660C129AC00EF0030EAA6E9E0E100E3D
:10586000CB6F05EE00F0E9EC65F0030EAA6E020EB8
:1058700000EE0EF0010ECB6FE9EC65F0030EAA6EA0
:10588000000E00EE0CF0010ECB6FE9EC65F039D0A4
:10589000FA0EF76E340EF66E20EEE6F018EC66F0B7
:1058A00023D0FA0EF76E440EF66E20EEE6F018ECFA
:1058B00066F01AD0FA0EF76E540EF66E20EEE6F091
:1058C00018EC66F011D0FA0EF76E640EF66E20EE4C
:1058D000E6F018EC66F008D0FA0EF76E740EF66E6D
:1058E00020EEE6F018EC66F03F8E00EED6F011EEFA
:1058F000B0F0100E976FE6CFEEFF972FFCD736EC87
:1059000066F043EC2DF02EA688EF0FF03D903D920F
:1059100003EE00F0410EEE6E540EEE6E2B0EEE6EA8
:10592000430EEE6E4D0EEE6E470EEE6E530EEE6EA5
:105930003D0EEE6E220EEE6E200E976F18EE32F0D8
:10594000200EE75C04E0E6CFEEFF972FF9D7220E9A
:10595000EE6EEE6A02EC66F0640EAE6F320EAD6F64
:105960003DB2B8EF2CF03FB2BAEF2CF0AD67F8D7EC
:105970003D926FD03F9203EE00F0530EEE6E4D0E4F
:10598000EE6E530EEE6E200EEE6E530EEE6E650E44
:10599000EE6E740EEE6E750EEE6E700EEE6E200EE6
:1059A000EE6E2F0EEE6E400E976F18EE52F0000E58
:1059B000E75C04E0E6CFEEFF972FF9D72F0EEE6EEF
:1059C000200EEE6E770EEE6E610EEE6E730EEE6EC4
:1059D000200EEE6E3FAE0DD0660EEE6E610EEE6ED8
:1059E000690EEE6E6C0EEE6E650EEE6E640EEE6E71
:1059F00012D0730EEE6E750EEE6E630EEE6EEE6EE0
:105A0000650EEE6E730EEE6EEE6E660EEE6E750E3B
:105A1000EE6E6C0EEE6E1A0EEE6EEE6A3D903D92DC
:105A20003F9402EC66F0640EAE6F320EAD6F3DB285
:105A300022EF2DF03DB026EF2DF03FB424EF2DF0F6
:105A4000AD67F5D73D9205D03F94F1D73D9088EFF3
:105A50000FF0FC0EF76E140EF66E20EED6F018EC7A
:105A600066F0FC0EF76E240EF66E20EEE6F018ECF3
:105A700066F036EC66F0640EAE6F140EAD6FAD6777
:105A8000FED788EF0FF0640EB06F140EAF6F42C0F8
:105A900084F07CEC61F03D903D9203EE00F0410E0D
:105AA000EE6E540EEE6E2B0EEE6E430EEE6E4D0E3F
:105AB000EE6E470EEE6E440EEE6E3D0EEE6E300E46
:105AC0007F637FC0EEFF806380C0EEFF81C0EEFF8A
:105AD000000EEE6E02EC66F0640EAE6FFA0EAD6F65
:105AE0003DB07AEF2DF03DB278EF2DF0AD67F8D7ED
:105AF0003D9201D03D90AF67FED71200A26B3B9064
:105B000015EE00F00A0EA203F350E126F450E22253
:105B100001EEB0F0FF0EE76026D0080ECB6FE7383D
:105B20000F0B300F806F080ECB6305D03B0E8063E8
:105B300002D02B0E806FE6500F0B300F816F200EBE
:105B40009A6F3F0E80619AC080F081619AC081F0A7
:105B5000EE50806308D0EE50816305D0CB2FDFD7A5
:105B60003C843B801200A22B400EA263C9D73B901D
:105B70001200A26B15EE00F00A0EA203F350E1260C
:105B8000F450E222FF0EE76202D03B801200A22B0B
:105B90003F0EA265EFD73B901200640EAB6FAB6770
:105BA000FED7EECF9DF0200E9D5DD8B436D028EC08
:105BB0005DF012EC62F0640EAB6FAB67FED7D2EC17
:105BC00061F0110E9E6103D09DC0E6FF20D0E7C0BA
:105BD000E6F0E8C0E7F0E9C0E8F0EAC0E9F0EBC0C1
:105BE000EAF0ECC0EBF0EDC0ECF0EEC0EDF0EFC091
:105BF000EEF0F0C0EFF0F1C0F0F0F2C0F1F0F3C061
:105C0000F2F0F4C0F3F0F5C0F4F09DC0F5F036EC1E
:105C100066F0974F02D09E2BC0D7000C640EAE6F7B
:105C2000050EAD6FAD67FED7EECF9DF0200E9D5DEA
:105C300033E012EC5DF00B0E9F612FD055EC18F0A5
:105C4000110E9E6103D09DC0E6FF20D0E7C0E6F0B4
:105C5000E8C0E7F0E9C0E8F0EAC0E9F0EBC0EAF03C
:105C6000ECC0EBF0EDC0ECF0EEC0EDF0EFC0EEF00C
:105C7000F0C0EFF0F1C0F0F0F2C0F1F0F3C0F2F0DC
:105C8000F4C0F3F0F5C0F4F09DC0F5F036EC66F02A
:105C9000974F02D09E2BC2D7000CFF0CC80EAB6FE3
:105CA000AB67FED7640EAB6F0BEC62F0AB67FED751
:105CB000D2EC61F03C0EAB6FAB67FED7110ECE6F2E
:105CC000000ECF6FF3EC62F0300ECE6F180ECF6F78
:105CD000F8EC62F0960EAB6FAB67FED7300ECE6F6E
:105CE000160ECF6FF8EC62F03C0EAB6FAB67FED7D1
:105CF000110ECE6F480ECF6FF3EC62F081B0FED77D
:105D00000CEC63F004EE00F0EECFCEF002EC63F0AA
:105D100081B0FED70CEC63F081B0FED70CEC63F0E1
:105D2000CB2FF2D7110ECE6F000ECF6FF3EC62F0D7
:105D300018EC62F0FA0EAB6FAB67FED71200110ED3
:105D4000CE6F000ECF6FF3EC62F0300ECE6F180EF8
:105D5000CF6FF8EC62F0FA0EAB6FAB67FED7300E88
:105D6000CE6F160ECF6FF8EC62F0960EAB6FAB678E
:105D7000FED7110ECE6F480ECF6FF3EC62F081B0FC
:105D8000FED70CEC63F004EE00F0EECFCEF002ECA8
:105D900063F081B0FED70CEC63F081B0FED70CEC61
:105DA00063F0CB2FF2D7110ECE6F000ECF6FF3EC56
:105DB00062F018EC62F01200110ECE6F000ECF6F81
:105DC000F3EC62F0500ECE6F180ECF6FF8EC62F06D
:105DD000FA0EAB6FAB67FED7500ECE6F160ECF6FBD
:105DE000F8EC62F0960EAB6FAB67FED7110ECE6F7C
:105DF000480ECF6FF3EC62F081B0FED70CEC63F08D
:105E000004EE00F0EECFCEF002EC63F081B0FED7EE
:105E10000CEC63F081B0FED70CEC63F0CB2FF2D723
:105E2000110ECE6F000ECF6FF3EC62F018EC62F043
:105E30001200CB6B04EE00F0800EEE6E000EEE6EE4
:105E4000020EEE6E000EEE6E11EE8CF0200EE7628A
:105E500005D0500EEE6E010ECB270AD0100E976FB4
:105E6000200EE75C05E0CB2BE6CFEEFF972FF8D7AF
:105E7000CBC003F4020ECB27CBC001F4020ECB271C
:105E8000CBC097F004EE00F0C86BEE50C827972FF8
:105E900045EF2FF0C81F010EC827C8C0EEFFCB2B5F
:105EA0001200376A100E976F01EEC2F0200EEE6EF0
:105EB000972FFCD708EE52F0500E976FEE6A972F8F
:105EC0005EEF2FF00CEC63F007EC63F03E0ECE6F4C
:105ED000160ECF6FFDEC62F0110ECE6F420ECF6F3B
:105EE000F3EC62F0640EB06F140EAF6FAF51D8B424
:105EF0009AD081B0FBD70CEC63F0CEC09AF007ECDF
:105F000063F09AA3F3D7AF51D8B48DD081B0FBD74B
:105F10000CEC63F0CFC09AF007EC63F09AAFF3D7C4
:105F20003E0ECE6F360ECF6FFDEC62F0110ECE6FCF
:105F3000410ECF6FF3EC62F0C86BCB6B08EE52F002
:105F4000AF5171E081B0FCD70CEC63F007EC63F06B
:105F5000CEC0EEFFCE51C827CB2BAF5164E081B04D
:105F6000FCD70CEC63F007EC63F0CEC0EEFFCEC0C4
:105F700097F0CE51C827CB27CB2B97510FE0AF51CD
:105F800052E081B0FCD70CEC63F007EC63F0CEC0BC
:105F9000EEFFCE51C827972FBFEF2FF0AF5143E050
:105FA00081B0FCD70CEC63F007EC63F0CEC0EEFFE1
:105FB000CE51C827CB2B110ECE6F000ECF6FF3EC56
:105FC00062F0C8672BD018EE52F0800EE66226D041
:105FD000E6CF97F0020EE76214D0E650E6CFCBF0A2
:105FE000500EE7601DD0CB5119E0100ECB6501D0EB
:105FF000CB6F01EEC2F0E6CFEEFFCB2FFCD73780A0
:106000001200040EE76201D00BD0E650E6CFCBF0D1
:10601000E650974F03D0CB2FFBD7DCD73784120045
:10602000378237801200FAD7120037A016D037B265
:106030000BD0100E976F11EEC2F000EEE6F0E6CF37
:10604000EEFF972FFCD711D0E70EF76E340EF66EE9
:1060500020EEE6F018EC66F008D0E70EF76E440E7E
:10606000F66E20EEE6F018EC66F036EC66F0120004
:1060700004EE40F0200E976F8B6BFF0EEF5C58E044
:10608000EF380F0B7A6FEE500F0B7B6FEF380F0B63
:106090007C6FEE500F0B7D6FEF380F0B7E6FEE5065
:1060A0000F0B7F6FEF380F0B806FEE500F0B816F70
:1060B0000F0E815D3DE00A0E7A6303D0FA0E7A6F0F
:1060C00005D00B0E7A6302D0FB0E7A6F300E7A2762
:1060D0007B277C277D277E277F27802711EED2F024
:1060E0007A51E66225D03F0E7B5D30E07B51E6625F
:1060F0001FD03F0E7C5D2AE07C51E66219D03F0E36
:106100007D5D24E07D51E66213D03F0E7E5D1EE092
:106110007E51E6620DD03F0E7F5D18D07F51E66262
:1061200007D03F0E805D12D08051E66201D00ED0C4
:106130008B2B040E8B03F35004EE40F0E926E86A43
:10614000EA22972F3DEF30F03996FF0C3996010E79
:1061500081633986000C39B607D039B202D038B223
:10616000AED23992399402D0398400D03892399223
:1061700039905790640EAE6F140EAD6F57B0C3EFE9
:1061800030F0AD67FBD75790389239B4838C39A47F
:10619000839C3D6A576A586A596A39803D903D929E
:1061A000E00EF76EE00EF66E23EE00F011EC66F0F6
:1061B000DE6A02EC66F0640EAE6F320EAD6F3DB07B
:1061C000EAEF30F03DB2E8EF30F0AD67F8D73AD003
:1061D0003D9238D03D90640EB06FFA0EAF6F57B05D
:1061E00021EF32F057B239EF32F057B68AEF32F082
:1061F00059B0C9EF32F059B2CCEF32F059B432EFA6
:1062000033F059B634EF33F059B848EF33F059BA98
:106210005CEF33F03DB235EF31F0AF67E0D7E50E1C
:10622000F76E540EF66E20EED6F018EC66F0E50E22
:10623000F76E640EF66E20EEE6F018EC66F036ECC3
:1062400066F040D2F90EF76EA40EF66E20EED6F090
:1062500018EC66F0F90EF76EB40EF66E20EEE6F06E
:1062600018EC66F036EC66F02DD23D923DB812D0B7
:106270000A0E405CD8B4A3D00B0E405C58E00C0E64
:10628000405C42E00D0E405C2BE0100E405CD8B448
:10629000B2D000D0F80EF76ED40EF66E20EED6F027
:1062A00018EC66F0F80EF76EE40EF66E20EEE6F0EF
:1062B00018EC66F010EEEEF0826B40C083F098ECC4
:1062C00061F0350E3DB87F6F300E7F637FC0E6FF13
:1062D000806380C0E6FF81C0E6FF36EC66F0F2D155
:1062E000F90EF76E840EF66E20EED6F018EC66F01E
:1062F000F90EF76E940EF66E20EEE6F018EC66F0EE
:1063000036EC66F00000DED1F80EF76EB40EF66ED5
:1063100020EED6F018EC66F0F80EF76EC40EF66EAE
:1063200020EEE6F018EC66F036EC66F0CBD111EE1C
:1063300040F039B411EE48F0200EE75CD8B46ED0CE
:1063400003EE00F0410EEE6E540EEE6E2B0EEE6E6E
:10635000430EEE6E500EEE6E490EEE6E4E0EEE6E6B
:106360003D0EEE6E080E976F200EE75C05E0E6CF5F
:10637000EEFF972FB4EF31F0000EEE6E3D903D92A0
:1063800002EC66F0640EAE6F320EAD6F3DB0CFEF33
:1063900031F03DB2D1EF31F0AD67F8D7A1D73D90E4
:1063A0001ED73D923DB876D70A0E405C08E00C0E31
:1063B000405CD8B4A9D7100E405C1DE06BD73D926D
:1063C000E40EF76EF40EF66E20EED6F018EC66F0E2
:1063D000E40EF76EE40EF66E20EEE6F018EC66F0D2
:1063E000310E39B4320EF06F39A4399C39B4399E6C
:1063F00036EC66F067D1F80EF76EA40EF66E20EE5E
:10640000D6F018EC66F0F90EF76E740EF66E20EE0C
:10641000E6F018EC66F036EC66F054D1F80EF76E44
:10642000540EF66E20EED6F018EC66F0F80EF76E0D
:10643000640EF66E20EEE6F018EC66F036EC66F0D0
:1064400041D15790E40EF76E940EF66E20EED6F022
:1064500018EC66F0E40EF76EB40EF66E20EEE6F081
:1064600018EC66F0310E39B4320EDC6F36EC66F0A3
:1064700029D157923D903D923D983D903D92E10E3D
:10648000F76EC80EF66E23EE00F011EC66F0DE6AD1
:1064900002EC66F0640EAE6F320EAD6F3DB068EF89
:1064A00032F03DB25AEF32F03DBC6AEF32F0AD67E8
:1064B000F5D7C8D63DA893D63D983D920F0E4062C1
:1064C000C1D6640EAE6F050EAD6FAD67FED7D5D7E2
:1064D0003D9085D63D9C000E6F6301D080D6010EA5
:1064E0006F6301D024D7020E6F6301D00DD7F90E70
:1064F000F76EC40EF66E20EED6F018EC66F0F90ECC
:10650000F76ED40EF66E20EEE6F018EC66F036EC80
:1065100066F0D8D057963D903D923D903D92E10E69
:10652000F76E040EF66E23EE00F011EC66F0DE6AF4
:1065300002EC66F0640EAE6F320EAD6F3DB0A9EFA7
:1065400032F03DB2A7EF32F0AD67F8D77BD63D927F
:1065500079D63D903D923D903D92E00EF76E100E43
:10656000F66E23EE00F011EC66F0DE6A02EC66F0E7
:10657000640EAE6F320EAD6F3DB0C7EF32F03DB27C
:10658000C5EF32F0AD67F8D75DD63D925BD63D9052
:1065900026D65990389223D65992388238A68FD071
:1065A00038961E389A6F030E9A17000E9A630ED013
:1065B0003D903D92E00EF76E340EF66E23EE00F045
:1065C00011EC66F0DE6A02EC66F01ED0010E9A63F2
:1065D0000ED03D903D92E00EF76E400EF66E23EE2B
:1065E00000F011EC66F0DE6A02EC66F00DD03D9032
:1065F0003D92E00EF76E4C0EF66E23EE00F011ECBD
:1066000066F0DE6A02EC66F0640EAE6F320EAD6FBD
:106610003DB014EF33F03DB211EF33F0AD67F8D772
:106620004ED03D923DA84BD03D903D903D92E10E25
:10663000F76E1C0EF66E23EE00F011EC66F0DE6ACB
:1066400002EC66F0640EAE6F320EAD6F3DB030EF0F
:1066500033F03DB22EEF33F0AD67F8D73D922FD037
:106660003D902DD05994BBD55996E50EF76E140E7A
:10667000F66E20EED6F018EC66F0E40EF76ED40E4F
:10668000F66E20EEE6F018EC66F036EC66F01AD006
:106690005998E50EF76E340EF66E20EED6F018EC33
:1066A00066F0E40EF76ED40EF66E20EEE6F018EC0F
:1066B00066F036EC66F006D0599A388200D0000CAD
:1066C0003D92C0D5060EC06FC16BBF8F640EAE6F1A
:1066D000320EAD6FAD67FED7D2EC61F034923490DC
:1066E000EE0C000E186201D01200010E18621200AA
:1066F00080868084808280901200000E186201D013
:106700001200010E186204D08086809480828090EE
:10671000020E18620FD08086808480828090640E82
:10672000AE6F19C0ADF0AD67FED7808680948082D1
:1067300080901200030E186212008096809480925E
:106740008090640EAE6F19C0ADF0AD67FED7808645
:106750008094808280901200A26B3B90E00E3C16E9
:1067600011EE8CF0200EE76201D0120015EE00F061
:106770000A0EA203F350E126F450E22201EE8CF05F
:10678000FF0EE7602FD0080ECB6FE7380F0B300FEE
:10679000806F080ECB6305D03B0E806302D02B0EBA
:1067A000806FE6500F0B300F816F200E9A6F3F0EF7
:1067B00080619AC080F081619AC081F0EE50806360
:1067C00011D0EE5081630ED0CB2FDFD7E7B03C80E5
:1067D000E7B23C82E7B43C84E7B63C86E7B83C8845
:1067E0003B801200A22B400EA263C0D73B90120048
:1067F000A26B3B90F00E3C1611EE9EF0200EE7626D
:1068000001D0120015EE00F00A0EA203F350E126AB
:10681000F450E22201EE9EF0FF0EE76031D0080E48
:10682000CB6FE7380F0B300F806F080ECB6305D0AE
:106830003B0E806302D02B0E806FE6500F0B300FA3
:10684000816F200E9A6F3F0E80619AC080F0816147
:106850009AC081F0EE50806313D0EE50816310D067
:10686000CB2FDFD73B80E7A412003C843B8614EE9D
:10687000C0F0A251E126E86AE222010EE76E1200A2
:10688000A22B400EA263BED73B901200A26B3B909E
:10689000F00E3C1611EE9EF0200EE76201D01200C1
:1068A00015EE00F00A0EA203F350E126F450E222A6
:1068B00001EE9EF0FF0EE76031D0080ECB6FE73897
:1068C0000F0B300F806F080ECB6305D03B0E80633B
:1068D00002D02B0E806FE6500F0B300F816F200E11
:1068E0009A6F3F0E80619AC080F081619AC081F0FA
:1068F000EE50806313D0EE50816310D0CB2FDFD7E2
:10690000E7A612003C863B803B8614EEC0F0A25105
:10691000E126E86AE222010EE76E1200A22B400E89
:10692000A263BED73B9012003990020EAB6FAB67EB
:10693000FED7839C020EAB6FAB67FED783AE398C5C
:1069400083BE399C12003990020EAB6FAB67FED745
:10695000838C020EAB6FAB67FED783AE398E83BEDE
:10696000399E1200C80EAB6FAB67FED7050E12EC56
:1069700062F0640EAB6FAB67FED7D2EC61F0640ED1
:10698000AB6FAB67FED7050E12EC62F0640EAB6F17
:10699000AB67FED7D2EC61F01200C80EAB6FAB67ED
:1069A000FED7050E12EC62F0FA0EAB6FAB67FED7A6
:1069B000D2EC61F0640EAB6FAB67FED7050E12EC44
:1069C00062F0FA0EAB6FAB67FED7D2EC61F012004B
:1069D00038903492E60EF76E640EF66E20EED6F026
:1069E00018EC66F02CEC66F036EC66F051EC5DF0DD
:1069F0009E6B716BB2EC34F001EED2F010EEE6F06B
:106A000081B288EF0FF0A0B107EF35F0F9D71FEC96
:106A100062F0230E9D5D75E09E2B200E9E659DC04D
:106A2000EEFF2A0E9A6F100E9E659AC0E6FF36ECB6
:106A300066F000EF35F001EED2F0300EEE6253D08A
:106A4000300EEE6250D0310EEE624DD0310EEE625D
:106A50004AD0320EEE6247D0320EEE6244D0330E90
:106A6000EE6241D0330EEE623ED001EE00F0300E09
:106A7000EE6EEE6EEE6EEE6E01EE0CF0310EEE6E20
:106A8000320EEE6E330EEE6E340EEE6E350EEE6E90
:106A9000360EEE6E370EEE6E380EEE6E01EE14F020
:106AA000310EEE6E320EEE6E330EEE6E340EEE6E74
:106AB000350EEE6E360EEE6E370EEE6E380EEE6E54
:106AC00001EE04F0340EEE6E320EEE6E330EEE6E0C
:106AD000380EEE6E360EEE6E370EEE6E380EEE6E31
:106AE000330EEE6E22D0E60EF76E740EF66E20EECA
:106AF000D6F018EC66F02CEC66F036EC66F077EF2A
:106B000014F0040E9E630DD001EED2F011EE00F0F1
:106B1000040E976FEE50E662E6D7972F8AEF35F0B6
:106B200010D0080E9E63DFD786D7B2EC34F0716BBD
:106B3000640EAE6F0F0EAD6FAD67FED781B20FEF73
:106B40005CF0000E716313D0E70EF76EE40EF66E84
:106B500020EED6F018EC66F0E70EF76EF40EF66E47
:106B600020EEE6F018EC66F036EC66F05AD0010E36
:106B7000716313D0E80EF76E040EF66E20EED6F0B9
:106B800018EC66F0E80EF76E140EF66E20EEE6F0E6
:106B900018EC66F036EC66F044D0020E716313D048
:106BA000E80EF76E240EF66E20EED6F018EC66F0C6
:106BB000E80EF76E340EF66E20EEE6F018EC66F096
:106BC00036EC66F02ED0030E716313D0E80EF76E2C
:106BD000440EF66E20EED6F018EC66F0E80EF76E76
:106BE000540EF66E20EEE6F018EC66F036EC66F029
:106BF00018D0040E716313D0E80EF76E640EF66EB3
:106C000020EED6F018EC66F0E80EF76E740EF66E15
:106C100020EEE6F018EC66F036EC66F002D0716B10
:106C200090D781B20FEF5CF0A0B118EF36F0F9D732
:106C30001FEC62F0230E9D631BD0000E716302D027
:106C400086EF57F0010E716302D0F7EF49F0020EA4
:106C5000716302D050EF44F0030E716302D0BBEFBA
:106C600039F0040E716302D040EF36F0716B69D7D2
:106C70002A0E9D6366D7712B050E7161716B61D70A
:106C8000B2EC34F0640EAE6F0F0EAD6FAD67FED791
:106C900081B20FEF5CF0FA0EF76E940EF66E20EEF6
:106CA000D6F018EC66F0FA0EF76EA40EF66E20EE33
:106CB000E6F018EC66F036EC66F081B295EF35F050
:106CC000A0B164EF36F0F9D71FEC62F0230E9D639C
:106CD000E9EF38F0FA0EF76ED40EF66E20EED6F02D
:106CE00018EC66F0FA0EF76EE40EF66E20EEE6F0A3
:106CF00018EC66F036EC66F051EC5DF09E6B81B2FC
:106D000042EF36F0A0B1A4EF36F0F9D70F0E9A6F2C
:106D1000100E9E619AC09EF09E5111EED2F09DC061
:106D2000E3FF00EEEEF0070E9A6F9EC097F0080E9C
:106D30009E619AC097F02A0E9A6F97519AC0EBFF06
:106D400036EC66F09E2BDBD71FEC62F0230E9D63C2
:106D5000DDD7080E9E630AD001EE14F011EED2F0DA
:106D6000EE50E66203D09E2FFBD71CD0FA0EF76ED2
:106D7000F40EF66E20EED6F018EC66F0FB0EF76E11
:106D8000040EF66E20EEE6F018EC66F036EC66F0D7
:106D9000CDEC34F0640EAE6F140EAD6FAD67FED760
:106DA00095EF35F0FB0EF76E540EF66E20EED6F032
:106DB00018EC66F02EB409D0FB0EF76E640EF66E7A
:106DC00020EEE6F018EC66F008D0FB0EF76E740EBD
:106DD000F66E20EEE6F018EC66F036EC66F081B266
:106DE00042EF36F0A0B1F6EF36F0F9D71FEC62F0C3
:106DF0002A0E9D6302D02E74D5D7230E9D63EFD744
:106E0000FB0EF76E940EF66E20EED6F018EC66F0E0
:106E10002EB609D0FB0EF76EA40EF66E20EEE6F04D
:106E200018EC66F008D0FB0EF76EB40EF66E20EE8E
:106E3000E6F018EC66F036EC66F081B242EF36F020
:106E4000A0B124EF37F0F9D71FEC62F02A0E9D6352
:106E500002D02E76D5D7230E9D63EFD7FB0EF76EAB
:106E6000C40EF66E20EED6F018EC66F02EB809D0FF
:106E7000FB0EF76ED40EF66E20EEE6F018EC66F020
:106E800008D0FB0EF76EE40EF66E20EEE6F018EC7E
:106E900066F036EC66F081B242EF36F0A0B152EF08
:106EA00037F0F9D71FEC62F02A0E9D6302D02E78DE
:106EB000D5D7230E9D63EFD7FC0EF76E340EF66E1A
:106EC00020EED6F018EC66F0100E976F00EEE6F0AC
:106ED00011EE1CF0E6CFEEFF972FFCD736EC66F0F4
:106EE0009E6B81B2A3EF37F0A0B178EF37F0F9D7FE
:106EF0001FEC62F02A0E9D6306D02CEC66F036EC97
:106F000066F09E6BEED7230E9D630BD0100E976F2D
:106F100010EEE6F001EE1CF0E6CFEEFF972FFCD767
:106F20001ED09E6704D02CEC66F010EEE6F0100E3A
:106F30009E619E690F0E9E179E519DC0E3FF36EC29
:106F400066F09E2BCED7100E976F10EEE6F001EE96
:106F50001CF0E6CFEEFF972FFCD742EF36F0FC0E89
:106F6000F76E440EF66E20EED6F018EC66F02CECC0
:106F700066F0080E976F00EEE6F011EE0CF0E6CF2B
:106F8000EEFF972FFCD736EC66F09E6B81B2EFEFE9
:106F900037F0A0B1CDEF37F0F9D71FEC62F02A0E31
:106FA0009D6308D02CEC66F010EEE6F036EC66F04F
:106FB0009E6BECD7230E9D5D1DE09E6704D02CECEC
:106FC00066F010EEE6F0080E9E619E690F0E9E17A9
:106FD0009E519DC0E3FF9E2B36EC66F0D7D7080E7E
:106FE000976F10EEE6F001EE0CF0E6CFEEFF972F74
:106FF000FCD748D6080E976F10EEE6F001EE0CF0C5
:10700000E6CFEEFF972FFCD7FC0EF76E540EF66E10
:1070100020EED6F018EC66F02CEC66F036EC66F05C
:107020009E6B81B242EF36F0A0B118EF38F0F9D77D
:107030001FEC62F02A0E9D6325D6FC0EF76E640EDF
:10704000F66E20EED6F018EC66F0FC0EF76E740EBD
:10705000F66E20EEE6F018EC66F036EC66F051ECD9
:107060005DF09E6B81B242EF36F0A0B157EF38F081
:10707000F9D70F0E9A6F100E9E619AC09EF09E5126
:1070800011EED2F09DC0E3FF00EEEEF0070E9A6F16
:107090009EC097F0080E9E619AC097F02A0E9A6FD4
:1070A00097519AC0EBFF36EC66F09E2BDBD71FECB6
:1070B00062F0230E9D63DDD7080E9E631BD011EE98
:1070C000D2F0330EE66216D0380EE66213D0370ED9
:1070D000E66210D0360EE6620DD0380EE6620AD0B7
:1070E000330EE66207D0320EE66204D0340EE6625A
:1070F00001D01CD0FC0EF76E840EF66E20EED6F09A
:1071000018EC66F0FC0EF76E940EF66E20EEE6F0CC
:1071100018EC66F036EC66F0CDEC34F0640EAE6F31
:10712000140EAD6FAD67FED795EF35F09E6BFC0E7C
:10713000F76EA40EF66E20EED6F018EC66F0100E88
:10714000976F00EEE6F011EE2EF0E6CFEEFF972FF0
:10715000FCD736EC66F081B2DDEF38F0A0B1B2EFCB
:1071600038F0F9D71FEC62F02A0E9D6306D02CECA4
:1071700066F036EC66F09E6BEED7230E9D630BD067
:10718000100E976F10EEE6F001EE2EF0E6CFEEFF58
:10719000972FFCD777D59E6704D02CEC66F010EEC5
:1071A000E6F0100E9E619E690F0E9E179E519DC0C7
:1071B000E3FF36EC66F09E2BCED7100E976F10EEE5
:1071C000E6F001EE2EF0E6CFEEFF972FFCD742EF70
:1071D00036F0FA0EF76EB40EF66E20EED6F018EC1E
:1071E00066F0FA0EF76EC40EF66E20EEE6F018ECBE
:1071F00066F036EC66F081B242EF36F0A0B102EFF5
:1072000039F0F9D71FEC62F0230E9D6344D5FB0ED5
:10721000F76E140EF66E20EED6F018EC66F02CEC3D
:1072200066F036EC66F051EC5DF09E6B81B242EF99
:1072300036F0A0B132EF39F0F9D70F0E9A6F100E79
:107240009E619AC09EF02A0E9A6F9E5111EED2F066
:1072500000EEE6F09DC0E3FF9AC0EBFF36EC66F06F
:107260009E2BE4D71FEC62F0230E9D63E6D7080E39
:107270009E637CD5080E976F11EE14F001EED2F0EC
:10728000E650EE6273D5972FFBD7FB0EF76E240EF8
:10729000F66E20EED6F018EC66F02CEC66F051ECB1
:1072A0005DF036EC66F09E6B81B242EF36F0A0B135
:1072B0005BEF39F0F9D71FEC62F0230E9D632BD002
:1072C0002F0E11EED2F0E7643BD03A0EE76038D0D3
:1072D000080E976F01EE14F0E6CFEEFF972FFCD764
:1072E000FB0EF76E340EF66E20EED6F018EC66F05C
:1072F000FB0EF76E440EF66E20EEE6F018EC66F02C
:1073000036EC66F0640EAE6F140EAD6FAD67FED74F
:10731000B2EC34F0B7D4070E9A6F080E9E619AC093
:107320009EF02A0E9A6F9E5111EED2F000EEE6F01A
:107330009DC0E3FF9AC0EBFF36EC66F09E2BB4D7FE
:10734000CDEC34F0FB0EF76EF40EF66E20EED6F0B8
:1073500018EC66F0FC0EF76E040EF66E20EEE6F00A
:1073600018EC66F036EC66F0640EAE6F140EAD6F7E
:10737000AD67FED787D4B2EC34F0640EAE6F0F0E5B
:10738000AD6FAD67FED781B20FEF5CF0F20EF76E16
:10739000840EF66E20EED6F018EC66F0F20EF76E64
:1073A000940EF66E20EEE6F018EC66F036EC66F021
:1073B00081B295EF35F0A0B1DFEF39F0F9D71FECCE
:1073C00062F0230E9D6395EF3BF0F20EF76EA40E74
:1073D000F66E20EED6F018EC66F0F20EF76EB40EF4
:1073E000F66E20EEE6F018EC66F056EC3BF080C04E
:1073F000F3F081C0F4F017EC3BF080C0E3F081C003
:10740000E4F036EC66F09E6B640EB06F060EAF6F64
:1074100081B2B2EF3AF0A0B12AEF3AF0AF67F8D7F5
:10742000200EE36FE46F36EC66F0640EB06F020E70
:10743000AF6F81B2B2EF3AF0A0B12AEF3AF0AF6786
:10744000F8D717EC3BF080C0E3F081C0E4F036ECF5
:1074500066F0DAD71FEC62F0230E9D5D25E02A0E60
:107460009D6303D0300E226EC6D7310E9D5D10E0B5
:10747000320E9D5D0DE0330E9D5D0AE0370E9D5D81
:107480000DE0380E9D5D0AE0390E9D5D07E0B3D733
:10749000000E2264B0D7F00E2226ADD7600E226017
:1074A000AAD7100E2226A7D717EC3BF080C0E3F036
:1074B00081C0E4F056EC3BF080C0F3F081C0F4F002
:1074C00036EC66F0640EB06F060EAF6F81B2B2EFAD
:1074D0003AF0A0B188EF3AF0AF67F8D7200EF36F1B
:1074E000F46F36EC66F0640EB06F020EAF6F81B2CF
:1074F000B2EF3AF0A0B188EF3AF0AF67F8D756ECA8
:107500003BF080C0F3F081C0F4F036EC66F0DAD7DF
:107510001FEC62F0230E9D5D25E02A0E9D6303D0D3
:10752000000E236EC7D7310E9D5D10E0320E9D5DBB
:107530000DE0330E9D5D0AE0370E9D5D0DE0380EC7
:107540009D5D0AE0390E9D5D07E0B4D70C0E235C0B
:10755000B1E0040E2326AED7F40E235CABE0FC0EA4
:107560002326A8D756EC3BF080C0F3F081C0F4F09E
:1075700036EC66F0D9EC3AF0640EAE6F320EAD6FB9
:107580003DB0C9EF3AF03DB2C8EF3AF0AD67F8D779
:107590003D92F8EC3AF0640EAE6F320EAD6F3DB036
:1075A000D8EF3AF03DB2D7EF3AF0AD67F8D73D9259
:1075B000E4D603EE00F0410EEE6E540EEE6E2B0E8E
:1075C000EE6E560EEE6E470EEE6E520EEE6E3D0EE7
:1075D000EE6E22C084F07CEC61F07FC0EEFF80C0D4
:1075E000EEFF81C0EEFFEE6A3D6A02EC66F012002B
:1075F00003EE00F0410EEE6E540EEE6E2B0EEE6EAC
:10760000560EEE6E470EEE6E540EEE6E3D0EEE6EA4
:1076100023C084F07CEC61F07FC0EEFF80C0EEFF01
:1076200081C0EEFFEE6A3D6A02EC66F01200100EB9
:10763000226005D02B0E806F360E816F1200200E57
:10764000226005D02B0E806F340E816F1200300E39
:10765000226005D02B0E806F320E816F1200400E1B
:10766000226005D0200E806F300E816F1200500E08
:10767000226005D02D0E806F320E816F1200600ED9
:10768000226005D02D0E806F340E816F1200700EB7
:10769000226005D02D0E806F360E816F1200300EE5
:1076A000226E200E806F300E816F12000C0E23624E
:1076B00005D02B0E806F360E816F1200080E2362EC
:1076C00005D02B0E806F340E816F1200040E2362E2
:1076D00005D02B0E806F320E816F1200000E2362D8
:1076E00005D0200E806F300E816F1200FC0E2362D9
:1076F00005D02D0E806F320E816F1200F80E2362BE
:1077000005D02D0E806F340E816F1200F40E2362AF
:1077100005D02D0E806F360E816F1200000E236E85
:10772000200E806F300E816F1200F20EF76EC40EC5
:10773000F66E20EED6F018EC66F0F20EF76ED40E70
:10774000F66E20EEE6F018EC66F036EC66F081B2EC
:10775000BDEF39F0A0B1AEEF3BF0F9D71FEC62F00E
:10776000230E9D63E9EF3CF0F20EF76EE40EF66E29
:1077700020EED6F018EC66F0F20EF76EF40EF66E10
:1077800020EEE6F018EC66F020C084F07CEC61F0AE
:10779000200EE36FE46F300E806380C0E4F081C0A0
:1077A000E5F021C084F07CEC61F0200EF36FF46F03
:1077B000300E806380C0F4F081C0F5F036EC66F0E6
:1077C000640EB06F060EAF6F81B21CEF3CF0A0B13B
:1077D0000EEF3CF0AF67F8D7200EE36FE46FE56F74
:1077E00036EC66F0640EB06F020EAF6F81B21CEF24
:1077F0003CF0A0B10EEF3CF0AF67F8D720C084F0AA
:107800007CEC61F0200EE36FE46F300E806380C08B
:10781000E4F081C0E5F036EC66F0D2D71FEC62F000
:10782000230E9D6301D018D02A0E9D63ADD7202A68
:107830000F0E2060206AA8D720C084F07CEC61F095
:10784000200EE36FE46F300E806380C0E4F081C0EF
:10785000E5F036EC66F067D020C084F07CEC61F097
:10786000200EE36FE46F300E806380C0E4F081C0CF
:10787000E5F021C084F07CEC61F0200EF36FF46F32
:10788000300E806380C0F4F081C0F5F036EC66F015
:10789000640EB06F060EAF6F81B284EF3CF0A0B102
:1078A00076EF3CF0AF67F8D7200EF36FF46FF56F0B
:1078B00036EC66F0640EB06F020EAF6F81B284EFEB
:1078C0003CF0A0B176EF3CF0AF67F8D721C084F070
:1078D0007CEC61F0200EF36FF46F300E806380C09B
:1078E000F4F081C0F5F036EC66F0D2D71FEC62F010
:1078F000230E9D6301D008D02A0E9D63BAD7212A9A
:107900000F0E2160216AB5D721C084F07CEC61F0B4
:10791000200EF36FF46F300E806380C0F4F081C0EE
:10792000F5F036EC66F003EE00F0410EEE6E540E0C
:10793000EE6E2B0EEE6E570EEE6E560EEE6E520E75
:10794000EE6E3D0EEE6E20C084F07CEC61F07FC0E8
:10795000EEFF80C0EEFF81C0EEFF2C0EEE6E21C068
:1079600084F07CEC61F07FC0EEFF80C0EEFF81C050
:10797000EEFFEE6A3D6A02EC66F0640EAE6F320E08
:10798000AD6F3DB0E6EF3CF03DB2C9EF3CF0AD6706
:10799000F8D73D92F30EF76E040EF66E20EED6F099
:1079A00018EC66F0F30EF76E140EF66E20EEE6F0AD
:1079B00018EC66F036EC66F0640EAE6F320EAD6F0A
:1079C000AD67FED7050E206E216ACED63D90348875
:1079D000D4D4F30EF76E240EF66E20EED6F018EC2B
:1079E00066F0F30EF76E340EF66E20EEE6F018EC4D
:1079F00066F036EC66F081B2BDEF39F0A0B102EF6F
:107A00003DF0F9D71FEC62F0230E9D63EAEF3DF0E5
:107A1000F30EF76E440EF66E20EED6F018EC66F01C
:107A200093EC3DF036EC66F0640EB06F060EAF6F6F
:107A300081B244EF3DF0A0B137EF3DF0AF67F8D72A
:107A4000F30EF76EC40EF66E20EEE6F018EC66F05C
:107A500036EC66F0640EB06F020EAF6F81B244EF89
:107A60003DF0A0B137EF3DF0AF67F8D7D9D71FECA5
:107A700062F02A0E9D6305D01F2A070E1F601F6A41
:107A8000CFD7230E9D63D0D793EC3DF036EC66F054
:107A900003EE00F0410EEE6E540EEE6E2B0EEE6E07
:107AA000570EEE6E4D0EEE6E420EEE6E530EEE6EF5
:107AB0003D0EEE6E1FC084F07CEC61F07FC0EEFFE7
:107AC00080C0EEFF81C0EEFFEE6A3D6A02EC66F018
:107AD000640EAE6F320EAD6F3DB090EF3DF03DB233
:107AE00074EF3DF0AD67F8D73D92F30EF76ED40E0C
:107AF000F66E20EED6F018EC66F0F30EF76EE40E9C
:107B0000F66E20EEE6F018EC66F036EC66F0640EE9
:107B1000AE6F320EAD6FAD67FED7050E1F6E78D714
:107B20003D9034882AD4000E1F6209D0F30EF76E00
:107B3000540EF66E20EEE6F018EC66F01200010E20
:107B40001F6209D0F30EF76E640EF66E20EEE6F0BB
:107B500018EC66F01200020E1F6209D0F30EF76EE9
:107B6000740EF66E20EEE6F018EC66F01200030ECE
:107B70001F6209D0F30EF76E840EF66E20EEE6F06B
:107B800018EC66F01200040E1F6209D0F30EF76EB7
:107B9000940EF66E20EEE6F018EC66F01200050E7C
:107BA0001F6209D0F30EF76EA40EF66E20EEE6F01B
:107BB00018EC66F01200060E1F6209D0F30EF76E85
:107BC000B40EF66E20EEE6F018EC66F01200050E2C
:107BD0001F6EA9D7F30EF76EF40EF66E20EED6F0F8
:107BE00018EC66F0F40EF76E040EF66E20EEE6F07A
:107BF00018EC66F036EC66F081B2BDEF39F0A0B15A
:107C000003EF3EF0F9D71FEC62F0230E9D6348EFBF
:107C10003EF0B2EC34F0F40EF76E140EF66E20EE79
:107C2000D6F018EC66F02CEC66F036EC66F001EE5F
:107C3000D2F010EEE6F09E6B81B2BBEF39F0A0B14E
:107C400023EF3EF0F9D71FEC62F0230E9D6312D0B4
:107C5000040E9E6373EF35F001EED2F011EE00F0EA
:107C6000EECFE6FFEECFE6FFEECFE6FFEECFE6FF8C
:107C7000BDEF39F09E2B200E9E659DC0EEFF2A0EB3
:107C80009A6F100E9E659AC0E6FF36EC66F0D4D768
:107C9000F40EF76E240EF66E20EED6F018EC66F0B9
:107CA000F40EF76E340EF66E20EEE6F018EC66F089
:107CB00036EC66F081B2BDEF39F0A0B161EF3EF075
:107CC000F9D71FEC62F0230E9D6319EF3FF0B2EC81
:107CD00034F0F80EF76E740EF66E20EED6F018EC57
:107CE00066F0F80EF76E840EF66E20EEE6F018ECF5
:107CF00066F03998310E39B8320EE56F9E6B080E7A
:107D0000976F00EEEEF011EE40F039B811EE48F04A
:107D1000E6CFEEFF972FFCD736EC66F0640EB06F1F
:107D2000060EAF6F81B217EF3FF0A0B1C3EF3EF088
:107D3000AF67F8D710EEEEF0200EE66EE66EE66E58
:107D4000E66EE66EE66EE66EE66E36EC66F0640EA5
:107D5000B06F020EAF6F81B217EF3FF0A0B1C3EF6B
:107D60003EF0AF67F8D7080E976F00EEEEF011EE19
:107D700040F039B811EE48F0E6CFEEFF972FFCD770
:107D800036EC66F0CBD71FEC62F0230E9D5D44E02D
:107D90002A0E9D630DD0080E976F11EE40F039B892
:107DA00011EE48F0200EE66E972FFCD79E6BA7D7FA
:107DB0009E670BD0080E976F11EE40F039B811EEA8
:107DC00048F0200EE66E972FFCD7080E9E610AD071
:107DD00011EE40F039B811EE48F09E519DC0E3FF1E
:107DE0009E2B8DD7F80EF76E940EF66E20EEE6F011
:107DF00018EC66F036EC66F081B217EF3FF0A0B1F8
:107E000003EF3FF0F9D7F80EF76E840EF66E20EE12
:107E1000E6F018EC66F0BFD730A202D0BDEF39F023
:107E20003978310E39B8320EE56F9E6B68D7BDEFE9
:107E300039F0F40EF76E640EF66E20EED6F018EC04
:107E400066F0F40EF76E740EF66E20EEE6F018ECA7
:107E500066F036EC66F081B2BDEF39F0A0B132EFDA
:107E60003FF0F9D71FEC62F0230E9D63AFEF3FF0B8
:107E7000B2EC34F0E30EF76EA40EF66E20EED6F000
:107E800018EC66F02CEC66F036EC66F051EC5DF028
:107E90009E6B01EED2F010EEE6F081B2BDEF39F04C
:107EA000A0B154EF3FF0F9D71FEC62F0230E9D5DB7
:107EB0000EE09E2B200E9E659DC0EEFF2A0E9A6F4F
:107EC000100E9E659AC0E6FF36EC66F0E6D701EE2E
:107ED000D2F0330EEE6235D0380EEE6232D0370E6D
:107EE000EE622FD0360EEE622CD0380EEE6229D024
:107EF000330EEE6226D0320EEE6223D0340EEE62E6
:107F000020D0E30EF76EC40EF66E20EED6F018EC1D
:107F100066F0E30EF76ED40EF66E20EEE6F018EC87
:107F200066F036EC66F0FF0ED16FD26F00EED1F046
:107F3000020ECB6F030EAA6EFE0EA96EE9EC65F081
:107F4000FF00E60EF76E740EF66E20EED6F018EC1B
:107F500066F02CEC66F036EC66F077EF14F0F40E79
:107F6000F76E840EF66E20EED6F018EC66F0F40E86
:107F7000F76E940EF66E20EEE6F018EC66F036EC36
:107F800066F081B2BDEF39F0A0B1C8EF3FF0F9D78C
:107F90001FEC62F0230E9D63DEEF43F0F40EF76EEC
:107FA000C40EF66E20EED6F018EC66F02CEC66F0FF
:107FB0003F963D903D92E00EF76EBA0EF66E23EEC0
:107FC00000F011EC66F0DE6A02EC66F0640EAE6F53
:107FD000320EAD6F3DB009EF40F0AD67FBD7F40E48
:107FE000F76ED40EF66E20EED6F018EC66F0F40EB6
:107FF000F76EE40EF66E20EEE6F018EC66F036EC66
:1080000066F0640EAE6F140EAD6FAD67FED795EFE0
:1080100035F0100E976F18EE12F000EEE6F0E6CF96
:10802000EEFF972FFCD736EC66F081B2BDEF39F04A
:10803000A0B11CEF40F0F9D71FEC62F02A0E9D634F
:1080400002D008EF41F0F50EF76E740EF66E20EEDA
:10805000D6F018EC66F0F50EF76E840EF66E20EE94
:10806000E6F018EC66F036EC66F09E6B81B2BDEF80
:1080700039F0A0B15BEF40F0F9D70F0E9A6F100EF8
:108080009E619AC09EF09E5111EED2F09DC0E3FF1A
:1080900000EEEEF0070E9A6F9EC097F0080E9E61FC
:1080A0009AC097F02A0E9A6F97519AC0EBFF36EC60
:1080B00066F09E2BDBD71FEC62F0230E9D63DDD7AD
:1080C000080E9E6389D001EE04F011EED2F0EE505E
:1080D000E66282D09E2FFBD7F50EF76E940EF66EF9
:1080E00020EED6F018EC66F0F50EF76EA40EF66EE4
:1080F00020EEE6F018EC66F036EC66F051EC5DF040
:1081000036EC66F09E6B81B2BDEF39F0A0B18AEF1C
:1081100040F0F9D71FEC62F0230E9D632CD02F0E98
:1081200011EED2F0E7643CD03A0EE76039D0080E89
:10813000976F01EE04F0E6CFEEFF972FFCD7F50E18
:10814000F76EB40EF66E20EED6F018EC66F0F50E73
:10815000F76EC40EF66E20EEE6F018EC66F036EC24
:1081600066F0640EAE6F140EAD6FAD67FED7B2EC65
:1081700034F0BDEF39F0070E9A6F080E9E619AC079
:108180009EF02A0E9A6F9E5111EED2F000EEEEF0A4
:108190009DC0E3FF9AC0EBFF36EC66F09E2BB3D791
:1081A000CDEC34F0F50EF76EF40EF66E20EED6F050
:1081B00018EC66F0F60EF76E040EF66E20EEE6F0A2
:1081C00018EC66F036EC66F0640EAE6F140EAD6F10
:1081D000AD67FED7BDEF39F0F50EF76ED40EF66E33
:1081E00020EED6F018EC66F0F50EF76EE40EF66EA3
:1081F00020EEE6F018EC66F036EC66F0CDEC34F0EC
:10820000640EAE6F140EAD6FAD67FED795EF35F00F
:10821000F40EF76EF40EF66E20EED6F018EC66F063
:10822000F50EF76E040EF66E20EEE6F018EC66F032
:1082300036EC66F051EC5DF09E6B81B2BDEF39F02B
:10824000A0B142EF41F0F9D70F0E9A6F100E9E6168
:108250009AC09EF09E5111EED2F09DC0E3FF00EE59
:10826000EEF0070E9A6F9EC097F0080E9E619AC0BE
:1082700097F02A0E9A6F97519AC0EBFF36EC66F092
:108280009E2BDBD71FEC62F0230E9D63DDD7080E1B
:108290009E630AD001EE04F011EED2F0EE50E662D9
:1082A00003D09E2FFBD71CD0F50EF76ED40EF66EC2
:1082B00020EED6F018EC66F0F50EF76EE40EF66ED2
:1082C00020EEE6F018EC66F036EC66F0CDEC34F01B
:1082D000640EAE6F140EAD6FAD67FED795EF35F03F
:1082E000F50EF76E140EF66E20EED6F018EC66F072
:1082F0002CEC66F036EC66F051EC5DF09E6B81B2D2
:10830000BDEF39F0A0B199EF41F0F9D70F0E9A6F98
:10831000100E9E619AC09EF09E5111EED2F09DC04B
:10832000E3FF00EEE6F09DC0EBFF36EC66F09E2B1F
:10833000E6D71FEC62F02A0E9D6301D0D9D7230E39
:108340009D63E4D70F0E9E6301D003D00E0E9E6393
:1083500040D03D903D92E00EF76EB00EF66E23EEEB
:1083600000F011EC66F0DE6A02EC66F0640EAE6FAF
:10837000640EAD6F3DB0FDEF41F03DB2C5EF41F091
:108380003FB8FFEF41F0AD67F5D73D92F40EF76EC1
:10839000A40EF66E20EED6F018EC66F0F40EF76E32
:1083A000B40EF66E20EEE6F018EC66F036EC66F0F1
:1083B000A66BA76B76EC63F0A68776EC63F0020EF3
:1083C000C06FC16BBF8F81A2E3EF41F0D2EC61F0CF
:1083D000FF00F50EF76E240EF66E20EED6F018ECC8
:1083E00066F0F50EF76E340EF66E20EEE6F018EC41
:1083F00066F036EC66F077EF14F03D90BBD73F980F
:108400003D9E640EAE6F640EAD6F3DBE03D0AD6792
:10841000FCD7BCD73D9E150EC963F7D7F50EF76E96
:10842000440EF66E20EED6F018EC66F036EC66F0F0
:10843000870EF76E160EF66E100E986F82EC43F0F4
:10844000100E986F78EC43F0870EF76E260EF66EDE
:10845000100E986F82EC43F0100E986F78EC43F09A
:10846000870EF76E360EF66E100E986F82EC43F0A4
:10847000100E986F78EC43F0870EF76E460EF66E8E
:10848000100E986F82EC43F0100E986F78EC43F06A
:10849000870EF76E560EF66E100E986F82EC43F054
:1084A000100E986F78EC43F0030E976F870EF76EFF
:1084B000660EF66E100E986F82EC43F0100E986FF9
:1084C00078EC43F0972FF2D7870EF76E760EF66EA4
:1084D000100E986F82EC43F0100E986F78EC43F01A
:1084E000870EF76E860EF66E100E986F82EC43F0D4
:1084F000100E986F78EC43F0870EF76E960EF66EBE
:10850000100E986F82EC43F0100E986F78EC43F0E9
:10851000350E976F870EF76EA60EF66E100E986FDB
:1085200082EC43F0100E986F78EC43F0972FF2D75F
:10853000870EF76EB60EF66E040E986F82EC43F05F
:10854000040E986F78EC43F0640EAE6F050EAD6FBD
:10855000AD67FED7870EF76EBA0EF66E010E986FF6
:1085600082EC43F0010E986F78EC43F0640EAE6F2E
:108570000A0EAD6FAD67FED78280576A640EAE6F8C
:10858000050EAD6FAD67FED78290640EAE6F140E10
:10859000AD6FAD67FED73D903D92E00EF76EE00EF9
:1085A000F66E23EE00F011EC66F0DE6A02EC66F087
:1085B000640EAE6F640EAD6F57B6E8EF42F057B081
:1085C000E8EF42F03DB003D0AD67F6D7DFD63D907F
:1085D0003D903D92E00EF76E580EF66E23EE00F0E1
:1085E00011EC66F0DE6A02EC66F0640EAE6F140EFB
:1085F000AD6F3DB002EF43F03DB2C6EF41F0AD6765
:10860000F8D7C4D63D903D92E00EF76E740EF66E2C
:1086100023EE00F011EC66F0DE6A02EC66F0640E08
:10862000AE6F320EAD6F3DB01DEF43F03DB21BEFAC
:1086300043F0AD67F8D73D92A9D6640EAE6F140E25
:10864000AD6FAD67FED703EE00F0410EEE6E540E37
:10865000EE6E2B0EEE6E570EEE6E490EEE6E4D0E5A
:10866000EE6E450EEE6E490EEE6E3D0EEE6E100E87
:10867000976F11EED2F0200EE76404D0E6CFEEFF44
:10868000972FF9D70D0EEE6EEE6A02EC66F0640ECF
:10869000AE6F640EAD6F3DB253EF43F03DB055EF9A
:1086A00043F0AD67F8D73D9271D6F50EF76E540ED4
:1086B000F66E20EED6F018EC66F0F50EF76E640E4E
:1086C000F66E20EEE6F018EC66F036EC66F0A66B7F
:1086D000A76B76EC63F0A68776EC63F0020EC06FB2
:1086E000C16BBF8F81A272EF43F0D2EC61F0FF004B
:1086F00003EE00F0EECFADFF00009EA8FED7982F4E
:10870000F9D71200F86A03EE00F00900F5CFEEFF8A
:10871000982FFBD712000201FE454550524F4D20C5
:1087200020202032382F30312F30302031323A3073
:1087300038002056657273696F6E2076316130366D
:1087400020202020202020433A5C544D505C746D42
:10875000705C3430305F6D3131622E35345C6F7552
:1087600074002020202020202020202020202020D5
:10877000202020202020207E81F7EB180000009090
:108780008258AD2A010200CDAB12000100005E014B
:108790000900BAD34D75FE4A6F92F11A1A1A1A1AC5
:1087A0001A1A1A1A1A1A1A1A1A1A1A1A1A1A1A1A29
:1087B0001A1A1A1A1A1A1A1A1A910400F60EF76ED1
:1087C000140EF66E20EED6F018EC66F0F60EF76E8C
:1087D000240EF66E20EEE6F018EC66F036EC66F04D
:1087E00081B2BDEF39F0A0B1F7EF43F0F9D71FEC3C
:1087F00062F0230E9D63BDEF39F0F60EF76E340E76
:10880000F66E20EED6F018EC66F030C081F030B095
:1088100009D0F60EF76E440EF66E20EEE6F018EC78
:1088200066F008D0F60EF76E540EF66E20EEE6F007
:1088300018EC66F036EC66F0640EAE6F060EAD6FA7
:1088400081B2BDEF39F0A0B13FEF44F0AD67F8D78A
:10885000F60EF76E640EF66E20EEE6F018EC66F09B
:1088600036EC66F0640EAE6F020EAD6F81B2BDEFF6
:1088700039F0A0B13FEF44F0AD67F8D7C8D71FEC8F
:1088800062F02A0E9D6302D03070C1D7230E9D6323
:10889000BED781A1BDEF39F030A03488BDEF39F0EB
:1088A000640EAE6F0F0EAD6FAD67FED781B20FEFE6
:1088B0005CF0EF0EF76E940EF66E20EED6F018EC2C
:1088C00066F0EF0EF76EA40EF66E20EEE6F018ECF2
:1088D00066F036EC66F081B295EF35F0A0B172EF3C
:1088E00044F0F9D71FEC62F0230E9D6311EF45F0C1
:1088F000EF0EF76EB40EF66E20EED6F018EC66F0C2
:10890000C5EC49F036EC66F0640EAE6F060EAD6F46
:1089100081B250EF44F0A0B1A7EF44F0AD67F8D7B3
:10892000EF0EF76EF40EF66E20EEE6F018EC66F041
:1089300036EC66F0640EAE6F020EAD6F81B250EF92
:1089400044F0A0B1A7EF44F0AD67F8D7D9D71FEC3A
:1089500062F02A0E9D630CD00CC081F0FC0E0C1648
:10896000030E8117812B8161816B81510C12C8D755
:10897000230E9D63C5D7F00EF76E040EF66E20EE43
:10898000D6F018EC66F00CB409D0F00EF76E240E99
:10899000F66E20EEE6F018EC66F008D0F00EF76EFA
:1089A000140EF66E20EEE6F018EC66F036EC66F08B
:1089B00081B250EF44F0A0B1DFEF44F0F9D71FECE3
:1089C00062F0230E9D5D02E00C74D5D7F00EF76EB9
:1089D000340EF66E20EED6F018EC66F00CB609D028
:1089E000F00EF76E540EF66E20EEE6F018EC66F020
:1089F00008D0F00EF76E440EF66E20EEE6F018EC9E
:108A000066F036EC66F081B250EF44F0A0B10AEFA8
:108A100045F0F9D71FEC62F0230E9D5D02E00C7665
:108A2000D5D7F00EF76E640EF66E20EED6F018EC89
:108A300066F0F00EF76E740EF66E20EEE6F018ECAF
:108A400066F036EC66F081B250EF44F0A0B12AEF48
:108A500045F0F9D71FEC62F0230E9D63F3EF45F06C
:108A6000F00EF76E840EF66E20EED6F018EC66F07F
:108A7000F00EF76E940EF66E20EEE6F018EC66F04F
:108A800036EC66F0640EB06F060EAF6F81B250EF39
:108A900044F0A0B165EF45F0AF67F8D7200EF56F51
:108AA00036EC66F0640EB06F020EAF6F81B250EF1D
:108AB00044F0A0B165EF45F0AF67F8D70E500F0B4B
:108AC000300FF56F36EC66F0DDD71FEC62F02A0E42
:108AD0009D6304D00E6A300EF56FD4D7230E9D63CC
:108AE00001D008D00F0E9D150E6E9DC0F5F036EC2E
:108AF00066F0C8D7F00EF76EA40EF66E20EED6F034
:108B000018EC66F02CEC66F001EE50F011EED2F0AD
:108B1000100E8B6FEECFE6FF8B2FFCD79E6B01EE16
:108B2000D2F010EEE6F0100E8B6FEECFE6FF8B2F3B
:108B3000FCD736EC66F081B2E7EF45F0A0B1A2EFCA
:108B400045F0F9D71FEC62F02A0E9D630AD0100E93
:108B50008B6F01EED2F0200EEE6E8B2FFCD79E6B4A
:108B6000DED7230E9D6301D027D09E6708D0100E5C
:108B70008B6F01EED2F0200EEE6E8B2FFCD7100E15
:108B80009E6115D0010E9E630BD0300E9D6308D000
:108B9000300E01EED2F0EF6203D09E6B2B0E9D6F74
:108BA0009E5111EED2F09DC0E3FF9E2BB8D7CDECC5
:108BB00034F0100E9E6FB3D7100E8B6F01EED2F013
:108BC00011EE50F0EECFE6FF8B2FFCD70CD0100E3D
:108BD0008B6F01EED2F011EE50F0EECFE6FF8B2F4F
:108BE000FCD750EF44F0F00EF76EB40EF66E20EEA8
:108BF000D6F018EC66F0F00EF76EC40EF66E20EEAE
:108C0000E6F018EC66F036EC66F081B250EF44F016
:108C1000A0B10CEF46F0F9D71FEC62F0230E9D6374
:108C2000B0EF48F0F00EF76ED40EF66E20EED6F0F0
:108C300018EC66F0F00EF76EE40EF66E20EEE6F03D
:108C400018EC66F09E6B10C084F07CEC61F080C084
:108C5000F4F081C0F5F036EC66F0640EB06F060EED
:108C6000AF6F81B250EF44F0A0B151EF46F0AF6763
:108C7000F8D7200EF46FF56F36EC66F0640EB06F27
:108C8000020EAF6F81B250EF44F0A0B151EF46F049
:108C9000AF67F8D780C0F4F081C0F5F036EC66F02D
:108CA000DCD71FEC62F02A0E9D6304D0010E106E1B
:108CB0009E6BC9D7230E9D5D25E09E6708D0200ED0
:108CC000F46FF56F300E7F6F806F816F9E6B030EB8
:108CD0009E6112D080C07FF081C080F09DC081F085
:108CE00032EC61F0000E846507D0210E846104D05F
:108CF00084C010F09E2BA7D7CDEC34F0010E106E7F
:108D00009E6BA1D7F00EF76EF40EF66E20EED6F045
:108D100018EC66F0F10EF76E040EF66E20EEE6F03B
:108D200018EC66F09E6B11C084F07CEC61F080C0A2
:108D3000F4F081C0F5F036EC66F0640EB06F060E0C
:108D4000AF6F81B250EF44F0A0B1C1EF46F0AF6712
:108D5000F8D7200EF46FF56F36EC66F0640EB06F46
:108D6000020EAF6F81B250EF44F0A0B1C1EF46F0F8
:108D7000AF67F8D780C0F4F081C0F5F036EC66F04C
:108D8000DCD71FEC62F02A0E9D6304D0010E116E39
:108D90009E6BC9D7230E9D5D25E09E6708D0200EEF
:108DA000F46FF56F300E7F6F806F816F9E6B030ED7
:108DB0009E6112D080C07FF081C080F09DC081F0A4
:108DC00032EC61F0000E846507D0210E846104D07E
:108DD00084C011F09E2BA7D7CDEC34F0010E116E9C
:108DE0009E6BA1D7F10EF76E140EF66E20EED6F044
:108DF00018EC66F0F10EF76E240EF66E20EEE6F03B
:108E000018EC66F012C084F07CEC61F080C0E8F0F1
:108E10002E0EE96F81C0EAF036EC66F0640EB06F9A
:108E2000060EAF6F81B250EF44F0A0B135EF47F0BE
:108E3000AF67F8D7200EE86FE96FEA6F36EC66F09F
:108E4000640EB06F020EAF6F81B250EF44F0A0B16C
:108E500035EF47F0AF67F8D780C0E8F02E0EE96F26
:108E600081C0EAF036EC66F0D9D71FEC62F0230E31
:108E70009D5D13E02A0E9D6303D0050E126EC2D7CE
:108E800012C084F0050E8427370E846103D084C09D
:108E900012F0B8D70A0E126EB5D7F10EF76E340E77
:108EA000F66E20EED6F018EC66F0F10EF76E440E7A
:108EB000F66E20EEE6F018EC66F013C084F07CEC61
:108EC00061F07FC0F4F080C0F5F036EC66F0640E1F
:108ED000B06F060EAF6F81B250EF44F0A0B18BEFD0
:108EE00047F0AF67F8D7200EF46FF56F36EC66F0F9
:108EF000640EB06F020EAF6F81B250EF44F0A0B1BC
:108F00008BEF47F0AF67F8D77FC0F4F080C0F5F083
:108F100036EC66F0DCD71FEC62F0230E9D5D16E0A8
:108F20002A0E9D6303D00A0E136EC7D713C084F0B8
:108F30000A0E8427FB0E846106D0090E846503D0D7
:108F400084C013F0BAD70A0E136EB7D7F10EF76EBE
:108F5000540EF66E20EED6F018EC66F00CBE09D07A
:108F6000F10EF76E640EF66E20EEE6F018EC66F089
:108F700008D0F10EF76E740EF66E20EEE6F018ECE7
:108F800066F036EC66F081B250EF44F0A0B1CAEF63
:108F900047F0F9D71FEC62F02A0E9D6302D00C7ED9
:108FA000D5D7230E9D63EFD7F10EF76E840EF66EC4
:108FB00020EED6F018EC66F0F10EF76E940EF66E19
:108FC00020EEE6F018EC66F09E6B080E976F11EE3F
:108FD00070F000EEEEF0E6CFEEFF972FFCD736EC08
:108FE00066F081B220EF48F0A0B1F8EF47F0F9D772
:108FF0001FEC62F02A0E9D6325D0080E976F01EEDC
:1090000070F0200EEE6E972FFCD79E6BDED79E671A
:1090100008D0080E976F01EE70F0200EEE6E972FBD
:10902000FCD79E2B090E9E6106D09E5111EE6FF06B
:109030009DC0E3FFCAD7CDEC34F0080E9E6FC5D7B4
:1090400050EF44F0230E9D63E2D7F10EF76EA40EAD
:10905000F66E20EED6F018EC66F0F10EF76EB40E58
:10906000F66E20EEE6F018EC66F09E6B040E976F3D
:1090700011EE78F000EEF2F0E6CFEEFF972FFCD77E
:1090800036EC66F081B271EF48F0A0B149EF48F0DC
:10909000F9D71FEC62F02A0E9D6325D0040E976F5E
:1090A00001EE78F0200EEE6E972FFCD79E6BDED788
:1090B0009E6708D0040E976F01EE78F0200EEE6EDA
:1090C000972FFCD79E2B050E9E6106D09E5111EE68
:1090D00077F09DC0E3FFCAD7CDEC34F0040E9E6F4D
:1090E000C5D750EF44F0230E9D63E2D7F10EF76E23
:1090F000C40EF66E20EED6F018EC66F0F10EF76EA8
:10910000D40EF66E20EEE6F018EC66F09E6B0F5073
:10911000300FF56F36EC66F081B2A9EF48F0A0B1E0
:1091200093EF48F0F9D71FEC62F02A0E9D6313D03D
:109130000F6A9E6BECD79E2B020E9E6105D09D514F
:10914000F56F0F0B0F6EE3D7CDEC34F09E6B0F6A0B
:10915000DED750EF44F0230E9D63EDD750EF44F07F
:10916000F10EF76EE40EF66E20EED6F018EC66F017
:10917000F10EF76EF40EF66E20EEE6F018EC66F0E7
:1091800036EC66F081B250EF44F0A0B1C9EF48F080
:10919000F9D71FEC62F0230E9D6350EF44F09E6BF5
:1091A000F20EF76E040EF66E20EED6F018EC66F0B6
:1091B000F20EF76E140EF66E20EEE6F018EC66F086
:1091C000000E146207D0320E7F6F350E806F300EA6
:1091D000816F20D0010E146207D0330E7F6F370EDF
:1091E000806F350E816F16D0020E146207D0340ED8
:1091F0007F6F300E806F300E816F0CD0030E1462C3
:1092000007D0350E7F6F300E806F300E816F02D029
:10921000146AD6D77FC0EEF080C0EFF081C0F0F0C6
:1092200036EC66F0640EB06F060EAF6F81B250EF91
:1092300044F0A0B139EF49F0AF67F8D7200EEE6FD8
:10924000EF6FF06F36EC66F0640EB06F020EAF6F2A
:1092500081B250EF44F0A0B139EF49F0AF67F8D7D1
:109260007FC0EEF080C0EFF081C0F0F036EC66F029
:10927000D9D71FEC62F02A0E9D6308D0142A040E81
:109280001460146AB1EC63F08E6F9AD7230E9D635D
:1092900097D79E6BF20EF76E240EF66E20EED6F088
:1092A00018EC66F0F20EF76E340EF66E20EEE6F075
:1092B00018EC66F0000E156207D0320E7F6F350E87
:1092C000806F300E816F20D0010E156207D0330EF3
:1092D0007F6F370E806F350E816F16D0020E1562CC
:1092E00007D0340E7F6F300E806F300E816F0CD040
:1092F000030E156207D0350E7F6F300E806F300E73
:10930000816F02D0156AD6D77FC0EEF080C0EFF033
:1093100081C0F0F036EC66F0640EB06F060EAF6FF1
:1093200081B250EF44F0A0B1B3EF49F0AF67F8D786
:10933000200EEE6FEF6FF06F36EC66F0640EB06FDC
:10934000020EAF6F81B250EF44F0A0B1B3EF49F01D
:10935000AF67F8D77FC0EEF080C0EFF081C0F0F0CB
:1093600036EC66F0D9D71FEC62F02A0E9D6308D068
:10937000152A040E1560156AC0EC63F08F6F9AD73A
:10938000230E9D6397D750EF44F00C50030B816F71
:10939000000E816309D0EF0EF76EC40EF66E20EE5C
:1093A000E6F018EC66F01200010E816309D0EF0EB2
:1093B000F76ED40EF66E20EEE6F018EC66F01200B2
:1093C000020E816309D0EF0EF76EE40EF66E20EE0A
:1093D000E6F018EC66F01200FC0E0C16EF0EF76EBD
:1093E000C40EF66E20EEE6F018EC66F01200640E85
:1093F000AE6F0F0EAD6FAD67FED781B20FEF5CF0B1
:10940000EA0EF76E040EF66E20EED6F018EC66F05B
:10941000EA0EF76E140EF66E20EEE6F018EC66F02B
:1094200036EC66F081B295EF35F0A0B119EF4AF055
:10943000F9D71FEC62F0230E9D637EEF4AF0EA0E2F
:10944000F76E240EF66E20EED6F018EC66F016B627
:1094500009D0EA0EF76E440EF66E20EEE6F018EC38
:1094600066F008D0EA0EF76E340EF66E20EEE6F0E7
:1094700018EC66F036EC66F0640EB06F060EAF6F57
:1094800081B2F7EF49F0A0B174EF4AF0AF67F8D7B7
:10949000EA0EF76E540EF66E20EEE6F018EC66F06B
:1094A00036EC66F0640EB06F020EAF6F81B2F7EF6C
:1094B00049F0A0B174EF4AF0AF67F8D716B609D0FB
:1094C000EA0EF76E440EF66E20EEE6F018EC66F04B
:1094D00008D0EA0EF76E340EF66E20EEE6F018ECC9
:1094E00066F036EC66F0C8D71FEC62F02A0E9D637A
:1094F00002D01676ACD7230E9D63BED7EA0EF76E68
:10950000640EF66E20EED6F018EC66F0EA0EF76EFA
:10951000740EF66E20EEE6F018EC66F036EC66F0AF
:1095200081B2F7EF49F0A0B197EF4AF0F9D71FECFD
:1095300062F0230E9D634AEF4BF0EA0EF76E740E55
:10954000F66E20EED6F018EC66F048EC57F036ECEC
:1095500066F0640EAE6F060EAD6F81B2F7EF49F0A4
:10956000A0B1CCEF4AF0AD67F8D7EA0EF76EC40EA3
:10957000F66E20EEE6F018EC66F036EC66F0640E5F
:10958000AE6F020EAD6F81B2F7EF49F0A0B1CCEF34
:109590004AF0AD67F8D7D9D71FEC62F02A0E9D6369
:1095A00007D0FC0E1E16812B030E81151E12CDD77F
:1095B000230E9D63CAD748EC57F036EC66F0EA0EEE
:1095C000F76ED40EF66E20EED6F018EC66F02CECAA
:1095D00066F001EE60F011EED2F0100E8B6FEECF60
:1095E000E6FF8B2FFCD79E6B01EED2F010EEE6F07B
:1095F000100E8B6FEECFE6FF8B2FFCD736EC66F0AC
:1096000081B23EEF4BF0A0B107EF4BF0F9D71FEC62
:1096100062F02A0E9D630AD0100E8B6F01EED2F01D
:10962000200EEE6E8B2FFCD79E6BDED7230E9D6334
:1096300001D019D09E6708D0100E8B6F01EED2F0CA
:10964000200EEE6E8B2FFCD79E2B110E9E6106D046
:109650009E5111EED1F09DC0E3FFC6D7CDEC34F0A2
:10966000100E9E6FC1D7100E8B6F01EED2F011EE6F
:1096700060F0EECFE6FF8B2FFCD70CD0100E8B6F77
:1096800001EED2F011EE60F0EECFE6FF8B2FFCD7AB
:10969000F7EF49F0EA0EF76EE40EF66E20EED6F024
:1096A00018EC66F0EA0EF76EF40EF66E20EEE6F0B9
:1096B00018EC66F036EC66F081B2F7EF49F0A0B135
:1096C00063EF4BF0F9D71FEC62F0230E9D6397EF29
:1096D0004BF0EB0EF76E040EF66E20EED6F018ECA3
:1096E00066F01EAC09D0EB0EF76E140EF66E20EE8F
:1096F000E6F018EC66F008D0EB0EF76E240EF66E6E
:1097000020EEE6F018EC66F036EC66F081B2F7EF8A
:1097100049F0A0B18DEF4BF0F9D71FEC62F02A0EA3
:109720009D6302D01E7CD5D7230E9D63DAD7EB0E46
:10973000F76E340EF66E20EED6F018EC66F0EB0EF7
:10974000F76E440EF66E20EEE6F018EC66F036EC9E
:1097500066F081B2F7EF49F0A0B1B0EF4BF0F9D766
:109760001FEC62F0230E9D6374EF4CF0EB0EF76E6E
:10977000940EF66E20EED6F018EC66F01EB609D008
:10978000EB0EF76EA40EF66E20EEE6F018EC66F027
:1097900008D0EB0EF76EB40EF66E20EEE6F018EC85
:1097A00066F036EC66F0640EB06F060EAF6F81B2F5
:1097B000F7EF49F0A0B10BEF4CF0AF67F8D7EB0E25
:1097C000F76EC40EF66E20EEE6F018EC66F036EC9E
:1097D00066F0640EB06F020EAF6F81B2F7EF49F022
:1097E000A0B10BEF4CF0AF67F8D71EB609D0EB0E67
:1097F000F76EA40EF66E20EEE6F018EC66F008D0D8
:10980000EB0EF76EB40EF66E20EEE6F018EC66F096
:1098100036EC66F0C8D71FEC62F02A0E9D6302D0CA
:109820001E76ACD7230E9D63A9D7EB0EF76ED40E30
:10983000F66E20EED6F018EC66F02EB009D0EB0EE6
:10984000F76EE40EF66E20EEE6F018EC66F008D047
:10985000EB0EF76EF40EF66E20EEE6F018EC66F006
:1098600036EC66F0640EB06F060EAF6F81B2F7EFA4
:1098700049F0A0B16AEF4CF0AF67F8D7EC0EF76E85
:10988000040EF66E20EEE6F018EC66F036EC66F0AC
:10989000640EB06F020EAF6F81B2F7EF49F0A0B166
:1098A0006AEF4CF0AF67F8D72EB009D0EB0EF76E29
:1098B000E40EF66E20EEE6F018EC66F008D0EB0E43
:1098C000F76EF40EF66E20EEE6F018EC66F036EC6D
:1098D00066F0C8D71FEC62F02A0E9D6302D02E708E
:1098E000ACD7230E9D63A9D7EC0EF76E140EF66E5F
:1098F00020EED6F018EC66F0EC0EF76E240EF66E45
:1099000020EEE6F018EC66F036EC66F081B2F7EF88
:1099100049F0A0B18DEF4CF0F9D71FEC62F0230EA7
:109920009D63F4EF4CF0EC0EF76E340EF66E20EE05
:10993000D6F018EC66F01EB409D0EC0EF76E640E8B
:10994000F66E20EEE6F018EC66F008D0EC0EF76E3E
:10995000540EF66E20EEE6F018EC66F036EC66F08B
:10996000640EB06F060EAF6F81B2F2EF4CF0A0B193
:10997000E8EF4CF0AF67F8D7EC0EF76E440EF66EDA
:1099800020EEE6F018EC66F036EC66F0640EB06F90
:10999000020EAF6F81B2F2EF4CF0A0B1E8EF4CF0E5
:1099A000AF67F8D71EB409D0EC0EF76E640EF66EF2
:1099B00020EEE6F018EC66F008D0EC0EF76E540ED0
:1099C000F66E20EEE6F018EC66F036EC66F0C8D7DE
:1099D0001FEC62F0230E9D5D26E02A0E9D63C0D72A
:1099E0001E74A9D7F7EF49F0EC0EF76E740EF66E01
:1099F00020EED6F018EC66F0EC0EF76E840EF66EE4
:109A000020EEE6F018EC66F036EC66F081B2F7EF87
:109A100049F0A0B10DEF4DF0F9D71FEC62F0230E25
:109A20009D63FDEF4FF0EC0EF76E940EF66E20EE98
:109A3000D6F018EC66F0EC0EF76EA40EF66E20EE83
:109A4000E6F018EC66F036EC66F081B2F7EF49F01C
:109A5000A0B12CEF4DF0F9D71FEC62F0230E9D5D05
:109A600005E02A0E9D63F1D7CFEF4FF0A26B51ECCA
:109A70005DF0EC0EF76EB40EF66E20EEE6F018EC2C
:109A800066F015EE00F001EED2F00A0EA203F350DC
:109A9000E126F450E222FF0EE76205D0780EE8CF0F
:109AA000D2F13C6A22D0080ECB6F200E806FE738CF
:109AB0000F0B300F816F3F0E816180C081F03B0E34
:109AC000816302D02B0E816F81C0EEFFE6500F0B39
:109AD0009A6F300F816F3F0E816180C081F081C02D
:109AE000EEFFCB2FE4D7E6CF3CF0100ECB6F11EE9C
:109AF000D2F000EED6F0E6CFEEFFCB2FFCD74E0E25
:109B00003CB0590EF16F4E0E3CB2590EF26F4E0E34
:109B10003CB4590EF36F4E0E3CB6590EF46F4E0E18
:109B20003CB8590EF56F826BA2C083F0832B98EC82
:109B300061F080C0E7F081C0E8F036EC66F081B2F9
:109B4000A1EF4FF0A0B1A6EF4DF0F9D71FEC62F0F6
:109B5000230E9D5D1EE02A0E9D5D20E0370E9D5D6B
:109B600018E0380E9D5D15E0390E9D5D12E0310E56
:109B70009D5D07E0320E9D5D04E0330E9D5D01E0CA
:109B8000DED7A2073F0ECB6F400EA261CBC0A2F082
:109B90006ED7A22B400EA261A26B69D79E6B640E9A
:109BA000B06F060EAF6F81B2A1EF4FF0A0B1FEEF24
:109BB0004DF0AF67F8D710EED6F0100ECB6F200E39
:109BC000E66ECB2FFDD736EC66F0640EB06F020E5A
:109BD000AF6F81B2A1EF4FF0A0B1FEEF4DF0AF67D4
:109BE000F8D711EED2F000EED6F0100ECB6FE6CF24
:109BF000EEFFCB2FFCD736EC66F0D1D71FEC62F02E
:109C0000230E9D5DD8B450D02A0E9D6312D051EC26
:109C10005DF0780EE8CFD2F1100ECB6F11EED2F0DE
:109C200000EED6F0E6CFEEFFCB2FFCD736EC66F099
:109C3000B5D79E6702D051EC5DF00F0E9E6120D02B
:109C4000010E9E630AD0300E9D6307D011EED2F054
:109C5000E76203D09E6B2B0E9D6F11EED2F09E51EA
:109C60009DC0E3FF00EED6F011EED2F0100ECB6FE8
:109C7000E6CFEEFFCB2FFCD736EC66F09E2B8FD7CE
:109C8000CDEC34F051EC5DF0780EE8CFD2F100EE7F
:109C9000D6F011EED2F0100ECB6FE6CFEEFFCB2F49
:109CA000FCD736EC66F07AD711EED2F000EED6F0A3
:109CB000100ECB6FE6CFEEFFCB2FFCD736EC66F065
:109CC000640EB06F060EAF6F81B2A1EF4FF0A0B17E
:109CD00083EF4EF0AF67F8D7200EF16F36EC66F0E9
:109CE000640EB06F020EAF6F81B2A1EF4FF0A0B162
:109CF00083EF4EF0AF67F8D74E0E3CB0590EF16FC0
:109D000036EC66F0DDD71FEC62F02A0E9D6308D0BA
:109D10003C704E0E3CB0590EF16F36EC66F0D0D769
:109D2000230E9D63CDD74E0E3CB0590EF16F640EDD
:109D3000B06F060EAF6F81B2A1EF4FF0A0B1BAEFD6
:109D40004EF0AF67F8D7200EF26F36EC66F0640E77
:109D5000B06F020EAF6F81B2A1EF4FF0A0B1BAEFBA
:109D60004EF0AF67F8D74E0E3CB2590EF26F36EC9C
:109D700066F0DDD71FEC62F02A0E9D6308D03C72BE
:109D80004E0E3CB2590EF26F36EC66F0D0D7230E71
:109D90009D63CDD74E0E3CB2590EF26F640EB06F7C
:109DA000060EAF6F81B2A1EF4FF0A0B1F1EF4EF010
:109DB000AF67F8D7200EF36F36EC66F0640EB06F25
:109DC000020EAF6F81B2A1EF4FF0A0B1F1EF4EF0F4
:109DD000AF67F8D74E0E3CB4590EF36F36EC66F011
:109DE000DDD71FEC62F02A0E9D6308D03C744E0E46
:109DF0003CB4590EF36F36EC66F0D0D7230E9D635A
:109E0000CDD74E0E3CB4590EF36F640EB06F060EF4
:109E1000AF6F81B2A1EF4FF0A0B128EF4FF0AF6765
:109E2000F8D7200EF46F36EC66F0640EB06F020EB9
:109E3000AF6F81B2A1EF4FF0A0B128EF4FF0AF6745
:109E4000F8D74E0E3CB6590EF46F36EC66F0DDD7FF
:109E50001FEC62F02A0E9D6308D03C764E0E3CB695
:109E6000590EF46F36EC66F0D0D7230E9D63CDD734
:109E70004E0E3CB6590EF46F640EB06F060EAF6F07
:109E800081B2A1EF4FF0A0B15FEF4FF0AF67F8D70D
:109E9000200EF56F36EC66F0640EB06F020EAF6FF9
:109EA00081B2A1EF4FF0A0B15FEF4FF0AF67F8D7ED
:109EB0004E0E3CB8590EF56F36EC66F0DDD71FEC50
:109EC00062F02A0E9D6308D03C784E0E3CB8590EC5
:109ED000F56F36EC66F0D0D7230E9D63CDD74E0ECE
:109EE0003CB8590EF56F05EE00F011EED2F00A0EF7
:109EF000A203F350E926F450EA22780EE7620BD071
:109F0000FF0EEE6EEE6EEE6EEE6EEE6EEE6EEE6EC0
:109F1000EE6EEE6A3ED6080ECB6F11EED2F0200E3A
:109F2000E764E768E638F00B816F200EE764E768C6
:109F30000F0EE6148111EE6ECB2FF1D73CC0EEFF71
:109F400028D605EE00F011EED2F00A0EA203F3506F
:109F5000E926F450EA22780EE7620CD0FF0EEE6E8E
:109F6000EE6EEE6EEE6EEE6EEE6EEE6EEE6EEE6A15
:109F7000F7EF49F0080ECB6F200EE764E768E6388C
:109F8000F00B816F200EE764E7680F0EE614811175
:109F9000EE6ECB2FF1D73CC0EEFFF7EF49F0A26B8E
:109FA00015EE00F00A0EA203F350E126F450E2226F
:109FB000FF0EE75CD8B437EF4DF0A22B3F0EA26541
:109FC000EFD7EC0EF76EC40EF66E20EED6F018EC5E
:109FD00066F0EC0EF76ED40EF66E20EEE6F018EC9E
:109FE00066F036EC66F0CDEC34F0640EAE6F140E15
:109FF000AD6FAD67FED736EF4DF0EC0EF76EE40EA9
:10A00000F66E20EED6F018EC66F0EC0EF76EF40E5D
:10A01000F66E20EEE6F018EC66F036EC66F081B2F3
:10A02000F7EF49F0A0B116EF50F0F9D71FEC62F04E
:10A03000230E9D6366EF50F0ED0EF76E040EF66E84
:10A0400020EED6F018EC66F024BC09D0ED0EF76EC9
:10A05000140EF66E20EEE6F018EC66F008D0ED0E69
:10A06000F76E240EF66E20EEE6F018EC66F036EC95
:10A0700066F0640EAE6F060EAD6F81B200EF4AF06F
:10A08000A0B15CEF50F0AD67F8D7ED0EF76E340E6F
:10A09000F66E20EEE6F018EC66F036EC66F0640E34
:10A0A000AE6F020EAD6F81B200EF4AF0A0B15CEF6F
:10A0B00050F0AD67F8D7C8D71FEC62F02A0E9D6349
:10A0C00002D0247CC1D7230E9D63D3D7ED0EF76E4B
:10A0D000440EF66E20EED6F018EC66F0ED0EF76E3C
:10A0E000540EF66E20EEE6F018EC66F036EC66F0F4
:10A0F00081B2F7EF49F0A0B17FEF50F0F9D71FEC34
:10A1000062F0230E9D63C2D0ED0EF76E640EF66E04
:10A1100020EED6F018EC66F01E389A6F030E9A17F0
:10A12000000E9A630AD09A6BED0EF76E740EF66EFF
:10A1300020EEE6F018EC66F017D0010E9A6309D015
:10A14000ED0EF76E840EF66E20EEE6F018EC66F07B
:10A150000BD0020E9A63E7D7ED0EF76E940EF66EF3
:10A1600020EEE6F018EC66F036EC66F0640EB06FA8
:10A17000060EAF6F81B200EF4AF0A0B1D3EF50F0FE
:10A18000AF67F8D72CEC66F036EC66F0640EB06F73
:10A19000020EAF6F81B200EF4AF0A0B1D3EF50F0E2
:10A1A000AF67F8D7B9D71FEC62F02A0E9D630AD0CB
:10A1B0009A2B030E9A619A6BCF0E1E169A391E12B5
:10A1C0003886AAD7230E9D63D1D7ED0EF76EA40E65
:10A1D000F66E20EED6F018EC66F01EAE09D0ED0E4D
:10A1E000F76EB40EF66E20EEE6F018EC66F008D0CE
:10A1F000ED0EF76EC40EF66E20EEE6F018EC66F08B
:10A2000036EC66F0640EB06F060EAF6F81B2F7EFFA
:10A2100049F0A0B13AEF51F0AF67F8D7ED0EF76E05
:10A22000D40EF66E20EEE6F018EC66F036EC66F032
:10A23000640EB06F020EAF6F81B2F7EF49F0A0B1BC
:10A240003AEF51F0AF67F8D71EAE09D0ED0EF76EBA
:10A25000B40EF66E20EEE6F018EC66F008D0ED0EC7
:10A26000F76EC40EF66E20EEE6F018EC66F036ECF3
:10A2700066F0C8D71FEC62F02A0E9D6302D01E7EE6
:10A28000ACD7230E9D63BED700EF4AF0ED0EF76EFC
:10A29000E40EF66E20EED6F018EC66F0ED0EF76EDA
:10A2A000F40EF66E20EEE6F018EC66F036EC66F092
:10A2B00081B2F7EF49F0A0B15FEF51F0F9D71FEC91
:10A2C00062F0230E9D6300EF4AF0EE0EF76E040E6F
:10A2D000F66E20EED6F018EC66F02438816F030E8F
:10A2E000811781670CD0CF0E2416816BEE0EF76EAE
:10A2F000140EF66E20EEE6F018EC66F017D0010EA4
:10A30000816309D0EE0EF76E240EF66E20EEE6F0B5
:10A3100018EC66F00BD0020E8163E5D7EE0EF76EF7
:10A32000540EF66E20EEE6F018EC66F036EC66F0B1
:10A3300081B2F7EF49F0A0B19FEF51F0F9D71FECD0
:10A3400062F02A0E9D630AD06487812B030E81611F
:10A35000816BCF0E241681392412BFD7230E9D6343
:10A36000E7D7000E815DD8B425D2010E815DD8B447
:10A3700089D0020E81631ED2EE0EF76E640EF66E69
:10A3800020EED6F018EC66F0EE0EF76E740EF66E58
:10A3900020EEE6F018EC66F09E6B9AC9F0F09BC9CF
:10A3A000F1F09CC9F2F09DC9F3F09EC9F4F09FC989
:10A3B000F5F036EC66F0640EB06F060EAF6F81B24A
:10A3C000F7EF49F0A0B10BEF52F0AF67F8D7200ECE
:10A3D000F06FF16FF26FF36FF46FF56F36EC66F0BC
:10A3E000640EB06F020EAF6F81B2F7EF49F0A0B10B
:10A3F0000BEF52F0AF67F8D79AC9F0F09BC9F1F0B4
:10A400009CC9F2F09DC9F3F09EC9F4F09FC9F5F024
:10A4100036EC66F0D0D71FEC62F02A0E9D6310D0A8
:10A420009E6B200EE8CF9AF9E8CF9BF9E8CF9CF914
:10A43000E8CF9DF9E8CF9EF9E8CF9FF96487ADD7C3
:10A44000230E9D5DD8B4B8D19E670DD0200EE8CF05
:10A450009AF9E8CF9BF9E8CF9CF9E8CF9DF9E8CFCE
:10A460009EF9E8CF9FF9060E9E6108D009EE9AF09A
:10A470009E519DC0EBFF9E2B64878FD7CDEC34F0AF
:10A480009E6B8BD7EE0EF76E340EF66E20EED6F086
:10A4900018EC66F0EE0EF76E440EF66E20EEE6F067
:10A4A00018EC66F09E6BA26B310EA225D66F19EEEA
:10A4B000A2F0080EA203F350E126F450E222E6CF08
:10A4C000E0F0E6CFE1F0E6CFE2F0E6CFE3F0E6CF72
:10A4D000E4F0E6CFE5F0E6CF83F0E6CF82F098EC4B
:10A4E00061F07DC0F1F07EC0F2F07FC0F3F080C07B
:10A4F000F4F081C0F5F036EC66F081B2F7EF49F088
:10A50000A0B184EF52F0F9D71FEC62F02A0E9D63E0
:10A5100005D0A22B040EA2614FD1C6D7230E9D6396
:10A52000ECD79E6BA26B310EA225D66F19EEA2F06E
:10A53000080EA203F350E126F450E222E6CFE0F049
:10A54000E6CFE1F0E6CFE2F0E6CFE3F0E6CFE4F0ED
:10A55000E6CFE5F0E6CF83F0E6CF82F098EC61F04D
:10A560007DC0F1F07EC0F2F07FC0F3F080C0F4F067
:10A5700081C0F5F036EC66F0640EB06F060EAF6F7A
:10A5800081B2F7EF49F0A0B1F4EF52F0AF67F8D71E
:10A59000200EE06FE16FE26FE36FE46FE56F36EC82
:10A5A00066F0640EB06F020EAF6F81B2F7EF49F044
:10A5B000A0B1F4EF52F0AF67F8D719EEA2F0080E91
:10A5C000A203F350E126F450E222E6CFE0F0E6CF1A
:10A5D000E1F0E6CFE2F0E6CFE3F0E6CFE4F0E6CF5D
:10A5E000E5F036EC66F0C8D71FEC62F02A0E9D63EA
:10A5F00011D09E6B19EEA2F0080EA203F350E126D3
:10A60000F450E222200EE66EE66EE66EE66EE66E30
:10A61000E66E89D7230E9D5D25E09E670FD019EE6B
:10A62000A2F0080EA203F350E126F450E222200E1D
:10A63000E66EE66EE66EE66EE66EE66E060E9E610F
:10A640000DD019EEA2F0080EA203F350E126F4504B
:10A65000E2229E519DC0E3FF9E2B65D7CDEC34F0E6
:10A660009E6B61D719EEA2F0080EA203F350E1260B
:10A67000F450E222E6CFE0F0E6CFE1F0E6CFE2F000
:10A68000E6CFE3F0E6CFE4F0E6CFE5F036EC66F0B7
:10A6900019EEA8F0080EA203F350E126F450E222CE
:10A6A000E6CF83F0E5CF82F098EC61F07DC0F1F069
:10A6B0007EC0F2F07FC0F3F080C0F4F081C0F5F00E
:10A6C00036EC66F09E6B640EB06F060EAF6F81B213
:10A6D000F7EF49F0A0B196EF53F0AF67F8D7200E2F
:10A6E000F16FF26FF36FF46FF56F36EC66F0640E96
:10A6F000B06F020EAF6F81B2F7EF49F0A0B196EFE5
:10A7000053F0AF67F8D7E6CF83F0E5CF82F098EC4F
:10A7100061F07DC0F1F07EC0F2F07FC0F3F080C048
:10A72000F4F081C0F5F036EC66F0CDD71FEC62F0A6
:10A730002A0E9D6303D0E66AE56AAAD7230E9D5DC3
:10A74000D8B432D09E6708D0E66AE56A300E7D6FD5
:10A750007E6F7F6F806F816F7EC07DF07FC07EF0E7
:10A7600080C07FF081C080F09DC081F07DC075F019
:10A770007EC076F07FC077F080C078F081C079F03D
:10A7800041EC61F083C0E6FF82C0E5FF9E2B7DC0F7
:10A79000F1F07EC0F2F07FC0F3F080C0F4F081C031
:10A7A000F5F036EC66F08FD7A22B040EA26104D030
:10A7B0009E6BB9D6CF0E2416EE0EF76E940EF66E83
:10A7C00020EED6F018EC66F0EE0EF76EA40EF66EE4
:10A7D00020EEE6F018EC66F09E6B28C0F0F029C081
:10A7E000F1F02AC0F2F02BC0F3F02CC0F4F02DC031
:10A7F000F5F036EC66F0640EB06F060EAF6F81B206
:10A80000F7EF49F0A0B12BEF54F0AF67F8D7200E67
:10A81000F06FF16FF26FF36FF46FF56F36EC66F077
:10A82000640EB06F020EAF6F81B2F7EF49F0A0B1C6
:10A830002BEF54F0AF67F8D728C0F0F029C0F1F043
:10A840002AC0F2F02BC0F3F02CC0F4F02DC0F5F0CC
:10A8500036EC66F0D0D71FEC62F02A0E9D630AD06A
:10A860009E6B300E286E200E296E2A6E2B6E2C6E7B
:10A870002D6EB3D7230E9D5D1DE09E670DD0200E7B
:10A88000E8CF28F0E8CF29F0E8CF2AF0E8CF2BF086
:10A89000E8CF2CF0E8CF2DF0060E9E6107D010EE29
:10A8A00028F09E519DC0E3FF9E2B97D7CDEC34F04E
:10A8B0009E6B93D7200E286202D0300E286EEE0ECB
:10A8C000F76E840EF66E20EED6F018EC66F024C01B
:10A8D00081F0030E8117000E81630BD0FC0E24164D
:10A8E000EE0EF76EB40EF66E20EEE6F018EC66F0A3
:10A8F00017D0010E816309D0EE0EF76EC40EF66E0E
:10A9000020EEE6F018EC66F00BD0020E8163E6D77D
:10A91000EE0EF76EE40EF66E20EEE6F018EC66F042
:10A9200036EC66F081B29EEF54F0A0B199EF54F08E
:10A93000F9D71FEC62F0230E9D6305D024C081F08F
:10A94000030E81170CD02A0E9D63ECD7812B030ECA
:10A950008161816BFC0E241681512412B8D7000E40
:10A9600081631FD03D903D92E00EF76ED40EF66EDF
:10A9700023EE00F011EC66F0DE6A02EC66F0640E85
:10A98000AE6F640EAD6F3DB0CEEF54F03DB2CBEF85
:10A9900054F0AD67F8D73D9293EF08F03D9000EF8B
:10A9A0004AF0010E816323D1EE0EF76ED40EF66EDF
:10A9B00020EEE6F018EC66F026C083F027C082F0A7
:10A9C00098EC61F07DC0EAF07EC0EBF07FC0ECF067
:10A9D00080C0EDF081C0EEF025C084F07CEC61F029
:10A9E0007FC0F3F080C0F4F081C0F5F036EC66F083
:10A9F0009E6B640EB06F060EAF6F81B2F7EF49F039
:10AA0000A0B12CEF55F0AF67F8D7200EEA6FEB6FCF
:10AA1000EC6FED6FEE6F36EC66F0640EB06F020E09
:10AA2000AF6F81B2F7EF49F0A0B12CEF55F0AF67EF
:10AA3000F8D726C083F027C082F098EC61F07DC083
:10AA4000EAF07EC0EBF07FC0ECF080C0EDF081C09A
:10AA5000EEF036EC66F0CDD71FEC62F02A0E9D6367
:10AA600003D0266A276AA8D7230E9D6306D02766DF
:10AA700039D0090E266433D035D09E6708D0266AB7
:10AA8000276A300E7D6F7E6F7F6F806F816F7EC013
:10AA90007DF07FC07EF080C07FF081C080F09DC0DF
:10AAA00081F07DC075F07EC076F07FC077F080C009
:10AAB00078F081C079F041EC61F083C026F082C06B
:10AAC00027F09E2B7DC0EAF07EC0EBF07FC0ECF05B
:10AAD00080C0EDF081C0EEF036EC66F08AD7CDECA8
:10AAE00034F06AD726C083F027C082F098EC61F07A
:10AAF0007DC0EAF07EC0EBF07FC0ECF080C0EDF0EE
:10AB000081C0EEF025C084F07CEC61F07FC0F3F0F2
:10AB100080C0F4F081C0F5F036EC66F09E6B640EF8
:10AB2000B06F060EAF6F81B2F7EF49F0A0B1BAEF88
:10AB300055F0AF67F8D7200EF36FF46FF56F36EC72
:10AB400066F0640EB06F020EAF6F81B246EF51F047
:10AB5000A0B1BAEF55F0AF67F8D725C084F07CEC10
:10AB600061F07FC0F3F080C0F4F081C0F5F036EC06
:10AB700066F0D5D71FEC62F02A0E9D6302D0256ADD
:10AB8000C1D7230E9D6307D0090E25641FD0700E18
:10AB900025601CD01ED09E6705D0256A300E7F6FC1
:10ABA000806F816F80C07FF081C080F09DC081F098
:10ABB00032EC61F084C025F09E2B7FC0F3F080C0A2
:10ABC000F4F081C0F5F036EC66F0A9D7CDEC34F0A6
:10ABD00099D725C084F07CEC61F07FC0F3F080C091
:10ABE000F4F081C0F5F036EC66F000EF4AF06493C3
:10ABF00061EC5DF03D903D92E00EF76EC60EF66E94
:10AC000023EE00F011EC66F0DE6A02EC66F0640EF2
:10AC1000AE6F640EAD6F3DB030EF56F03DB213EF46
:10AC200056F0AD67F8D73D92EE0EF76EF40EF66E65
:10AC300020EED6F018EC66F0EF0EF76E040EF66E0E
:10AC400020EEE6F018EC66F036EC66F0CDEC34F071
:10AC5000640EAE6F140EAD6FAD67FED700EF4AF015
:10AC6000EF0EF76E140EF66E20EED6F018EC66F0CE
:10AC7000EF0EF76E240EF66E20EEE6F018EC66F09E
:10AC8000070E976FCB6B19EE00F0300ECB25D66F09
:10AC9000160ECB03F350E126F450E226E6CFE8F09F
:10ACA000E6CFE9F0E6CFEAF0E6CFEBF0E6CFECF066
:10ACB000E6CFEDF0E6CFDBF0E6CFDCF0E6CFDDF07F
:10ACC000E6CFDEF0E650E650E650E650E6CFF2F092
:10ACD000E6CFF3F0E6CFF4F0E6CFF5F0E6CFE3F021
:10ACE000E6CFE3F0E6CFE4F0E6CFE5F036EC66F051
:10ACF00081B27FEF56F0A0B181EF56F0F9D700EFA7
:10AD00004AF01FEC62F02A0E9D6304D0CB2B972FE4
:10AD1000BAD7B6D7230E9D636AD719EE00F0160E88
:10AD2000CB03F350E126F450E226200EE76220D058
:10AD3000EF0EF76E340EF66E20EED6F018EC66F0DD
:10AD4000EF0EF76E440EF66E20EEE6F018EC66F0AD
:10AD500036EC66F081B2B4EF56F0A0B1B4EF56F025
:10AD6000F9D7FC0E2416FED5FC0E241646EF51F042
:10AD7000EF0EF76E540EF66E20EED6F018EC66F07D
:10AD8000EF0EF76E640EF66E20EEE6F018EC66F04D
:10AD900036EC66F019EE0EF0160ECB03F350E126FA
:10ADA000F450E22603EE00F0410EEE6E540EEE6E0D
:10ADB0002B0EEE6E430EEE6EEE6E450EEE6E4C0EEC
:10ADC000EE6EEE6E3D0EEE6EE6CFEEFFE6CFEEFFE0
:10ADD000E6CFEEFFE6CFEEFFEE6A5A6A649302EC2E
:10ADE00066F0640EAE6FC80EAD6F5AB02AEF57F022
:10ADF0005AB209EF57F05AB409EF57F05AB609EFB3
:10AE000057F05AB82AEF57F05ABA09EF57F0AD6722
:10AE1000ECD7CDEC34F05A6AEF0EF76E340EF66EC6
:10AE200020EED6F018EC66F0EF0EF76E440EF66EDC
:10AE300020EEE6F018EC66F036EC66F081B225EF15
:10AE400057F0A0B125EF57F0F9D71FEC62F0FC0ED8
:10AE5000241688D56483EF0EF76E740EF66E20EE1E
:10AE6000D6F018EC66F0EF0EF76E840EF66E20EE5C
:10AE7000E6F018EC66F036EC66F081B246EF51F081
:10AE8000A0B144EF57F0F9D71FEC62F046EF51F054
:10AE90001E50030B816F000E816309D0EA0EF76E1E
:10AEA000840EF66E20EEE6F018EC66F01200010E4D
:10AEB000816309D0EA0EF76E940EF66E20EEE6F08E
:10AEC00018EC66F01200020E816309D0EA0EF76EEC
:10AED000A40EF66E20EEE6F018EC66F01200030EFB
:10AEE000816309D0EA0EF76EB40EF66E20EEE6F03E
:10AEF00018EC66F01200FC0E1E16EA0EF76E840EB9
:10AF0000F66E20EEE6F018EC66F01200640EAE6FFE
:10AF10000F0EAD6FAD67FED781B20FEF5CF0E80E9C
:10AF2000F76E840EF66E20EED6F018EC66F0E80EA2
:10AF3000F76E940EF66E20EEE6F018EC66F036EC46
:10AF400066F081B295EF35F0A0B1A8EF57F0F9D7D0
:10AF50001FEC62F0230E9D639BEF59F0E90EF76E34
:10AF6000640EF66E20EED6F018EC66F0E90EF76E81
:10AF7000740EF66E20EEE6F018EC66F08B6B9E6BAE
:10AF8000826B8BC083F0832B98EC61F0200ED76F1F
:10AF900080C0D8F081C0D9F004EE40F0040E8B03DD
:10AFA000F350E926E86AEA22EF380F0B7A6FEE5089
:10AFB0000F0B7B6FEF380F0B7C6FEE500F0B7D6F1D
:10AFC000EF380F0B7E6FEE500F0B7F6FEF380F0BCC
:10AFD000806FEE500F0B816F45EC59F036EC66F048
:10AFE00081B21BEF59F0A0B1F7EF57F0F9D71FEC82
:10AFF00062F0230E9D6305D08B2B200E8B618B6B33
:10B00000BED72A0E9D5D20E0370E9D5D18E0380EFC
:10B010009D5D15E0390E9D5D12E0310E9D5D07E0EE
:10B02000320E9D5D04E0330E9D5D01E0D9D78B07A4
:10B030001F0ECB6F200E8B61CBC08BF0A0D78B2B5C
:10B04000200E8B618B6B9BD79E6B640EB06F060ED0
:10B05000AF6F81B270EF58F0A0B14EEF58F0AF670C
:10B06000F8D7200EE56F36EC66F0640EB06F020E76
:10B07000AF6F81B270EF58F0A0B14EEF58F0AF67EC
:10B08000F8D7480E9A6F0F0E816381C09AF09AC06C
:10B09000E5F0300EE52736EC66F0D7D71FEC62F00E
:10B0A0002A0E9D6307D00F0E816F780EE56F36EC88
:10B0B00066F0CAD7230E9D5D13E0300E9D650DD05E
:10B0C000330E9D610AD00F0E9D15816F81C0E5F092
:10B0D000300EE52736EC66F0B7D7CDEC34F0E3D789
:10B0E000480E9A6F0F0E816381C09AF09AC0E5F006
:10B0F000300EE52736EC66F09E6B640EB06F060EE0
:10B10000AF6F81B21BEF59F0A0B1A4EF58F0AF6759
:10B11000F8D7200EEF6FF06FF16FF26FF36FF46FEF
:10B12000F56F36EC66F0640EB06F020EAF6F81B251
:10B130001BEF59F0A0B1A4EF58F0AF67F8D745EC7A
:10B1400059F036EC66F0D9D71FEC62F0230E9D5D06
:10B150004AE02A0E9D5D0FE19E530DE00F0E7A6FBF
:10B160007B6F7C6F7D6F7E6F7F6F806F45EC59F0DA
:10B1700036EC66F0C1D79E5308E10F0E7A6F7B6FF5
:10B180007C6F7D6F7E6F7F6F806F070E9E611CD01E
:10B19000010E9E6309D0300E9D6306D0000E7A63C7
:10B1A00003D09E6B0B0E9D6F0F0E9D1710EE7AF065
:10B1B0009E51E126E86AE2229DC0E3FF45EC59F08A
:10B1C0009E2B36EC66F099D7CDEC34F00F0E7A6FEB
:10B1D0007B6F7C6F7D6F7E6F7F6F806F45EC59F06A
:10B1E00036EC66F089D714EE40F0040E8B03F35072
:10B1F000E126E86AE222200E7A6307D0FF0EE66EAF
:10B20000E66EE66EF00EE66EF7D60F0E7A177B1737
:10B210007C177D177E177F17801781177A397B116E
:10B22000E66E7C397D11E66E7E397F11E66E8039DF
:10B230008111E66EE1D614EE40F0040E8B03F3505C
:10B24000E126E86AE222780E7A6308D0FF0EE66E05
:10B25000E66EE66EF00EE66E86EF57F00F0E7A178A
:10B260007B177C177D177E177F17801781177A3918
:10B270007B11E66E7C397D11E66E7E397F11E66EBC
:10B2800080398111E66E86EF57F0480E9A6F0F0EE7
:10B29000816381C09AF09AC0E5F00A0E7A6303D008
:10B2A000FA0E9A6F0CD00B0E7A6303D0FB0E9A6FD6
:10B2B00006D0480E9A6F0F0E7A637AC09AF09AC041
:10B2C000EFF0F00E9A6F0F0E7B637BC09AF09AC07E
:10B2D000F0F0F00E9A6F0F0E7C637CC09AF09AC06B
:10B2E000F1F0F00E9A6F0F0E7D637DC09AF09AC058
:10B2F000F2F0F00E9A6F0F0E7E637EC09AF09AC045
:10B30000F3F0F00E9A6F0F0E7F637FC09AF09AC031
:10B31000F4F0F00E9A6F0F0E806380C09AF09AC01E
:10B32000F5F0300EE527EF27F027F127F227F32776
:10B33000F427F5271200E80EF76EA40EF66E20EE45
:10B34000D6F018EC66F0E80EF76EB40EF66E20EE4E
:10B35000E6F018EC66F036EC66F081B286EF57F056
:10B36000A0B1B4EF59F0F9D71FEC62F0230E9D6342
:10B3700024EF5AF0640EAE6FFA0EAD6FE90EF76E61
:10B38000840EF66E20EED6F018EC66F0E90EF76E3D
:10B39000940EF66E20EEE6F018EC66F017C084F01E
:10B3A0007CEC61F010EEE8F080C0E6FF2E0EE66E59
:10B3B00081C0E6FF36EC66F0640EB06F060EAF6F2C
:10B3C00081B222EF5AF0A0B107EF5AF0AF67F8D779
:10B3D00010EEE8F0200EE66EE66EE66E36EC66F0F5
:10B3E000640EB06F020EAF6F81B222EF5AF0A0B1BF
:10B3F00007EF5AF0AF67F8D710EEE8F080C0E6FF2D
:10B400002E0EE66E81C0E6FF36EC66F0D5D71FEC57
:10B4100062F0230E9D5D16E02A0E9D6305D0050E99
:10B42000846F84C017F0BAD717C084F0050E842744
:10B43000370E846103D084C017F0B0D7320EE8CF46
:10B4400017F0ACD786EF57F0E80EF76EC40EF66E25
:10B4500020EED6F018EC66F0E80EF76ED40EF66E1D
:10B4600020EEE6F018EC66F036EC66F081B286EF7E
:10B4700057F0A0B13DEF5AF0F9D71FEC62F0230E60
:10B480009D63E8EF5AF0CAEC5AF0B6EC5AF036EC8D
:10B4900066F0640EB06F060EAF6F81B2B4EF5AF073
:10B4A000A0B16CEF5AF0AF67F8D7200EE36FE46FEE
:10B4B000E56F36EC66F0640EB06F020EAF6F81B2CE
:10B4C000B4EF5AF0A0B16CEF5AF0AF67F8D7B6EC12
:10B4D0005AF036EC66F0DDD71FEC62F02A0E9D6361
:10B4E00002D01674D2D7230E9D63D3D7B6EC5AF090
:10B4F000640EB06F060EAF6F81B2B4EF5AF0A0B118
:10B500009FEF5AF0AF67F8D7E90EF76E340EF66E7C
:10B5100020EEE6F018EC66F036EC66F0640EB06FE4
:10B52000020EAF6F81B2B4EF5AF0A0B19FEF5AF0A4
:10B53000AF67F8D7CAEC5AF036EC66F0D9D71FECF3
:10B5400062F02A0E9D630CD09A2B030E9A171650A8
:10B55000FC0B9A11166ECAEC5AF036EC66F0C8D79E
:10B56000230E9D63C5D78FD786EF57F016B409D049
:10B57000E80EF76EF40EF66E20EED6F018EC66F0DC
:10B580001200E80EF76EE40EF66E20EED6F018EC20
:10B5900066F012001650030B9A6F000E9A6309D0E2
:10B5A000E90EF76E040EF66E20EEE6F018EC66F08B
:10B5B0000ED0010E9A6309D0E90EF76E140EF66EE6
:10B5C00020EEE6F018EC66F002D09A6BE9D7120094
:10B5D000E90EF76E440EF66E20EED6F018EC66F02B
:10B5E000E90EF76E540EF66E20EEE6F018EC66F0FB
:10B5F00036EC66F081B286EF57F0A0B101EF5BF058
:10B60000F9D71FEC62F0230E9D638FEF57F0B2EC79
:10B6100034F0E90EF76EA40EF66E20EED6F018ECBC
:10B6200066F018C0A2F0000EA26309D0E90EF76E12
:10B63000B40EF66E20EEE6F018EC66F02ED0010E99
:10B64000A26309D0E90EF76EC40EF66E20EEE6F0A6
:10B6500018EC66F022D0020EA26309D0E90EF76E54
:10B66000D40EF66E20EEE6F018EC66F016D0030E5F
:10B67000A26309D0E90EF76EE40EF66E20EEE6F056
:10B6800018EC66F00AD0A26B186AE90EF76EB40ED9
:10B69000F66E20EEE6F018EC66F036EC66F0640E1E
:10B6A000B06F060EAF6F81B20DEF5CF0A0B175EF19
:10B6B0005BF0A2511862F3D7AF67F5D710EEEBF04D
:10B6C0000B0ECB6F200EE66ECB2FFDD736EC66F05F
:10B6D000640EB06F020EAF6F81B20DEF5CF0A0B1DF
:10B6E00075EF5BF0AF67F8D79ED71FEC62F02A0EBC
:10B6F0009D6305D0A22B040EA261A26B94D7230EEA
:10B700009D6391D7A2C018F0010EA2658CD7020EDE
:10B71000A26309D0E90EF76ED40EF66E20EED6F0D5
:10B7200018EC66F00BD0030EA26308D0E90EF76E9A
:10B73000E40EF66E20EED6F018EC66F0E90EF76E29
:10B74000F40EF66E20EEE6F018EC66F0826B19C08F
:10B7500083F098EC61F09E6B200EF46F300E8063E6
:10B7600080C0F4F081C0F5F036EC66F0640EB06F86
:10B77000060EAF6F81B20DEF5CF0A0B1DCEF5BF0B5
:10B78000AF67F8D7200EF46FF56F36EC66F0640EF5
:10B79000B06F020EAF6F81B20DEF5CF0A0B1DCEFC5
:10B7A0005BF0AF67F8D7300E806380C0F4F081C0E3
:10B7B000F5F036EC66F0DAD71FEC62F0230E9D63ED
:10B7C00015D0300E805F815F0A0E8003F3CF19F031
:10B7D00081511926000E196403D0320E196419D74D
:10B7E000300E806F310E816F9E6BB6D72A0E9D632F
:10B7F00006D0300E806F310E816F9E6BADD7000E7C
:10B800009E6302D0300E816F81C080F09DC081F0B8
:10B810009E2B030E9E63A0D7E3D786EF57F0640EEE
:10B82000AE6F0F0EAD6FF60EF76E740EF66E20EE65
:10B83000D6F018EC66F0F60EF76E840EF66E20EE7B
:10B84000E6F018EC66F036EC66F005EC65F0AD67F6
:10B85000FED7716B81A2A1EF35F088EF0FF0A06BDE
:10B86000916B926B936B956B946B966B906BA083C3
:10B87000A095A09B120044EC62F0A0A312000D5012
:10B8800009E0A0A706D0A08B640EB06F0DC0AFF08A
:10B8900001D0A09B32A016D0130E926513D0380EA3
:10B8A000926110D092C084F07CEC61F07F51E7ECA3
:10B8B0005CF08051E7EC5CF08151E7EC5CF00D0E40
:10B8C000E7EC5CF08E51060F926105D08E51FA0FB5
:10B8D000926501D008D08F51060F926112008F51EE
:10B8E000FA0F92651200A0B90BD0A0B705D092C094
:10B8F00095F0926BA079120092C093F0926B1200B7
:10B90000A0A704D092C094F0926B120092C096F05F
:10B91000926B9351945FD8A0946D9551965FD8A087
:10B92000966D0A0E94610ED096610CD032B0A6ECE2
:10B930005CF0902B050E90651200A093A099A08555
:10B94000906B1200A099A095906B120093C084F0A8
:10B950007CEC61F07F51E7EC5CF08051E7EC5CF04F
:10B960008151E7EC5CF0200EE7EC5CF095C084F0D0
:10B970007CEC61F07F51E7EC5CF08051E7EC5CF02F
:10B980008151E7EC5CF0200EE7EC5CF094C084F0B1
:10B990007CEC61F07F51E7EC5CF08051E7EC5CF00F
:10B9A0008151E7EC5CF0200EE7EC5CF096C084F08F
:10B9B0007CEC61F07F51E7EC5CF08051E7EC5CF0EF
:10B9C0008151E7EC5CF00D0EE7EC5CF0120000003A
:10B9D0000000A4A8FDD76D6E1200349034A21200AE
:10B9E00038A007D04150E842E842070B9A6F9AC04E
:10B9F000E6F0A12B030EA117000EA16302D03D0EAD
:10BA00000BD0010EA16302D07E0E06D0020EA16300
:10BA100002D07C0E01D07F0E10EEECF0E76E36EC1B
:10BA200066F012009F692A0E9D6301D01200230E5A
:10BA30009D6301D01200300E9D6303D00A0E9F6FEC
:10BA400012003A0E9D6112009D510F0B9F6F120064
:10BA50009DC09BF0300E9D6302D00A0E1DD02A0EB1
:10BA60009D6302D00B0E18D0230E9D6302D00C0EE6
:10BA700013D0410E9D6302D00D0E0ED0420E9D6379
:10BA800002D00E0E09D0430E9D6302D00F0E04D0DB
:10BA9000440E9D6302D0000E9B6F9B510F0B10094B
:10BAA000120001EED2F0200E976F200EEE6E972F4F
:10BAB00055EF5DF01200976F200EE66E972FFCD7C2
:10BAC000120009EE00F09A0E976F200EEE6E972F7F
:10BAD000FCD71200F4C19AF0000E9A6309D0F30E5D
:10BAE000F76E540EF66E20EEE6F018EC66F01200DB
:10BAF000010E9A6309D0F30EF76E640EF66E20EE17
:10BB0000E6F018EC66F01200020E9A6309D0F30E0C
:10BB1000F76E740EF66E20EEE6F018EC66F012008A
:10BB2000030E9A6309D0F30EF76E840EF66E20EEC4
:10BB3000E6F018EC66F01200040E9A6309D0F30EDA
:10BB4000F76E940EF66E20EEE6F018EC66F012003A
:10BB5000050E9A6309D0F30EF76EA40EF66E20EE72
:10BB6000E6F018EC66F01200060E9A6309D0F30EA8
:10BB7000F76EB40EF66E20EEE6F018EC66F01200EA
:10BB8000E60EF76E540EF66E20EEE6F018EC66F058
:10BB9000120022EE00F00D0EDF5CD8B41200410E50
:10BBA000DE6204D0540EDE6201D0120038BCE6D250
:10BBB0000000F86ADF0E686F2A0E696F68C0F7FF31
:10BBC00069C0F6FF22EE00F0060E6E6F0900F55018
:10BBD00006E0F550DE5C12E16E2FE6EF5DF068C026
:10BBE000F7FF69C0F6FF060EF626E86AF72209009D
:10BBF000F5CF6AF0000E6A630DD01200080E6927B7
:10BC0000E86A6823DF0E685DD9E1F20E695DD6E16E
:10BC10006A6B1200010E6A6302D03D801200FF0EB3
:10BC20006A6302D03D8212000E0E6A6302D03E802B
:10BC300012000F0E6A6302D03E82120022EE00F064
:10BC40002B0EDF621200060E6A5DD8A42AEF5EF0AA
:10BC500038841200110E6A5DD8A437EF5EF0CEEC86
:10BC600060F0E2EC60F06FC040F03D821200030E25
:10BC70006A5DD8A460EF5EF0CEEC60F0E2EC60F0BC
:10BC80003DB81200000E6F6302D059801200010E01
:10BC90006F6302D059821200020E6F6302D0598482
:10BCA0001200030E6F6302D059861200040E6F63F8
:10BCB00002D059881200050E6F631200598A1200D3
:10BCC000020E6A5DD8A4B4EF5EF0CEEC60F0E2EC58
:10BCD00060F03DB81200000E6F6302D05780120072
:10BCE000010E6F6302D057821200020E6F6302D002
:10BCF00057841200030E6F6302D057861200040EA1
:10BD00006F6302D057881200050E6F6306D0578A02
:10BD1000E2EC60F06FC070F01200060E6F6306D0A8
:10BD2000578CE2EC60F06FC070F01200070E6F638A
:10BD300002D0578E1200080E6F6302D05880120096
:10BD4000090E6F6302D058821200000E6F6302D09A
:10BD5000588412000B0E6F6302D0588612000C0E2E
:10BD60006F63120058881200160E6A5DD8A4DFEFC8
:10BD70005EF0CEEC60F0D9EC60F0E2EC60F03DB843
:10BD80001200000E6F6302D05A801200010E6F6322
:10BD900002D05A821200020E6F6302D05A8412003F
:10BDA000030E6F6302D05A861200040E6F6302D036
:10BDB0005A881200050E6F6312005A8A1200070E8D
:10BDC0006A5DD8A4FDEF5EF001EE8CF0120EA86F54
:10BDD000200EEE6EA82FE8EF5EF002EE08F011EEF6
:10BDE0008CF0100EA86F220EEF5C05E0EECFE6FFA0
:10BDF000A82FF3EF5EF03D861200100E6A5DD8A406
:10BE00001BEF5FF001EE9EF0120EA86F200EEE6E9B
:10BE1000A82F06EF5FF002EE08F011EE9EF0100E74
:10BE2000A86F220EEF5C05E0EECFE6FFA82F11EF22
:10BE30005FF03D841200040E6A5DD8A427EF5FF026
:10BE4000CEEC60F0E2EC60F06F51416E1200120E29
:10BE50006A5DD8A451EF5FF03D8C02EE07F0520E00
:10BE6000EF6202D06F6B1200530EEF6218D002EE39
:10BE70000CF0490EEF6208D002EE0EF00D0EEF62EC
:10BE80000ED0010E6F6F1200550EEF6208D002EE59
:10BE90000EF00D0EEF6203D0020E6F6F12006F698D
:10BEA0001200050E6A5DD8A495EF5FF0CEEC60F04D
:10BEB000E2EC60F0080EA86F11EE7CF0200EE66E4A
:10BEC000A82FFCD7020E6F6314D001EE7CF0550E44
:10BED000EE6E6E0EEE6E520EEE6E650EEE6E670E2E
:10BEE000EE6E690EEE6E730EEE6E2E0EEE6E3D8AE7
:10BEF000120002EE0BF0220EEF5C09E0050EA86FB7
:10BF000011EE7CF0EECFE6FFA82FFCD70CD0EE5060
:10BF100011EE7CF0080EA86F220EEF5C04E0EECF6D
:10BF2000E6FFA82FF9D73D8A1200080E6A5DD8A453
:10BF3000A9EF5FF0CEEC60F0D9EC60F0E3EC60F0DC
:10BF400000EE43F06FC042F06F516FC0EBFF388AD4
:10BF500012000B0E6A5DD8A4C0EF5FF0CEEC60F06B
:10BF6000D9EC60F0DE50200EA86F08EE32F0220E01
:10BF7000DF5C04E0DECFEEFFA82FF9D7388C12008B
:10BF80000C0E6A5DD8A4C7EF5FF03F841200130E59
:10BF90006A5DD8A4E4EF5FF0CEEC60F0DE50100EE6
:10BFA000A86F08EE12F0200EEE6EA82FFCD708EE58
:10BFB00012F0100EA86FDF500D0804E0DECFEEFF88
:10BFC000A82FF9D73F861200140E6A5DD8A4F3EFAC
:10BFD0005FF0CEEC60F0E2EC60F03F98000E6F6333
:10BFE00012003F881200150E6A5DD8A49FEF60F022
:10BFF000CEEC60F009EE00F03CEC60F0DE50D9ECE5
:10C0000060F0D9EC60F0D9EC60F0D9EC60F0D9ECDC
:10C0100060F018EC61F02C0EDF621200DE5009EEC9
:10C0200016F03CEC60F00D0EDE5CD8B4120009EEA8
:10C030002CF03CEC60F00D0EDE5CD8B4120009EE82
:10C0400042F03CEC60F00D0EDE5CD8B4120009EE5C
:10C0500058F03CEC60F00D0EDE5CD8B4120009EE36
:10C060006EF03CEC60F00D0EDE5CD8B4120009EE10
:10C0700084F03CEC60F0120018EC61F0200E7C6F54
:10C080007D6F7E6F7F6F806F816F10EE7CF0200E72
:10C09000866386C0E6FF876387C0E6FF886388C043
:10C0A000E6FF896389C0E6FFDE5018EC61F0200EE0
:10C0B000866386C0E6FF876387C0E6FF886388C023
:10C0C000E6FF896389C0E6FF7CC0EEFF7DC0EEFF1E
:10C0D0007EC0EEFF7FC0EEFF80C0EEFF81C0EEFFAE
:10C0E000DE50D9EC60F018EC61F086C0EEFF87C03E
:10C0F000EEFF88C0EEFF89C0EEFFDE5018EC61F065
:10C1000086C0EEFF87C0EEFF88C0EEFF89C0EEFF5D
:10C11000DE5018EC61F086C0EEFF87C0EEFF88C0ED
:10C12000EEFF89C0EEFFDE5018EC61F086C0EEFF36
:10C1300087C0EEFF88C0EEFF89C0EEFF1200170E29
:10C140006A5DD8A4B1EF60F0CEEC60F0E2EC60F094
:10C150006FC0F2F1D9EC60F0E3EC60F06FC0F3F186
:10C160001200180E6A5DD8A4BDEF60F0CEEC60F04E
:10C17000E2EC60F06FC0F4F112001200389C780E0F
:10C18000A86F08EE52F012EE00F00D0EE75C04E02E
:10C19000E6CFEEFFA82FF9D7EF6A120022EE00F0EB
:10C1A000800E6E6F3A0EDE5C03E06E2FD2EF60F011
:10C1B0001200FF0E6E6F2C0EDE5C03E06E2FDBEFC5
:10C1C00060F01200DE503D98300E876F886F896FE7
:10C1D000DECF89F00D0EDF5C13E02C0EDF5C10E08B
:10C1E00089C088F0DECF89F00D0EDF5C09E02C0EEF
:10C1F000DF5C06E088C087F089C088F0DECF89F078
:10C20000320E876503D03D88300E876F6F6B300E1E
:10C21000875F885F895F0A0E8703F3500A0DF3CFAB
:10C220006FF00A0E8803F3506F2789516F271200B1
:10C23000200E866F876F886F896F040EA86F2C0E93
:10C24000DF5CD8B412000D0EDF5CD8B4120087C0DA
:10C2500086F088C087F089C088F0DECF89F0A82FEB
:10C26000EED71200846B300E7F5D640DF3CF84F047
:10C27000300E805D0A0DF3508427300E815D8427D7
:10C280001200836B826B300E755F765F775F785F2D
:10C29000795F060E75612DD0000E756507D0100E02
:10C2A0008327270E8223752F4FEF61F0000E7665EE
:10C2B00007D0E80E8327030E8223762F59EF61F013
:10C2C000000E776507D0640E8327000E8223772F38
:10C2D00063EF61F0000E786507D00A0E8327000E29
:10C2E0008223782F6DEF61F079518327E86A8223EA
:10C2F00012008269836912007F6B806B816B630E11
:10C30000846506D0640E845F02E37F2BFBD784270D
:10C31000090E846506D00A0E845F02E3802BFBD7EA
:10C32000842784C081F0300E7F2780278127120068
:10C330007D6B7E6B7F6B806B816B100E835F270E36
:10C34000825B02E37D2BF9D7100E8327270E822311
:10C35000E80E835F030E825B02E37E2BF9D7E80EC3
:10C360008327030E8223640E835F000E825B02E349
:10C370007F2BF9D7640E8327000E82230A0E835F7A
:10C38000000E825B02E3802BF9D70A0E8327000E92
:10C39000822383C081F0300E7D277E277F27802770
:10C3A0008127120018EC62F0C06BC16BBF9F1200B6
:10C3B000D9C9E8FF070BE8461009CE6F0C0ECF6F06
:10C3C000F8EC62F01200DBC9E8FF070BE846100941
:10C3D000CE6F0D0ECF6FF8EC62F01200DDC9E8FFF2
:10C3E000070BE8461009CE6F0D0ECF6FF8EC62F028
:10C3F0001200DFC9E8FF070BE8461009CE6F0E0EEA
:10C40000CF6FF8EC62F01200120ECE6F0C0ECF6FF1
:10C41000F8EC62F01200120ECE6F0F0ECF6FF8EC38
:10C4200062F01200CF6F160ECE6FF8EC62F01200C1
:10C43000000ECE6F000ECF6FF8EC62F012000CEC25
:10C4400063F0CF510F0B9D6F9D6703D00F0E9D6F53
:10C4500017D0090E9D6514D00A0E9D6303D0000EFF
:10C460009D6F0ED00B0E9D6303D0FA0E9D6F08D00A
:10C470000C0E9D6303D0F30E9D6F02D00F0E9D6FC7
:10C48000300E9D27A09112000CEC63F0CEB5A08772
:10C49000CEA5A097A0911200110ECE6F800ECF6F87
:10C4A000F3EC62F01E0EAB6FAB6754EF62F0110E4F
:10C4B000CE6F000ECF6FF3EC62F0800ED16F000EE6
:10C4C000D26FE2EC62F0CAC9D1F0CBC9D2F0E2EC93
:10C4D00062F0D6C9D1F0D7C9D2F0E2EC62F0CCC993
:10C4E000D1F0CDC9D2F0E2EC62F0D6C9D1F0D7C913
:10C4F000D2F0E2EC62F0CEC9D1F0CFC9D2F0E2ECDA
:10C5000062F0D6C9D1F0D7C9D2F0E2EC62F0D0C95E
:10C51000D1F0D1C9D2F0E2EC62F0D6C9D1F0D7C9DE
:10C52000D2F0E2EC62F0D2C9D1F0D3C9D2F0E2ECA1
:10C5300062F0D6C9D1F0D7C9D2F0E2EC62F0D4C92A
:10C54000D1F0D5C9D2F0E2EC62F0D6C9D1F0D7C9AA
:10C55000D2F0E2EC62F01C0ED16F680ED26FE2EC0A
:10C5600062F0240ED16FA20ED26FE2EC62F0240EC4
:10C57000D16FAD0ED26FE2EC62F0240ED16FA20E3D
:10C58000D26FE2EC62F0110ECE6F16EC63F0120087
:10C590001E0ECE6F010ECF6FFDEC62F0110ECE6F4E
:10C5A000410ECF6FF3EC62F012001E0ECE6F030E41
:10C5B000CF6FFDEC62F0110ECE6F440ECF6FF3EC37
:10C5C00062F01200D1C0CEF0D2C0CFF011EC63F017
:10C5D000020EAB6FAB67EAEF62F01200010ECD6F97
:10C5E00055EC63F01200E00ECD6F33EC63F01200F7
:10C5F000E10ECD6F33EC63F01200E20ECD6F33EC41
:10C6000063F01200E30ECD6F1BEC63F01200E50E39
:10C61000CD6F26EC63F01200E60ECD6F42EC63F0B6
:10C620001200E80ECD6F33EC63F01200EC0ECD6F0C
:10C630001BEC63F012008498CDC0CCF055EC63F095
:10C64000CEC0CCF055EC63F0848812008498CDC045
:10C65000CCF055EC63F0000ECC6F55EC63F0CCC021
:10C66000CEF0848812008498CDC0CCF055EC63F0F5
:10C67000CEC0CCF055EC63F0CFC0CCF055EC63F0FD
:10C68000848812008498CDC0CCF055EC63F0000E85
:10C69000CC6F55EC63F0CCC0CEF0000ECC6F55ECF7
:10C6A00063F0CCC0CFF084881200000000000000CE
:10C6B0000000080ED06FD890CC37D8A08394D8B0A3
:10C6C000838483920000000000000000000000004E
:10C6D000000000000000838200008350010BCC1397
:10C6E00000000000D02F5BEF63F01200849C849A5E
:10C6F000100EA36FA6C0A4F0A7C0A5F0D890A533D4
:10C70000A433D8A0849ED8B0848E0000000000001E
:10C710000000848C00000000000000000000000009
:10C7200000000000849CA32F7EEF63F00000000057
:10C73000000000000000000000000000848A0000EB
:10C7400000000000000000000000000000000000E9
:10C750000000000000000000000000000000849ABB
:10C760001200000E1464190C010E1464250C020E44
:10C770001464280C030E1464320C030E146E320C75
:10C78000000E1564190C010E1564250C020E1564BB
:10C79000280C030E1564320C156A190C240EE8CF10
:10C7A000D6F9A20EE8CFD7F9D8C9FDF00F0EFD17C4
:10C7B000000EFD630DD0040EE8CFCAF9AB0EE8CF32
:10C7C000CBF9050EE8CFCCF9DE0EE8CFCDF92FD0AE
:10C7D000010EFD630DD0040EE8CFCAF9AB0EE8CF11
:10C7E000CBF9060EE8CFCCF9000EE8CFCDF91FD07B
:10C7F000020EFD630DD0050EE8CFCAF9550EE8CF45
:10C80000CBF9050EE8CFCCF9DE0EE8CFCDF90FD08D
:10C81000030EFD63D0D7050EE8CFCAF9550EE8CF59
:10C82000CBF9000EE8CFCCF9000EE8CFCDF9DAC98C
:10C83000FDF00F0EFD17000EFD630DD0060EE8CFC4
:10C84000CEF9670EE8CFCFF9080EE8CFD0F9450E44
:10C85000E8CFD1F92FD0010EFD630DD0050EE8CF42
:10C86000CEF9550EE8CFCFF9000EE8CFD0F9000E83
:10C87000E8CFD1F91FD0020EFD630DD0050EE8CF31
:10C88000CEF9AA0EE8CFCFF9000EE8CFD0F9000E0E
:10C89000E8CFD1F90FD0030EFD63D0D7050EE8CF56
:10C8A000CEF9550EE8CFCFF9000EE8CFD0F9000E43
:10C8B000E8CFD1F9DEC9FDF00F0EFD17000EFD63C4
:10C8C0000DD0050EE8CFD2F9DE0EE8CFD3F9060E73
:10C8D000E8CFD4F9670EE8CFD5F91200010EFD6359
:10C8E0000DD0050EE8CFD2F9550EE8CFD3F9060EDC
:10C8F000E8CFD4F9000EE8CFD5F91200020EFD639F
:10C900000DD0050EE8CFD2F9AA0EE8CFD3F9000E6C
:10C91000E8CFD4F9000EE8CFD5F91200030EFD637D
:10C92000D0D7050EE8CFD2F9550EE8CFD3F9000ED7
:10C93000E8CFD4F9000EE8CFD5F9120000EE0CF0E4
:10C94000260ECB6F030EAA6E000EA96EF9EC64F0F2
:10C9500009EED8F0140ECB6F030EAA6ECA0EA96EA4
:10C96000F9EC64F009EE9AF0280ECB6F030EAA6E74
:10C97000260EA96EF9EC64F001EE00F07C0ECB6F90
:10C98000030EAA6E4E0EA96EF9EC64F004EE40F0B0
:10C99000800ECB6F000EAA6E000EA96EF9EC64F04B
:10C9A00005EE00F0A00ECB6F000EAA6E800EA96EF1
:10C9B000F9EC64F005EEA0F0A00ECB6F010EAA6EAC
:10C9C000200EA96EF9EC64F006EE40F0A00ECB6FDD
:10C9D000010EAA6EC00EA96EF9EC64F006EEE0F04E
:10C9E000A00ECB6F020EAA6E600EA96EF9EC64F079
:10C9F0001200A69EA69CA6800000A8CFEEFFA92A42
:10CA0000E86AAA22CB2FF7D7120001EE04F0180E25
:10CA1000CB6F030EAA6E520EA96EE9EC65F022EC04
:10CA200065F02DEC65F04CEC65F057EC65F076ECBC
:10CA300065F08BEC65F0A0EC65F0B5EC65F0C0EC52
:10CA400065F0120001EE00F0040ECB6F030EAA6E2B
:10CA50004E0EA96EE9EC65F0120000EE0CF00A0E25
:10CA6000CB6F030EAA6E000EA96EE9EC65F001EE25
:10CA700070F00C0ECB6F030EAA6EBE0EA96EE9EC21
:10CA800065F001EE50F0100ECB6F030EAA6E9E0EF5
:10CA9000A96EE9EC65F0120000EE16F0080ECB6FFF
:10CAA000030EAA6E0A0EA96EE9EC65F0120000EE04
:10CAB0001EF0060ECB6F030EAA6E120EA96EE9ECE5
:10CAC00065F001EE60F0100ECB6F030EAA6EAE0E95
:10CAD000A96EE9EC65F001EE40F0100ECB6F030E8D
:10CAE000AA6E8E0EA96EE9EC65F0120000EE24F03D
:10CAF0000A0ECB6F030EAA6E180EA96EE9EC65F054
:10CB000009EE9AF0280ECB6F030EAA6E260EA96EC0
:10CB1000E9EC65F0120000EE2EF0010ECB6F030E73
:10CB2000AA6E220EA96EE9EC65F001EE1CF0240E4F
:10CB3000CB6F030EAA6E6A0EA96EE9EC65F01200C7
:10CB400000EE30F0010ECB6F030EAA6E240EA96E1C
:10CB5000E9EC65F009EED8F0140ECB6F030EAA6E67
:10CB6000CA0EA96EE9EC65F0120004EE40F0800EEA
:10CB7000CB6F000EAA6E000EA96EE9EC65F01200F4
:10CB800005EE00F0A00ECB6F000EAA6E800EA96E0F
:10CB9000E9EC65F005EEA0F0A00ECB6F010EAA6ED9
:10CBA000200EA96EE9EC65F006EE40F0A00ECB6F0A
:10CBB000010EAA6EC00EA96EE9EC65F006EEE0F07B
:10CBC000A00ECB6F020EAA6E600EA96EE9EC65F0A6
:10CBD0001200A69EA69CA684F29EF29CEECFA8FF11
:10CBE000550EA76EAA0EA76EA682F28CF28EA6B282
:10CBF000F7EF65F0A92AE86AAA22CB2FECEF65F0DF
:10CC0000A694120003EE00F0EE5005E0AD6E0000B9
:10CC10009EA8FED7F9D70D0EAD6E00009EA8FED7D8
:10CC20001200F86A0900F5500CE0DE6E04D0120024
:10CC3000F86A100E986F0900F55003E0DE6E982F29
:10CC4000FAD71200100EC76F20EED6F0200EDE6E5F
:10CC5000C72F26EF66F01200100EC76F20EEE6F029
:10CC6000200EDE6EC72F30EF66F01200080E91EC3A
:10CC700066F0000E91EC66F0100EC76F20EED6F055
:10CC8000DE50A0EC66F0C72F40EF66F00C0E91EC82
:10CC900066F0000E91EC66F0100EC76F20EEE6F025
:10CCA000DE50A0EC66F0C72F50EF66F01200030EC6
:10CCB00091EC66F0280EAB6FAB675CEF66F0030E8D
:10CCC00091EC66F00A0EAB6FAB6764EF66F0030E93
:10CCD00091EC66F0020E91EC66F0020E91EC66F0BB
:10CCE000080E91EC66F0000E91EC66F0080E91ECE7
:10CCF00066F0000E91EC66F0010E91EC66F00A0E03
:10CD0000AB6FAB6781EF66F0000E91EC66F0060E3C
:10CD100091EC66F0000E91EC66F00C0E91EC66F072
:10CD20001200E83AF00B856E8596859485820000A6
:10CD3000000085923C0E9C6F9C2F9CEF66F01200C9
:10CD4000C66FF00B856E8586859485820000000095
:10CD50008592C639F00B856E8586859485820000A4
:10CD6000000085923C0E9C6F9C2FB4EF66F0120081
:10CD7000F29E040E91EC66F0000E91EC66F0000E4F
:10CD8000A0EC66F0000EA0EC66F0000EA0EC66F0E1
:10CD9000000EA0EC66F0000EA0EC66F0000EA0EC19
:10CDA00066F0000EA0EC66F0180EA0EC66F0000E27
:10CDB000A0EC66F0000EA0EC66F0000EA0EC66F0B1
:10CDC000000EA0EC66F0000EA0EC66F0000EA0ECE9
:10CDD00066F0180EA0EC66F0180EA0EC66F0000EDF
:10CDE000A0EC66F0000EA0EC66F0000EA0EC66F081
:10CDF000000EA0EC66F0000EA0EC66F01C0EA0EC9D
:10CE000066F0180EA0EC66F0180EA0EC66F0000EAE
:10CE1000A0EC66F0000EA0EC66F0000EA0EC66F050
:10CE2000000EA0EC66F01C0EA0EC66F01C0EA0EC50
:10CE300066F0180EA0EC66F0180EA0EC66F0000E7E
:10CE4000A0EC66F0000EA0EC66F0000EA0EC66F020
:10CE50001E0EA0EC66F01C0EA0EC66F01C0EA0EC02
:10CE600066F0180EA0EC66F0180EA0EC66F0000E4E
:10CE7000A0EC66F0000EA0EC66F01E0EA0EC66F0D2
:10CE80001E0EA0EC66F01C0EA0EC66F01C0EA0ECD2
:10CE900066F0180EA0EC66F0180EA0EC66F0000E1E
:10CEA000A0EC66F01F0EA0EC66F01E0EA0EC66F083
:10CEB0001E0EA0EC66F01C0EA0EC66F01C0EA0ECA2
:10CEC00066F0180EA0EC66F0180EA0EC66F01F0ECF
:10CED000A0EC66F01F0EA0EC66F01E0EA0EC66F053
:10CEE0001E0EA0EC66F01C0EA0EC66F01C0EA0EC72
:10CEF00066F0180EA0EC66F0180EA0EC66F0F28E4C
:10CF000012000AEE00F00D0EEF6209D00BEE00F0F9
:10CF10003F0EEE6E0D0EEE6E87EC6FF01200440EBB
:10CF2000EE6226D04C0EEE6223D0440EEE6220D08C
:10CF3000FF0ED16FD26F00EED1F0020ECB6F030E59
:10CF4000AA6EFE0EA96EE9EC65F0E30EF76EC40E54
:10CF5000F66E20EED6F018EC66F0E30EF76ED40E07
:10CF6000F66E20EEE6F018EC66F036EC66F0FF00A8
:10CF70000AEE00F0440EEE622BD0420EEE6228D094
:10CF8000470EEE6225D0C3EC6CF0080E8461A3EF6F
:10CF90006CF084C0FBF02C0EEE62A3EF6CF0C3ECDF
:10CFA0006CF0020E8461A3EF6CF00D0EEE62A3EF45
:10CFB0006CF0FB2BD89081698137FB2FFDD7815115
:10CFC00084A13216E81E84B132126BEC6FF01200AD
:10CFD0000AEE00F0430EEE625AD0500EEE6257D0C9
:10CFE000570EEE6254D0339E00C1E8FFEE6225D0AA
:10CFF00001C1E8FFEE6221D002C1E8FFEE621DD060
:10D0000003C1E8FFEE6219D00D0EEE6216D0338E2A
:10D010006BEC6FF0DAEC6CF0F2EC6CF036EC6DF07F
:10D0200063EC6DF097EC6DF0E8EC6DF003EC6EF0F6
:10D0300064EC6EF0D0EC6EF012000AEE03F0450ED8
:10D04000EE62A3EF6CF0750EEE62A3EF6CF0720E61
:10D05000EE62A3EF6CF06F0EEE62A3EF6CF0740E55
:10D06000EE62A3EF6CF0650EEE62A3EF6CF0630E60
:10D07000EE62A3EF6CF0680EEE62A3EF6CF00D0EA3
:10D08000EE62A3EF6CF0338E6BEC6FF012000AEEE1
:10D0900000F0520EEE621ED0420EEE621BD0540E15
:10D0A000EE6218D0E30EF76EE40EF66E20EED6F0C8
:10D0B00018EC66F0E30EF76EF40EF66E20EEE6F076
:10D0C00018EC66F036EC66F005EC65F00000000048
:10D0D000AAEF07F00AEE00F0500EEE6224D0530ED5
:10D0E000EE6221D0570EEE621ED033AEA3EF6CF08D
:10D0F000EECF7EF0EECF7FF0EECF80F0EECF81F07E
:10D100000D0EEE62A3EF6CF001EE00F07EC0EEFFBC
:10D110007FC0EEFF80C0EEFF81C0EEFF22EC65F025
:10D120006BEC6FF0120033AEA3EF6CF00AEE00F080
:10D13000460EEE62BBD0580EEE62B8D04F0EEE62D5
:10D14000B5D0C3EC6CF084C000FC2C0EEE62A3EFF3
:10D150006CF0100E1CEE01F05BEC5DF0100EFB6F3E
:10D160001CEE01F02C0EEF5C04E0EECFE6FFFB2F8F
:10D17000F9D72C0EEE62A3EF6CF0C3EC6CF084C018
:10D1800011FC2C0EEE62A3EF6CF0C3EC6CF084C0CB
:10D1900012FC2C0EEE62A3EF6CF0C3EC6CF084C0BA
:10D1A00013FC2C0EEE62A3EF6CF0C3EC6CF084C0A9
:10D1B00014FC2C0EEE62A3EF6CF0C3EC6CF084C098
:10D1C00015FC2C0EEE62A3EF6CF0C3EC6CF084C087
:10D1D00016FC2C0EEE62A3EF6CF0C3EC6CF084C076
:10D1E00017FC2C0EEE62AFD30C0E1CEE18F05BECAD
:10D1F0005DF0080EFB6F1CEE18F02C0EEF5C04E0E7
:10D20000EECFE6FFFB2FF9D72C0EEE629CD3040E77
:10D21000FB6F1CEE20F02C0EEF5C04E0EECFE6FF7F
:10D22000FB2FF9D72C0EEE628ED3C3EC6CF084C0CA
:10D2300024FC2C0EEE6287D3C3EC6CF084C025FC7A
:10D240000D0EEE6280D300CC0CF025CC0DF011CC8D
:10D250000EF024CC0FF012CC10F013CC11F014CC43
:10D2600012F015CC13F016CC14F017CC15F00C0EF0
:10D27000FB6F1CEE18F001EE70F0E6CFEEFFFB2F17
:10D28000FCD7100EFB6F1CEE01F001EE50F0E6CF64
:10D29000EEFFFB2FFCD72DEC65F06BEC6FF0B1ECE3
:10D2A00063F08E6FC0EC63F08F6F12000AEE00F037
:10D2B000460EEE6253D0580EEE6250D0530EEE6220
:10D2C0004DD0C3EC6CF084C000FC2C0EEE623BD35E
:10D2D000C3EC6CF084C001FC2C0EEE6234D3C3ECC2
:10D2E0006CF084C002FC2C0EEE622DD3C3EC6CF00B
:10D2F00084C003FC2C0EEE6226D3C3EC6CF084C019
:10D3000004FC2C0EEE621FD3C3EC6CF084C005FC51
:10D310002C0EEE6218D3C3EC6CF084C006FC2C0E0D
:10D32000EE6211D3C3EC6CF084C007FC0D0EEE620C
:10D330000AD300CC16F006CC18F007CC19F001CCBB
:10D3400017F002CC1AF003CC1BF004CC1CF005CC77
:10D350001DF04CEC65F06BEC6FF012000AEE00F083
:10D36000470EEE628AD0530EEE6287D04D0EEE620B
:10D3700084D0C3EC6CF084C000FC2C0EEE62E3D2CF
:10D38000100E1CEE01F05BEC5DF0100EFB6F1CEE5E
:10D3900001F02C0EEF5C04E0EECFE6FFFB2FF9D797
:10D3A0002C0EEE62D0D2C3EC6CF084C011FC2C0EBB
:10D3B000EE62C9D2C3EC6CF084C012FC2C0EEE629B
:10D3C000C2D2100E1CEE13F05BEC5DF0080EFB6F8A
:10D3D0001CEE13F02C0EEF5C04E0EECFE6FFFB2F0B
:10D3E000F9D72C0EEE62AFD2080EFB6F1CEE1BF0CD
:10D3F0002C0EEF5C04E0EECFE6FFFB2FF9D72C0EEE
:10D40000EE62A1D2C3EC6CF084C023FC2C0EEE6261
:10D410009AD2C3EC6CF084C024FC2C0EEE6293D242
:10D42000C3EC6CF084C025FC0D0EEE628CD200CCF7
:10D430001EF011CC22F012CC23F023CC20F024CC0F
:10D4400021F025CC1FF0100EFB6F1CEE01F001EE59
:10D4500060F0E6CFEEFFFB2FFCD7100EFB6F1CEE4B
:10D4600013F001EE40F0E6CFEEFFFB2FFCD757ECB8
:10D4700065F038866BEC6FF012000AEE00F04E0E8D
:10D48000EE62BCD0450EEE62B9D0540EEE62B6D05C
:10D49000C3EC6CF084C000FC2C0EEE6254D2C3ECE2
:10D4A0006CF084C001FC2C0EEE624DD2A6EC6CF048
:10D4B00083C002FC82C003FC2C0EEE6244D22E0E0E
:10D4C0001CEE04F05BEC5DF0060EFB6F1CEE04F04E
:10D4D0002C0EEF5C04E0EECFE6FFFB2FF9D72C0E0D
:10D4E000EE62060EFB6F1CEE0AF02C0EEF5C04E001
:10D4F000EECFE6FFFB2FF9D72C0EEE6224D2060EFC
:10D50000FB6F1CEE12F02C0EEF5C04E0EECFE6FF9A
:10D51000FB2FF9D72C0EEE6216D2A6EC6CF083C06E
:10D5200018FC82C019FC2C0EEE620DD2060EFB6FA9
:10D530001CEE1AF02C0EEF5C04E0EECFE6FFFB2FA2
:10D54000F9D72C0EEE62FFD1A6EC6CF083C020FC64
:10D5500082C021FC2C0EEE62F6D1060EFB6F1CEE93
:10D5600022F02C0EEF5C04E0EECFE6FFFB2FF9D7A4
:10D570002C0EEE62E8D1A6EC6CF083C028FC82C0D1
:10D5800029FC2C0EEE62DFD1060EFB6F1CEE2AF09A
:10D590002C0EEF5C04E0EECFE6FFFB2FF9D72C0E4C
:10D5A000EE62D1D1A6EC6CF083C030FC82C031FCBD
:10D5B0000D0EEE62C8D100CC24F001CC25F002CCD7
:10D5C00026F003CC27F004CC28F005CC29F006CCBB
:10D5D0002AF007CC2BF008CC2CF009CC2DF0280E2B
:10D5E000FB6F09EE9AF01CEE0AF0E6CFEEFFFB2F80
:10D5F000FCD776EC65F06BEC6FF012000AEE00F0F1
:10D60000530EEE623FD04D0EEE623CD0530EEE62F2
:10D6100039D0C3EC6CF084C000FC2C0EEE6293D1C8
:10D62000240E1CEE01F05BEC5DF0100EFB6F1CEEA7
:10D6300001F02C0EEF5C04E0EECFE6FFFB2FF9D7F4
:10D640002C0EEE6280D1100EFB6F1CEE13F00D0E4F
:10D65000EF5C04E0EECFE6FFFB2FF9D70D0EEE6294
:10D6600072D100CC2EF0240EFB6F1CEE01F001EE07
:10D670001CF0E6CFEEFFFB2FFCD78BEC65F06BECDC
:10D680006FF012000AEE00F0500EEE6251D0520E12
:10D69000EE624ED0460EEE624BD0C3EC6CF02C0E18
:10D6A000EE6251D1210E84614ED1000E84654BD1C2
:10D6B000840784C000FC080EFB6F1CEE01F0E668D6
:10D6C000FB2FFDD7070EFB6F1CEE01F02C0EEF5C5D
:10D6D00005E0EE500F0BE66EFB2FF8D72C0EEE6236
:10D6E00032D1C3EC6CF084C008FC0D0EEE622BD17D
:10D6F000040EFB6F1CEE01F004EE40F000CCE8FFDE
:10D70000040DF350E926F450EA22E638F00BEF6EF0
:10D71000E6500F0BEE12FB2FF8D71F0E006103D05F
:10D720006BEC6FF01200B5EC65F06BEC6FF0120073
:10D730000AEE00F04C0EEE6253D0530EEE6250D063
:10D74000540EEE624DD0C3EC6CF02C0EEE62FBD0AA
:10D75000410E8461F8D0000E8465F5D0840784C042
:10D7600000FC100EFB6F1CEE01F0E668FB2FFDD7EE
:10D77000100EFB6F1CEE01F02C0EEF5C05E0EE507E
:10D780000F0BE66EFB2FF8D72C0EEE62DCD0C3EC4D
:10D790006CF084C011FC0D0EEE62D5D0080EFB6F4C
:10D7A0001CEE01F005EE00F000CCE8FF0A0DF3508E
:10D7B000E926F450EA22E638F00BEF6EE6500F0B44
:10D7C000EE12FB2FF8D711CCEFFF3F0E006103D014
:10D7D0006BEC6FF01200C0EC65F06BEC6FF01200B8
:10D7E0000AEE00F0470EEE62AED0570EEE62ABD0FE
:10D7F000500EEE62A8D0C3EC6CF084C000FC2C0E7E
:10D80000EE62A1D0C3EC6CF084C001FC2C0EEE6281
:10D810009AD0C3EC6CF084C002FC2C0EEE6293D064
:10D82000C3EC6CF084C003FC2C0EEE628CD0C3EC15
:10D830006CF084C004FC2C0EEE6285D0C3EC6CF05E
:10D8400084C005FC2C0EEE627ED0C3EC6CF084C06C
:10D8500006FC2C0EEE6277D0C3EC6CF084C007FCA3
:10D860002C0EEE6270D0C3EC6CF084C008FC2C0E61
:10D87000EE6269D0C3EC6CF084C009FC2C0EEE6241
:10D8800062D0C3EC6CF084C00AFC2C0EEE625BD05C
:10D89000C3EC6CF084C00BFC2C0EEE6254D0C3ECD5
:10D8A0006CF084C00CFC2C0EEE624DD0C3EC6CF01E
:10D8B00084C00DFC2C0EEE6246D0C3EC6CF084C02C
:10D8C0000EFC2C0EEE623FD0C3EC6CF084C00FFC5B
:10D8D0002C0EEE6238D0C3EC6CF084C010FC2C0E21
:10D8E000EE6231D0C3EC6CF084C011FC2C0EEE6201
:10D8F0002AD0C3EC6CF084C012FC2C0EEE6223D054
:10D90000C3EC6CF084C013FC2C0EEE621CD0C3EC94
:10D910006CF084C014FC0D0EEE6215D000CC30F01B
:10D92000140EFB6F1CEE01F009EED8F0E6CFEEFF0F
:10D93000FB2FFCD7A0EC65F06BEC6FF0CEEC63F046
:10D940004CEC62F0120076EC6FF01200300E756F46
:10D95000766F776F786F796F050E976F2C0EEF5C8F
:10D960000FE00D0EEF5C0CE076C075F077C076F03E
:10D9700078C077F079C078F0EECF79F0972FEED7B6
:10D9800041EC61F01200300E7F6F806F816F030EEB
:10D99000976F2C0EEF5C0BE00D0EEF5C08E080C083
:10D9A0007FF081C080F0EECF81F0972FF2D732EC7C
:10D9B00061F01200FF0EF76EB20EF66E0BEE00F085
:10D9C000560EEE6E450EEE6E520EEE6E100EFA6FA5
:10D9D0000900F5CFEEFFFA2FFBD70D0EEE6E87ECA8
:10D9E0006FF012000BEE00F0460EEE6E580EEE6E6B
:10D9F0004F0EEE6E0CC084F036EC6FF011EE50F06E
:10DA0000100E5EEC6FF00EC084F034EC6FF010C0BE
:10DA100084F034EC6FF011C084F034EC6FF012C07D
:10DA200084F034EC6FF013C084F034EC6FF014C069
:10DA300084F034EC6FF015C084F034EC6FF011EE2C
:10DA400070F0080E5EEC6FF011EE78F0040E5EECF4
:10DA50006FF00FC084F034EC6FF00DC084F034EC44
:10DA60006FF00D0EEE6E87EC6FF012000BEE00F013
:10DA7000460EEE6E580EEE6E530EEE6E16C084F02D
:10DA800036EC6FF017C084F034EC6FF01AC084F0FD
:10DA900034EC6FF01BC084F034EC6FF01CC084F0E9
:10DAA00034EC6FF01DC084F034EC6FF018C084F0DB
:10DAB00034EC6FF019C084F034EC6FF00D0EEE6EA4
:10DAC00087EC6FF012000BEE00F0470EEE6E530E77
:10DAD000EE6E4D0EEE6E1EC084F036EC6FF011EE61
:10DAE00060F0100E5EEC6FF022C084F034EC6FF04A
:10DAF00023C084F034EC6FF011EE40F0080E5EECC1
:10DB00006FF011EE48F0080E5EEC6FF020C084F06C
:10DB100034EC6FF021C084F034EC6FF01FC084F05F
:10DB200034EC6FF00D0EEE6E87EC6FF012000BEE22
:10DB300000F04E0EEE6E450EEE6E540EEE6E24C0EC
:10DB400084F036EC6FF025C084F034EC6FF026C022
:10DB500083F027C082F045EC6FF0060E10EE28F03F
:10DB60005EEC6FF019EE9AF0060E5EEC6FF019EEB7
:10DB7000A2F0060E5EEC6FF0A8C983F0A9C982F08E
:10DB800045EC6FF019EEAAF0060E5EEC6FF0B0C92E
:10DB900083F0B1C982F045EC6FF019EEB2F0060ED9
:10DBA0005EEC6FF0B8C983F0B9C982F045EC6FF054
:10DBB00019EEBAF0060E5EEC6FF0C0C983F0C1C971
:10DBC00082F045EC6FF00D0EEE6E87EC6FF01200F8
:10DBD0000BEE00F0530EEE6E4D0EEE6E530EEE6E2B
:10DBE0002EC084F036EC6FF011EE1CF0100E5EECDF
:10DBF0006FF011EE2EF0100E5EEC6FF00D0EEE6E6B
:10DC000087EC6FF012000BEE00F0470EEE6E570E31
:10DC1000EE6E500EEE6E30C084F036EC6FF0D8C968
:10DC200084F034EC6FF0D9C984F034EC6FF0DAC9C9
:10DC300084F034EC6FF0DBC984F034EC6FF0DCC9B5
:10DC400084F034EC6FF0DDC984F034EC6FF0DEC9A1
:10DC500084F034EC6FF0DFC984F034EC6FF0E0C98D
:10DC600084F034EC6FF0E1C984F034EC6FF0E2C979
:10DC700084F034EC6FF0E3C984F034EC6FF0E4C965
:10DC800084F034EC6FF0E5C984F034EC6FF0E6C951
:10DC900084F034EC6FF0E7C984F034EC6FF0E8C93D
:10DCA00084F034EC6FF0E9C984F034EC6FF0EAC929
:10DCB00084F034EC6FF0EBC984F034EC6FF00D0EAF
:10DCC000EE6E87EC6FF01200200EFC6F14EE40F049
:10DCD0000BEE00F0500EEE6E520EEE6E460EEE6E35
:10DCE000D880210EFC55846F7CEC61F080C0EEFF83
:10DCF00081C0EEFF2C0EEE6EE7380F0B7A6F0A0E26
:10DD00007A6302D02A0E07D00B0E7A6302D02B0E54
:10DD100002D0300E7A257A6FE6500F0B300F7B6FF2
:10DD2000E7380F0B300F7C6FE6500F0B300F7D6F15
:10DD3000E7380F0B300F7E6FE6500F0B300F7F6F01
:10DD4000E7380F0B300F806FE6500F0B300F816FED
:10DD50003A0E7A611AD07AC0EEFF7B6116D07BC092
:10DD6000EEFF7C6112D07CC0EEFF7D610ED07DC0E5
:10DD7000EEFF7E610AD07EC0EEFF7F6106D07FC0DD
:10DD8000EEFF806102D080C0EEFF2C0EEE6E81C0EF
:10DD9000EEFF0D0EEE6E87EC6FF0FC2F99D71200A0
:10DDA000400EFC6F15EE00F00BEE00F04C0EEE6E28
:10DDB000530EEE6E540EEE6ED880410EFC55846FFD
:10DDC0007CEC61F080C0EEFF81C0EEFF2C0EEE6EA9
:10DDD000E6CF7AF0E6CF7BF0E6CF7CF0E6CF7DF0C1
:10DDE000E6CF7EF0E6CF7FF0E6CF80F0E6CF81F0A1
:10DDF000E6CF79F0E6507A390F0B300FFD6F3C0E0D
:10DE0000FD6127D03B0EFD5DD8B4FD99FDC0EEFF4E
:10DE10007A510F0B300F7A6F3A0E7A611AD07AC0AE
:10DE2000EEFF070EFB6F20EE7BF0DF380F0B300F9D
:10DE3000FD6F3A0EFD610DD0FDC0EEFFDE500F0B01
:10DE4000300FFD6F3A0EFD6104D0FDC0EEFFFB2FD9
:10DE5000ECD779C084F034EC6FF00D0EEE6E87ECE9
:10DE60006FF0FC2FA1D712002C0EEE6E7CEC61F04F
:10DE7000300E7F6303D0806303D004D07FC0EEFFF9
:10DE800080C0EEFF81C0EEFF12002C0EEE6E98EC0B
:10DE900061F0300E7D6307D07E6307D07F6307D0CB
:10DEA000806307D008D07DC0EEFF7EC0EEFF7FC04C
:10DEB000EEFF80C0EEFF81C0EEFF1200FA6F2C0E65
:10DEC000EE6E01D0FA6F200EE75C04E0E6CFEEFFC5
:10DED000FA2FF9D712000BEE00F04F0EEE6E4B0E3C
:10DEE000EE6E0D0EEE6E87EC6FF012000BEE00F092
:10DEF000450EEE6E520EEE6E520EEE6E4F0EEE6E42
:10DF0000520EEE6E0D0EEE6E87EC6FF01200EF6AA1
:10DF1000F96B0BEE00F0A4A8FED7EE5003E06D6E97
:10DF2000F92FF9D7A4A8FED7120041540000000031
:10DF300000004F4B0000000001002B57494E443AAF
:10DF400002002B435245473A03002B4353513A20DA
:10DF500004002B434F50533A05002B4352494E4780
:10DF600006002B434C49503A07002B434D54493A85
:10DF700008002B434D47573A09002B434D53533A62
:10DF80000A002B434D47523A0B002B434D47533A5F
:10DF90000C004E4F20414E530E0042555359000085
:10DFA0000F002B434357413A10002B434D450000CF
:10DFB00011002B4350494E3A12004552524F520025
:10DFC000FF002B57494D454913002B5744574C3AF6
:10DFD00014002B434345443A15002B4343454C4C16
:10DFE00016002B5756523A2017002B574D42533AE2
:10DFF00018000000000000000000415400004154DF
:10E0000045310000415448000000415441000000E7
:10E0100041542B434D45453D3100000041542B43B5
:10E020004C49503D3100000041542B434C49503D78
:10E030003000000041542B434C49523D3000000059
:10E0400041542B434C49523D3100000041542B4375
:10E050004C49523D3200000041542B4950523D3949
:10E0600036303000000041542B4950523D31393296
:10E070003030000041542B4946433D302C300000E5
:10E0800041542B575356473D3100000041542B5704
:10E09000494E443D31303233000041542B57494EF4
:10E0A000443D3F00000041542B43474D52000000C7
:10E0B00041542B5744574C00000041542B57494DB5
:10E0C00045493F00000041542B434345443D302C1B
:10E0D0003300000041542B4343454C4C3D3000007D
:10E0E00041542B4346554E3D3100000041542B57BF
:10E0F0004344503D3100000041542B435245473DBD
:10E100003000000041542B435245473D3100000090
:10E1100041542B435245473D3200000041542B43AC
:10E120004345443D312C3800000041542B435243B9
:10E130003D31000041542B434943423D3200000031
:10E1400041542657000041542B434F50533D30005B
:10E15000000041542B434F50533D320000004154C6
:10E160002B434F50533D332C3000000041542B4380
:10E170004F50533D332C3100000041542B434F503E
:10E18000533F000041542B43434944000000415495
:10E190002B43494D4900000041542B434E554D003F
:10E1A000000041542B434C49523D30000000415483
:10E1B0002B434C49523F000041542B434357413DB0
:10E1C000312C312C3100000041542B4350494E3F3B
:10E1D000000041542B5756523F00000041542B572A
:10E1E0004D42533F000041542B434D45523D2C308E
:10E1F000000041542B4543484F3D312C332C3330E4
:10E200002C383030302C32353000000041542B5344
:10E21000494445543D312C33000041542B53504563
:10E22000414B45523D30000041542B57464D3D3146
:10E230002C333300000041542B5647543D3000002E
:10E2400041542B5647543D343000000041542B5666
:10E2500047523D363400000041542B4543484F3D62
:10E26000312C362C33302C35302C36342C323030A7
:10E270002C3535302C31352C33323736372C353080
:10E2800030302C32373438342C33383639372C3759
:10E290003331312C3400000041542B534944455450
:10E2A0003D30000041542B535045414B45523D30C9
:10E2B000000041542B57464D3D312C3333000000B4
:10E2C00041542B4543484F3D312C332C33302C38AF
:10E2D0003030302C32353600000041542B53494445
:10E2E00045543D312C33000041542B535045414B94
:10E2F00045523D31000041542B57464D3D312C33A2
:10E300003300000041542B43534D533D3000000077
:10E3100041542B434D47463D3100000041542B43AF
:10E320004E4D493D322C312C302C302C3000000029
:10E3300041542B434D47443D000041542B434D472E
:10E34000443D312C3400000041542B434D47523D95
:10E35000000041542B434D53533D000041542B4387
:10E360004D47573D000041542B434D47533D00005E
:10E3700041542B43484C443D3200000041542B4350
:10E38000484C443D3132000041542B43484C443DFD
:10E39000330000002A204741544557415920475334
:10E3A0004D20202A4C6F6164657220506173737731
:10E3B0006F726420436F64653A2020202020202063
:10E3C000202020204761746577617920697320726D
:10E3D00065616479746F2074686520757064617418
:10E3E000696E6721536176696E6720506172616D55
:10E3F000657465722052657374617274696E67200A
:10E400004757202047534D3A202D506F7765722093
:10E410004F4E2D202020202D506F776572204F46C3
:10E42000462D20204E6574776F726B3A2020202095
:10E430002020202053494D783A204175746F6D613A
:10E440007469632053494D783A20204D616E75619F
:10E450006C2020204552524F523A20204D6F647557
:10E460006C6520202020206E6F7420616E737765AC
:10E47000722020204552524F523A20202020202046
:10E4800020202020415420436F6D6D616E64206612
:10E4900061696C2E20202053494D202063617264F5
:10E4A00020202020206973206E6F742070726573A5
:10E4B000656E742020207761732072656D6F7665BC
:10E4C00064202020202077617320696E7365727448
:10E4D0006564202020202020496E736572742020FE
:10E4E00020202020496E736572742053494D2020EE
:10E4F000636172644E6574776F726B20776173200D
:10E500006C6F737447534D3A202020202D496E695B
:10E51000742D2020204E6574776F726B2064656EB9
:10E5200069656420204368616E67652074686520B2
:10E5300053494D202053494D20756E6B6E6F776E99
:10E54000202020204E6574776F726B2069732066DF
:10E550006F756E642020204E6574776F726B20207B
:10E560002020202020776173206E6F7420666F75E5
:10E570006E642020526F616D696E6720697320663A
:10E580006F756E644E6574776F726B3A20756E6B43
:10E590006E6F776E4E6574776F726B3A2020202015
:10E5A0002020202053494D783A2053657474696EB9
:10E5B00067202020204D616E75616C2053656C656D
:10E5C000637420204E6574776F726B3A2020202090
:10E5D000202020204E6574776F726B3A2020202017
:10E5E00020202020202069732073656C656374658A
:10E5F0006420202020206E6F7420616C6C6F776522
:10E600006420202020436F6465206F66204E65746F
:10E61000776F726B2020697320616473656E742E4E
:10E6200020202020204E6574776F726B7320636FFB
:10E6300064657320202061726520616273656E7469
:10E6400020202020566F69636520524154453A7856
:10E65000782C787820202047534D2042616E64202A
:10E660003F20202020456E746572205061737377BF
:10E670006F726420496E76616C69642050617373B7
:10E68000776F72645374657020323A20436F6D6DFA
:10E69000616E6420202020697320696E76616C6948
:10E6A000642E20204469616C3A2046585320506FF4
:10E6B0007274202052696E673A20202047534D2EF5
:10E6C00053494D314469616C3A20202047534D2E07
:10E6D00053494D3143616C6C3A20202047534D2EF5
:10E6E00053494D31576169743A20202047534D2ECC
:10E6F00053494D3154616C6B3A20202047534D2EC5
:10E7000053494D31202047534D204469616C696E57
:10E710006720202020446972656374204469616C1D
:10E72000696E672E204F6E6C7920546F6E652044A1
:10E7300069616C2E202020205052495641544520BA
:10E7400020202020434944206973206E6F74206686
:10E750006F756E644469616C3A2046584F20506F63
:10E760007274202054616C6B3A2046584F20506FD1
:10E77000727420204469616C3A20464F4C4C4F57CC
:10E78000204D452054616C6B3A20464F4C4C4F57FE
:10E79000204D45204469616C3A6E6F74207375702A
:10E7A000706F727420205245504C4143494E4720AF
:10E7B00053494D2053494D313A206C6F6164696E65
:10E7C0006720202053494D323A206C6F6164696E96
:10E7D000672020204572726F72206F66205265613B
:10E7E0006464722E4D656E75202320312E302020FA
:10E7F0002020202020202046585320504F525420C3
:10E80000202020204D656E75202320322E302020C0
:10E810002020202020202047534D204E4554574F84
:10E82000524B20204D656E75202320332E30202042
:10E830002020202020202046584F20504F52542086
:10E84000202020204D656E75202320342E3020207E
:10E850002020202020202020474154455741592086
:10E86000202020204D656E75202320352E3020205D
:10E870002020202020534D5320504152414D4554DB
:10E88000455253204D656E75202320312E312020B6
:10E8900020202020507265666978657320666F724B
:10E8A0002047534D4D656E75202320312E32202098
:10E8B000202020202020204449414C205041555305
:10E8C000452020204D656E75202320312E332020D9
:10E8D000202020202047656E65726174696F6E206C
:10E8E000434C492047656E65726174696F6E3A20CA
:10E8F000204F4E2047656E65726174696F6E3A20D5
:10E90000204F4646434C493A202042656C6C636F69
:10E9100072652020434C493A204254204F6E2D68A6
:10E920006F6F6B20434C493A20562E323320202003
:10E9300020202020434C493A202020202020202045
:10E94000202020204D656E75202320312E3420207C
:10E95000202020205245564552534520504F4C41CF
:10E9600052495459237878782020666F7220534991
:10E970004D3A207820507265666978203A78787828
:10E9800078787878204469616C6C696E6720506192
:10E99000757365202020782E78207365636F6E6410
:10E9A000732020205265766572736520506F6C610C
:10E9B00072697479547970653A2044697361626C44
:10E9C00065202020547970653A4261742E52657634
:10E9D00065727365547970653A44626C2E5265763F
:10E9E0002E506F6C547970653A427265616B204CA1
:10E9F000696E65203130306D7320782054696D6503
:10EA00003A2020204D656E75202320322E312020A3
:10EA10002020202020554E4C49535445442043414A
:10EA20004C4C202020556E6C6973746564204361E2
:10EA30006C6C202020416363657074202D20656E0E
:10EA400061626C6520416363657074202D64697335
:10EA500061626C6520416363657074202D20202005
:10EA6000202020204D656E75202320322E3220205C
:10EA70002020202047534D20414343455353204DF0
:10EA80004F44453A4469726563746C7920746F2011
:10EA9000465853204469726563746C7920746F2002
:10EAA00046584F2047534D2F46584F2043616C6CBA
:10EAB0004261636B2047534D20436F6E66657265FC
:10EAC0006E63652020202020202020202020202070
:10EAD000202020204175746F6469616C206E756D13
:10EAE000626572204D656E75202320322E33202002
:10EAF0002020202020205245504541542043414CA5
:10EB00004C2020205265706561742063616C6C201C
:10EB100046584F2066726F6D2047534D3A20656E00
:10EB200061626C6566726F6D2047534D3A6469731C
:10EB300061626C654D656E75202320322E34202075
:10EB40002020202020202043414C4C4241434B2098
:10EB5000202020202043414C4C4241434B20534530
:10EB60005455502043616C6C6261636B3A656E6111
:10EB7000626C652043616C6C6261636B3A646973BB
:10EB800061626C6543616C6C6261636B3A2020204A
:10EB90002020202043414C4C4241434B2077696C5C
:10EBA0006C2062657669613A20202047534D202011
:10EBB000202020207669613A20202046584F2020CE
:10EBC000202020207669613A20202020202020204B
:10EBD000202020202041646465642043414C4C4245
:10EBE00041434B2076696120534D53203A64697349
:10EBF00061626C6576696120534D53203A20656EE1
:10EC000061626C6576696120534D53203A20202063
:10EC1000202020204D656E75202320322E352020A7
:10EC20002020202020414343455353207669612012
:10EC30004C495354204163636573732076696120A6
:10EC40004C697374766961204C4953543A202020F2
:10EC500020202020766961204C4953543A20656E6B
:10EC600061626C65766961204C4953543A646973FA
:10EC700061626C654D656E75202320322E36202032
:10EC80002020202047534D204E554D4245525320C1
:10EC90004C49535447534D204E756D626572732035
:10ECA0004C6973746B65793A2A2D4164642C232D69
:10ECB000456469742378783A53544154453D203073
:10ECC000303030304D61782E20616D6F756E74205C
:10ECD0006F662020746865206E756D6265727320A2
:10ECE0003D2036344D656E75202320322E3720208E
:10ECF000202020202052494E474241434B20544F70
:10ED00004E4520202052696E674261636B20546F2C
:10ED10006E65202066726F6D2047534D3A646973AB
:10ED200061626C6566726F6D2047534D3A656E6126
:10ED3000626C652066726F6D2047534D3A2020202B
:10ED4000202020204D656E75202320322E38202073
:10ED500020202020434C495220616E6420505249AB
:10ED60005641544520204D79204E756D6265723AAA
:10ED70002020202020736574206279204E657477EE
:10ED80006F726B202064697361626C6564206E75BC
:10ED90006D6265722020656E61626C6564206E75BF
:10EDA0006D626572507269766174652063616C6C26
:10EDB00020746F204C6F63616C204C6E3A656E61FD
:10EDC000626C65204C6F63616C204C6E3A646973B1
:10EDD00061626C654C6F63616C204C6E3A20202040
:10EDE000202020204D656E75202320322E392020D2
:10EDF00020202020204E45542F43454C4C20534585
:10EE00004C454354204E4554574F524B2053454C8C
:10EE1000454354202020204175746F2053656C6554
:10EE20006374202020506572696F646963205365A4
:10EE30006C65637478204E6574776F726B3A20202E
:10EE400020202020506572696F642F7365633A201B
:10EE500020202020204D616E75616C2053656C650B
:10EE600063742020204D616E75616C2053656C6564
:10EE7000637420204E6574776F726B3A20202020D7
:10EE800020202020202043454C4C2053454C454316
:10EE90005420202043656C6C2053656C656374209E
:10EEA00066726F6D4E6574776F726B3A202020200A
:10EEB000202020202020204175746F2053656C6530
:10EEC0006374202020506572696F64696320536504
:10EED0006C6563745072643D78787878782C5278D9
:10EEE0003D787878204D616E75616C2053656C6556
:10EEF000637420204552524F523A20202020202077
:10EF000020202020202043656C6C2053656C6563B5
:10EF1000742020207820434C3A787878782C5278E6
:10EF20003A7878784E3A7878787878782C43483AF6
:10EF3000787878782053656C6563746564204365E0
:10EF40006C6C20206973206E6F7420617661696C2F
:10EF500061626C6557616974696E673A2020202090
:10EF600020202020202043656C6C2053656C656355
:10EF7000742020202053656C6563746564204365AC
:10EF80006C6C202020202020776173207365742E04
:10EF9000202020204D656E75202320332E31202027
:10EFA000202020202046584F2041434345535320E2
:10EFB0004D4F444546584F20416363657373204D60
:10EFC0006F64653A4469726563746C7920746F206C
:10EFD000465853204469726563746C7920746F20BD
:10EFE00047534D202027464F4C4C4F57204D452727
:10EFF0002020202020202020202020202020202011
:10F00000202020202047534D2053656C6563746990
:10F010006F6E202062792050726566697865733A58
:10F020002059455362792050726566697865733A54
:10F0300020204E4F20202020546F205465737420D0
:10F04000202020204E756D626572204C6973743AE1
:10F05000205945534E756D626572204C6973743A40
:10F0600020204E4F4D656E75202320332E322020F8
:10F0700020202020202027464F4C4C4F57204D4524
:10F0800027202020202027466F6C6C6F77204D654D
:10F09000272020202752696E677327204E756D62E6
:10F0A00065723A20466F6C6C6F77204D65274E7500
:10F0B0006D6265724D656E75202320332E332020DE
:10F0C0002020202020204449414C494E47204D4FCC
:10F0D00044452020204D696E2E204469616C6C6986
:10F0E0006E672020204469676974733A20202020CD
:10F0F00020207878204D61782E204469616C6C69FD
:10F100006E672020204469676974733A20202020AC
:10F1100020207878204469616C6C696E67205061AA
:10F12000757365202020782E78207365636F6E6478
:10F13000732020202054696D652057616974696EC1
:10F1400067206F666469616C6C696E6728736563BC
:10F15000293A7878205053544E2F4578742E204CFD
:10F16000696E65204469616C696E6720203A20549D
:10F170006F6E65204469616C696E6720203A20508B
:10F18000756C7365202020436F756E747279202032
:10F190002020202020436F646520203A202020205A
:10F1A000202020204E6174696F6E616C204469726A
:10F1B000656374204469616C696E672F4E44443AFC
:10F1C000202020205061757365206166746572206F
:10F1D0006469616C204E44442028312073656320AB
:10F1E0002A293A204D656E75202320332E342020A5
:10F1F000202020205053544E2F4578742E4C2054FC
:10F200006F6E657320204275737920546F6E653A76
:10F21000202020204F4E2F4F46463A2035303020B8
:10F220006D7365632052656F7264657220546F6EF2
:10F23000653A20204F4E2F4F46463A203235302037
:10F240006D7365634D656E75202320332E35202048
:10F25000202020202052494E4720504152414D4508
:10F26000544552532052696E672046726571756528
:10F270006E63792020202020202020203A207878DA
:10F280007820487A4D656E75202320342E31202059
:10F290002020202020204761696E20436F6E747209
:10F2A0006F6C2020537065616B6572202020203ABE
:10F2B000202D78204D6963726F70686F6E65203AFB
:10F2C000202B78204D656E75202320342E3220208F
:10F2D00020202020566F6963652052617465205498
:10F2E000797065204F757420436F64696E672020C4
:10F2F0003A202020496E20436F64696E67202020E9
:10F300003A202020205468697320566F6963652075
:10F31000526174652020206E6F7420737570706F59
:10F3200072742E204D656E75202320342E332020DC
:10F330002020202020202047534D2042616E642051
:10F34000202020204672657175656E6379204261C8
:10F350006E643A204D6F6E6F3A2020202038353091
:10F36000204D487A4D6F6E6F3A202020393030455D
:10F37000204D487A4D6F6E6F3A2020203138303062
:10F38000204D487A4D6F6E6F3A2020203139303051
:10F39000204D487A4475616C3A3835302F31393018
:10F3A000304D487A4475616C3A3930302F313830FD
:10F3B000304D487A4475616C3A3930302F313930EC
:10F3C000304D487A2020202020202020202020207E
:10F3D0002020202020546869732047534D2042612B
:10F3E0006E64202020206E6F7420616C6C6F7765D6
:10F3F000642E20204D656E75202320342E3420206D
:10F400002020202053455454494E47205041535307
:10F41000574F524420456E746572206E65772050B8
:10F42000535720204D656E75202320342E35202023
:10F430002020202053455454494E472050494E2007
:10F44000434F44452020202053657474696E672023
:10F450002020202050494E20434F444520666F72A3
:10F460002053494D4D656E75202320342E362020C3
:10F4700020202020202020205550444154494E4730
:10F48000202020204D656E75202320342E3720202B
:10F49000202020204D6F64756C6520494420284D44
:10F4A000494429204368616E67696E67204D49446D
:10F4B0002020202020202020776173206661696C45
:10F4C00065642021202043757272656E74204D4959
:10F4D000442020204552524F523A20202020202004
:10F4E0002020202052656164696E67206F66204D80
:10F4F000494421204368616E67696E67206F66200A
:10F500004D494420636F6E6669726D3A2020202059
:10F5100020202020456E746572206E6577204D494D
:10F52000443A20204D49442073686F756C6420680C
:10F53000617665206F662031342F3135206469672C
:10F540006974732E2053657474696E67206F66202A
:10F550004D4944204368616E67696E67206F66207D
:10F560004D4944202077617320636F6D706C657422
:10F5700065642021436F6E6669726D207468652032
:10F580006F6C64204D4944205053573A202020206E
:10F590002020202020456E74657220746865206EDE
:10F5A000657720204D4944205053573A2020202091
:10F5B0002020202020204E6577204D4944205053A4
:10F5C000572020202020207761732073657421202C
:10F5D00020202020456E7465726564204D494420CA
:10F5E0005053572020697320494E56414C494420BE
:10F5F00021212120456E7465726564206E65772037
:10F60000505357202077617320756E636F72726557
:10F6100063742E204D656E75202320342E382020F3
:10F6200020202020524F5554455220574F524B20F6
:10F630004D4F444520576F726B204D6F64653A20E3
:10F64000202020202020566F696365204D6F64655F
:10F650002020202020202044617461204D6F6465AB
:10F66000202020202020202020202020202020209A
:10F67000202020202020536176696E6720202020E2
:10F6800020202020202020504152414D45544552F9
:10F6900053202020202047534D207C2054656C2E81
:10F6A0004C696E6520206E6F742070726573656E94
:10F6B0007420202020496E636F6D696E672043615E
:10F6C0006C6C20202020746F2046584F20506F72A1
:10F6D000742E202046584F3A2020496E636F6D6982
:10F6E0006E67202020202020202020202020202085
:10F6F0002020202052696E673A4E6574776F726BD6
:10F700002047534D205053544E2F46585320697371
:10F71000206E6F74636F6E6E656374656420746FC2
:10F720002046584F205053544E2F4658532020699E
:10F7300073202020636F6E6E656374656420746F40
:10F740002046584F466F6C6C6F77204D65274E757D
:10F750006D626572206973206E6F742070726573BC
:10F76000656E742120446973636F6E6E656374699E
:10F770006F6E20202066726F6D2046585320506FA8
:10F780007274202020446973636F6E6E65637469C0
:10F790006F6E20202066726F6D2046584F20506F8C
:10F7A0007274202020446973636F6E6E65637469A0
:10F7B0006F6E20202066726F6D2043454C4C554C77
:10F7C0004152202046584F2043616C6C20746F20BA
:10F7D00047534D204175746F6469616C20746F20CC
:10F7E00046584F202046584F2F204578742E204CE5
:10F7F000696E652077617320646973636F6E6E65EF
:10F800006374656443616C6C4261636B207669610B
:10F810002046584F2047534D206E6F7420616E7301
:10F8200077657220202047534D20496E636F6D69C4
:10F830006E6720202063616C6C20776173206465A3
:10F840006E696564436C6261636B3A2047534D2E69
:10F8500053494D782053494D20697320626C6F6382
:10F860006B65642E53494D2050494E207265717569
:10F870006972656453657474696E672050494E20DF
:10F8800053494D7850494E2053494D3A202020206D
:10F89000202020204572726F723A3E203820646921
:10F8A0006769747320496E636F7272656374205068
:10F8B000494E202053494D2050554B20726571759B
:10F8C00069726564205245504C4143452053494D6F
:10F8D00020212121202020526563656976656420FE
:10F8E000202020204552524F523A20202020202014
:10F8F0002020202053494D31206973207072657398
:10F90000656E742E456D70747920736F636B6574CA
:10F9100020312E2053494D32206973207072657357
:10F92000656E742E456D70747920736F636B6574AA
:10F9300020322E204C6F6164696E672074686520E8
:10F9400053494D314C6F6164696E6720746865205E
:10F9500053494D3246584F206E6F7420666F756E56
:10F96000642E202044656E6965642046584F20430C
:10F97000616C6C2044656E6965642047534D20437B
:10F98000616C6C2E202053494D206661696C757244
:10F99000652E2020205245504C4143452053494D6F
:10F9A00020212121202020204661696C757265206C
:10F9B000202020206F6620737769746368696E6702
:10F9C0002053494D2053494D207265717569726508
:10F9D000206F66206F7468657220706172616D655A
:10F9E000746572212050756C7365206469616C6C5C
:10F9F000696E673A206D757374206265206469676B
:10FA00006974732020496E6974696C697A617469DC
:10FA10006F6E202020206F6620534D53204D4F44A1
:10FA20004520202052656164696E6720534D532044
:10FA30006661696C6973206E6F7420636F6E6669AE
:10FA4000726D656420636F6D6D616E6420657272A6
:10FA50006F72202020204C697374206973206675B2
:10FA60006C6C2020534D53206E6F74207072697639
:10FA70006174652020776173206E6F7420666F75E6
:10FA80006E642020436C6F7365642043616C6C620C
:10FA900061636B204D656E75202320352E3120204B
:10FAA00020202020434F4E54524F4C207669612035
:10FAB000534D53204D656E75202320352E32202066
:10FAC0002020202050726976617465205061737324
:10FAD000776F726453657474696E6720666F722005
:10FAE00020534D53436F6E6669726D3A202020207B
:10FAF000202020202020456E7465726564205053BC
:10FB00005720202020697320494E56414C494420FB
:10FB100021212120436F6E6669726D206F6C642015
:10FB20005053573A20456E746572206E65772050A9
:10FB30005357203A4E65772050524956415445203C
:10FB400050535720202020776173207365742E2036
:10FB500020202020436F6E74726F6C206279204CDD
:10FB60004953542076696120534D53203A64697398
:10FB700061626C6576696120534D53203A656E6110
:10FB8000626C652076696120534D53203A20202015
:10FB90002020202020436F6E6669726D20206163F3
:10FBA00074696F6E76696120534D53203A646973AE
:10FBB00061626C6576696120534D53203A656E61D0
:10FBC000626C65202050726976617465206E756D77
:10FBD00062657220666F7220534D53203A646973D8
:10FBE00061626C65666F7220534D53203A656E6199
:10FBF000626C6520456E7465726564206E65772061
:10FC0000505357202077617320756E636F72726551
:10FC100063742E2020534D5320436F6E6669726DBE
:10FC2000696E67202020776173206661696C656466
:10FC30002E2020202050726976617465204E756DEB
:10FC40006265722020436F6E74726F6C2044696726
:10FC500069747320536572766963652053657474A3
:10FC6000696E672E53657276696365205365747497
:10FC7000696E672E436F6E6669726D3A2020202090
:10FC8000202020202020456E74657265642050532A
:10FC90005720202020697320494E56414C4944206A
:10FCA000212121202053657276696365204E756D90
:10FCB0006265722020544553542052494E472046D5
:10FCC000584F2020506572696F643A202020202010
:10FCD00020206D732020534D5320434F4E54524FDC
:10FCE0004C202020202020697320636C6F73656492
:10FCF0002E202020464D453A204E4F5420414E5351
:10FD000057455220464D453A204E4F5420434152CC
:10FD100052494552464D453A2020425553592020DC
:10FD200020202020464D453A4E6574776F726B2037
:10FD30006C6F737352413A20204E4F5420414E5302
:10FD40005745522052413A20204E4F5420434152B1
:10FD50005249455252413A202020425553592020C1
:10FD60002020202052413A204E6574776F726B201C
:10FD70006C6F73735254523A204E4F5420414E537D
:10FD8000574552205254523A204E4F54204341522C
:10FD9000524945525254523A20204255535920203C
:10FDA000202020205254523A4E6574776F726B2097
:10FDB0006C6F7373434C423A204E4F5420414E5364
:10FDC00057455220434C423A204E4F542043415213
:10FDD00052494552434C423A202042555359202023
:10FDE0002000434C423A4E6574776F726B206C6F03
:10FDF0007373434F4E464552454E43453A20436147
:10FE00006C6C436F6E666572656E6365206D6F64C2
:10FE1000652020207761732066696E697368656468
:10FE20002E20434F4E464552454E43453A2057619A
:10FE30006974434F4E464552454E43453A204275FC
:10FE40007379434F4E462E3A4E6F7420416E73774E
:10FE50006572434F4E464552454E43453A205461E4
:10FE60006C6B20436F6E666572656E6365204D6FC7
:10FE70006465202020204552524F5220212121200C
:10FE800020202020202047534D2043616C6C2020EF
:10FE9000202020206E6F7420616C6C6F7765642E5B
:10FEA00020202050726566697820776173206E6F1C
:10FEB000742020666F756E6420696E207461626CB8
:10FEC000652E4552524F523A20205365747570206A
:10FED0006F667370656564203D3139323030206261
:10FEE000707352342E30202D44415441204D4F44E4
:10FEF000452D20202020313932303020627073208F
:10FF000020204552524F523A2020274543484F2740
:10FF1000202020202052455354415254494E47201E
:10FF200020202743616C6C4261636B27206D6F64F6
:10FF3000652020776173206E6F74207365742121B2
:10FF400021202053494D206E6F7420737570706F9F
:10FF500072742743616C6C6261636B27204D6F6420
:10FF600065204572726F723A20534D53204D6F6475
:10FF7000652020696E697469616C697A6174696F62
:10FF80006E204669726D776172652056657273697D
:10FF90006F6E50726F6772616D6D20566572736916
:10FFA0006F6E5254522D342E39302D52342E302D46
:10FFB000422D475734393052342E302D32353033BC
:02FFC0003038D7
:06FFFA0082FFD5D75A0476
:020000040030CA
:0600010022001E83838033
:0600080000800F800F4094
:0200000400F00A
:10000000052FFFF1050FFFF2FFFFFFF1FFFFFFF1EB
:10001000FFFFFFF1FFFFFFF1FFFFFFF1FFFFFFF128
:10002000FFFFFFF1FFFFFFF1FFFFFFF1FFFFFFF118
:10003000FFFFFFF1FFFFFFF1FFFFFFF1FFFFFFF108
:10004000FFFFFFF2FFFFFFF2FFFFFFF2FFFFFFF2F4
:10005000FFFFFFF2FFFFFFF2FFFFFFF2FFFFFFF2E4
:10006000FFFFFFF2FFFFFFF2FFFFFFF2FFFFFFF2D4
:10007000FFFFFFF2FFFFFFF2FFFFFFF2FFFFFFF2C4
:10008000FFFFFFFFFFFFFFFF00FFFFFFFFFFFFFF7F
:10009000FFFF00FFFFFFFFFFFFFFFFFF00FFFFFF6E
:1000A000FFFFFFFFFFFF00FFFFFFFFFFFFFFFFFF5F
:1000B00000FFFFFFFFFFFFFFFFFF00FFFFFFFFFF4E
:1000C000FFFFFFFF00FFFFFFFFFFFFFFFFFF00FF3E
:1000D000FFFFFFFFFFFFFFFF00FFFFFFFFFFFFFF2F
:1000E000FFFF00FFFFFFFFFFFFFFFFFF00FFFFFF1E
:1000F000FFFFFFFFFFFF00FFFFFFFFFFFFFFFFFF0F
:1001000000FFFFFFFFFFFFFFFFFF00FFFFFFFFFFFD
:10011000FFFFFFFF00FFFFFFFFFFFFFFFFFF00FFED
:10012000FFFFFFFFFFFFFFFF00FFFFFFFFFFFFFFDE
:10013000FFFF00FFFFFFFFFFFFFFFFFF00FFFFFFCD
:10014000FFFFFFFFFFFF00FFFFFFFFFFFFFFFFFFBE
:1001500000FFFFFFFFFFFFFFFFFF00FFFFFFFFFFAD
:10016000FFFFFFFF00FFFFFFFFFFFFFFFFFF00FF9D
:10017000FFFFFFFFFFFFFFFF00FFFFFFFFFFFFFF8E
:10018000FFFF00FFFFFFFFFFFFFFFFFF00FFFFFF7D
:10019000FFFFFFFFFFFF00FFFFFFFFFFFFFFFFFF6E
:1001A00000FFFFFFFFFFFFFFFFFF00FFFFFFFFFF5D
:1001B000FFFFFFFF00FFFFFFFFFFFFFFFFFF00FF4D
:1001C000FFFFFFFFFFFFFFFF00FFFFFFFFFFFFFF3E
:1001D000FFFF00FFFFFFFFFFFFFFFFFF00FFFFFF2D
:1001E000FFFFFFFFFFFF00FFFFFFFFFFFFFFFFFF1E
:1001F00000FFFFFFFFFFFFFFFFFF00FFFFFFFFFF0D
:10020000FFFFFFFF00FFFFFFFFFFFFFFFFFF00FFFC
:10021000FFFFFFFFFFFFFFFF00FFFFFFFFFFFFFFED
:10022000FFFF00FFFFFFFFFFFFFFFFFF00FFFFFFDC
:10023000FFFFFFFFFFFF00FFFFFFFFFFFFFFFFFFCD
:1002400000FFFFFFFFFFFFFFFFFF00FFFFFFFFFFBC
:10025000FFFFFFFF00FFFFFFFFFFFFFFFFFF00FFAC
:10026000FFFFFFFFFFFFFFFF00FFFFFFFFFFFFFF9D
:10027000FFFF00FFFFFFFFFFFFFFFFFF00FFFFFF8C
:10028000FFFFFFFFFFFF00FFFFFFFFFFFFFFFFFF7D
:1002900000FFFFFFFFFFFFFFFFFF00FFFFFFFFFF6C
:1002A000FFFFFFFF00FFFFFFFFFFFFFFFFFF00FF5C
:1002B000FFFFFFFFFFFFFFFF00FFFFFFFFFFFFFF4D
:1002C000FFFF00FFFFFFFFFFFFFFFFFF00FFFFFF3C
:1002D000FFFFFFFFFFFF00FFFFFFFFFFFFFFFFFF2D
:1002E00000FFFFFFFFFFFFFFFFFF00FFFFFFFFFF1C
:1002F000FFFFFFFF00FFFFFFFFFFFFFFFFFF00FF0C
:1003000000320000030A323203000032000F32963E
:100310000000000501013000400C100E30202020AC
:10032000202000000000202020202020000020208D
:1003300020202020100E202020202020100E202001
:1003400020202020100E202020202020100E3030D1
:10035000303034323338363738333132333435365F
:1003600037383132333435363738202020202020BA
:10037000202020202020202020202020202020207D
:10038000202020202020202020202020202020206D
:10039000202020202020202020202020202020205D
:1003A000202020202020202020202020202020204D
:1003B000202020202020202020202020202020203D
:1003C00020202020202020202020000100010001EA
:0E03D000000132323232191919196496009662
:0403FC00FAFF000004
:00000001FF
